:0900000C312E332E302E32383033
:1000000AF81319FB3F341AF53A464A2904442207E1
:1000000A25280A4A3726290F343A123C40151C255E
:1000000A201D201F25212521685C4E196E616B5029
:1000000A286853572C3C34353A3E39393D413C39FE
:1000000A3E484944494444484C47445252544F5448
:1000000A4F4F5357524F565B5E5A5F5A5A5E625D64
:1000000A5A7D5F815288777A608585637D8166AF84
:0600000AA39560968588B5
:020000040800F2
:40800000F0C202200107080813070808E136090817070808190708081B07080800000000000000000000000000000000498300081F070808000000000D84000881840008C2
:408040002507080825070808250708082507080825070808250708082507080825070808250708082507080825070808A95E0508B35E050825070808BF5E0508CB5E05089E
:40808000D75E0508E35E050803420508B94705088B48050825070808250708082507080825070808250708082507080825070808F59705080198050825070808F38505084D
:4080C00003860508138605081D8605089D960508A7960508A5750508FF7505080976050825070808250708082507080825070808250708082507080825070808EF5E0508D8
:4081000025070808250708080B980508B1960508137605081D7605082507080879990508FB5E0508055F0508115F05081D5F0508295F0508250708082507080821480508D2
:4081400001490508774905082507080825070808355F0508415F05084D5F050827760508278605083786050825070808250708082507080825070808250708080000000002
:408180002507080825070808317605083B760508BB96050825070808250708082507080800000000000000002507080800F002F800F087F80AA090E8000C82448344AAF1D8
:4081C0000107DA4501D100F07CF8AFF2090EBAE80F0013F0010F18BFFB1A43F0010318471CCB18005CCB18000A444FF0000C10F8013B13F0070408BF10F8014B1D1108BFEB
:4082000010F8015B641E05D010F8016B641E01F8016BF9D113F0080F1EBF10F8014BAD1C0C1B09D16D1E58BF01F801CBFAD505E014F8016B01F8016B6D1EF9D59142D6D37C
:40824000704700000023002400250026103A28BF78C1FBD8520728BF30C148BF0B607047662910F0E48B692908F05E8C642908F05B8C752908F0588C782908F0918C632984
:4082800009F0B58C732909F0BA8C002070471FB590F05FFB9DE8030089F0CFF988F0ADFE89F0AEF90400002000218FF027FC401C6060002000218FF037FCE0601FBD10B541
:4082C00010BD8AF0A9F81146FFF7E1FF0FF08DFC8AF044FB03B4FFF7F2FF03BC8AF074FB80F309887047EFF309807047684680F3098804480078C00714BF0220032080F33D
:40830000148870470CF10A08DFF818C0EFF305831B0618BF6047EFF31483DB0708BF604700DF7047C76B0908DFF818C0EFF305831B0618BF6047EFF31483DB0708BF604700
:4083400000DF7047CD6D0908EFF30980816911F8021C01B142E010B590E80F10E047BDE81040EFF3098C254B93E80600914232D041B91EF0100F16D12149086820F001001E
:40838000086010E00CB41EF0100F06BF2CED108A0323012381F826302CE9F00FC1F82CC08FF0C6F80CBC1A60D2F82CC0BCE8F00F92F8263013F0020F1ABFBCEC108A6FF0E8
:4083C000120E6FF0020E8CF3098813F0010F08BF704792F82500CCF80000704710B5094A1268914209D8084C54F8214090E80F10A047EFF3098C8CE80F0010BDD81200208D
:4084000034EF00E0D0360908D036090810B58EF027FFBDE81040194B93E80600914208BF70470CB4EFF3098C1EF0100F06BF2CED108A0223002381F826302CE9F00FC1F8B7
:408440002CC08FF075F80CBC1A60D2F82CC0BCE8F00F92F8263013F0020F1ABFBCEC108A6FF0120E6FF0020E8CF3098813F0010F1CBF92F82530CCF800307047D8120020FA
:4084800010B58FF025F9C4E710B58EF09BFB8FF01FF9BEE70B49D1F800C04A685CF8043B1068184442F8040B8C4528BFA1F1DC0C8A4228BFA1F1DC02C1F800C04A6020F0D3
:4084C00000407047E4BE022010B5044620465DF020FA10BD07B588B00020069000210A98017008980078CE2882F00986810000BF794449688F440000380300003C03000030
:40850000740300000604000084040000020500001E06000090060000062C0000060700005C070000E607000012080000DC080000A60900003A0B0000100C0000660E000060
:40854000062C0000062C00002E0F00007C10000098100000FE10000064110000062C0000941200006A1300004E140000D4160000A8170000761800001C190000EA1900007D
:40858000B81A0000062C00005E1B0000062C00003C1C0000581C0000081D0000281D00008C270000B8270000EC270000062C0000062C0000481D0000BC1500004816000039
:4085C0005A1D0000B21D0000EE1D0000301E0000861E0000C01E0000062C0000062C0000062C0000001F0000561F0000EC1F0000E620000004210000062C0000062C000096
:40860000062C0000062C0000062C0000062C0000062C0000062C0000062C0000062C000006210000202100003C210000700A0000241500007C150000441500009C15000097
:4086400090210000CA110000062C0000A02100003A22000014220000062C0000062C0000062C0000062C0000062C0000B6070000062C0000062C0000062C0000062C00006A
:40868000062C0000062C00000A200000062C0000C8200000062C0000062C0000062C0000062C0000062C0000062C0000062C0000062C0000062C0000062C0000062C0000EC
:4086C000062C0000062C00004E220000062C000062220000062C000074220000062C0000862200009A220000AE220000C2220000D6220000EA220000FE2200001223000085
:40870000062C0000062C00002623000074230000062C0000062C0000062C000076230000062C0000062C0000D60C0000A00D0000062C0000D823000034240000902400009A
:40874000EC240000482500009E250000F42500004A26000062260000B62600000A270000062C0000062C0000062C00007E270000062C0000062C0000062C0000062C000098
:40878000062C0000062C0000062C0000062C00001C28000036280000062C0000062C00002227000052280000062C0000062C000006290000422900005E2900008E290000EC
:4087C000B6290000062C00002E2A00004A2A0000062C0000062C0000062C0000062C0000062C0000062C0000062C0000062C00004C2A00006C2A0000802A0000062C000024
:40880000A02A00001C2B0000062C0000062C0000762B0000062C0000062C0000E62B0000062C0000062C0000062C00006415000002F066BC13F0ABFE18B101210A980170E0
:4088400013E00898007A03280FD10898807A0490FC4890F8E0040390089800790290DDE9031285F0C9FE0A990870E1E713F08FFEF0BB0898007A03280DD10898807A04903E
:408880000898808880B2FF22039004990CF095FA0A99087032E00898007A012812D10CF08BF90122099902FB010080B204900898807AFF220146039004980CF07EFA0A995E
:4088C00008701BE00898007A022817D10CF074F90122099902FB110080B204900898807AFF220146039004980CF067FA0A9900E001E0087002E001210A98017098E7089837
:40890000007A03280CD10898807A04900898808880B20390049985F02BFE0A9908702AE00898007A012811D184F0E6FB0122099902FB010080B204900898807A0146039043
:40894000049885F015FE0A99087014E00898007A022810D184F0D0FB0122099902FB110080B204900898807A01460390049885F0FFFD0A9908700120069059E70898007A1A
:4089800003280CD10898807A04900898808880B20390049985F005FE0A9908702AE00898007A012811D184F044F80122099902FB010080B204900898807A0146039004986C
:4089C00085F0EFFD0A99087014E00898007A022810D184F02EF80122099902FB110080B204900898807A01460390049885F0D9FD0A990870012006901AE70898406842F205
:408A0000067188420AD00898406846F21E31884204D008984068491C884209D117F06CFB30B101201EF067FB0520FFF74DFD6FE00898007A03280ED1089890ED010AB8EED7
:408A4000C00A8DED040AFF209DED040A0CF098FA0A9908705CE00898007A01282AD142F0D6FB98B90CF058F9DDED090AF8EE600AB7EE001A01EE200A8DED040AFF209DEDF3
:408A8000040A0CF07DFA0A99087041E00CF044F9DDED090AF8EE600A9FED6B1A01EE200A8DED040AFF209DED040A0CF069FA0A9908702DE00898007A022829D142F0A7FB91
:408AC00098B90CF029F9DDED090AF8EE600AB7EE001A01EE600A8DED040AFF209DED040A0CF04EFA0A99087012E00CF015F9DDED090AF8EE600A9FED541A01EE600A8DED2E
:408B0000040AFF209DED040A0CF03AFA0A990870012006908CE613F03AFD80BB0898007A032808D108984068FF2104900CF0BCF90A99087020E00898007A01280CD10CF085
:408B400070F80122099902FB0100FF2104900CF0ABF90A9908700FE00898007A02280BD10CF05FF80122099902FB1100FF2104900CF09AF90A9908700120069003E0FFE748
:408B800001210A98017053E613F001FD90BB0898007A032808D10898808880B204900CF0CDF90A99087022E00898007A01280DD12448B0F894130122099802FB001080B2B1
:408BC00004900CF0BBF90A99087010E00898007A02280CD11B48B0F894130122099802FB101080B204900CF0A9F90A9908700120069003E0FFE701210A98017018E613F03D
:408C0000C6FCE8B90898007A032819D10D4890F878130898406881420BD000200CF033FA00200A4908700A480978405C04900CF00EFA0898007904900CF0F1F90A9908706B
:408C4000F6E50000982400205C8F22404F030010F4B1090813F09BFC00BB0898007A032824D10898007903900DF028F904900CF00AFA0A9908700020F949087008980079DD
:408C800004900DF01BF9172809D1F64890F87803401EC0B2059005980CF0D9F906E0F248EF490978405C04900CF0D1F9C0E513F06EFC98B90898007A03280FD10898406846
:408CC00000280BDD08980079E5490870E6480978405C04900CF0BBF90A990870A8E514F0EDFAFA2810D014F0E9FAFB280CD00898007A032808D10898807A04900898007936
:408D0000039004990CF0D7F992E50898007A032812D1D44890F8E1040490D24890F8E00403900898808800B20290DDE9031212F0FDF80A9908704AE00898007A012821D12A
:408D4000C84890F8E01400F5946000EB8101C54890F8E10431F810200121099801FB002000B20290BF4890F8E1040490BD4890F8E00403900146049A029812F0D7F80A991C
:408D8000087024E00898007A022820D1B54890F8E01400F5946000EB8101B24890F8E10431F810100122099802FB101000B20290AC4890F8E1040490AA4890F8E004039078
:408DC0000146049A029812F0B1F80A990870012006902DE50898007A032812D1A14890F8E10404909F4890F8E00403900898808800B20290DDE9031211F09CFE0A990870F0
:408E00004AE00898007A012821D1964890F8E01400F58C6000EB8101924890F8E10431F810100122099802FB001000B202908D4890F8E10404908B4890F8E0040390014697
:408E4000049A029811F076FE0A99087024E00898007A022820D1834890F8E01400F58C6000EB81017F4890F8E10431F810100122099802FB101000B202907A4890F8E1048B
:408E80000490784890F8E00403900146049A029811F050FE0A99087001200690C8E40898007A032812D16F4890F8E10404906D4890F8E00403900898808800B20290DDE9CD
:408EC000031211F0BFFE0A9908704AE00898007A012821D1634890F8E01400F58D6000EB8101604890F8E10431F810100122099802FB001000B202905A4890F8E104049099
:408F0000584890F8E00403900146049A029811F099FE0A99087024E00898007A022820D1504890F8E01400F58D6000EB81014D4890F8E10431F810100122099802FB101098
:408F400000B20290474890F8E1040490454890F8E00403900146049A029811F073FE0A9908700120069063E40898007A032812D13C4890F8E10404903A4890F8E004039059
:408F80000898808800B20290DDE9031212F017F80A9908704AE00898007A012821D1314890F8E01400F5936000EB81012D4890F8E10431F810100122099802FB001000B267
:408FC0000290284890F8E1040490264890F8E00403900146049A029811F0F1FF0A99087024E00898007A022820D11E4890F8E01400F5936000EB81011A4890F8E10431F80E
:4090000010100122099802FB101000B20290154890F8E1040490134890F8E00403900146049A029811F0CBFF0A990870012006901BE40898007A032818D10A4890F8E1042B
:409040000490084890F8E00403900898808800B20290DDE9031211F033FE0A99087050E04F03001098240020F4B109080898007A012821D1FD4890F8E01400F58E6000EB11
:409080008101FA4890F8E10431F810100122099802FB001000B20290F44890F8E1040490F24890F8E00403900146049A029811F007FE0A99087024E00898007A022820D1D2
:4090C000EA4890F8E01400F58E6000EB8101E74890F8E10431F810100122099802FB101000B20290E14890F8E1040490DF4890F8E00403900146049A029811F0E1FD0A9917
:4091000008700120069038E40898007A032810D1D64890F8E1040490D44890F8E00403900898808800B20290DDE9031211F044FE4AE00898007A012821D1CC4890F8E0148B
:4091400000F58F6000EB8101C84890F8E10431F810200121099801FB002000B20290C34890F8E1040490C14890F8E00403900146049A029811F020FE0A99087024E0089834
:40918000007A022820D1B94890F8E01400F58F6000EB8101B54890F8E10431F810200121099801FB102000B20290B04890F8E1040490AE4890F8E00403900146049A0298E9
:4091C00011F0FAFD0A9908700120069014E40898007A032812D1A54890F8E1040490A34890F8E00403900898808800B20290DDE9031211F0A3FD0A9908704AE00898007AE6
:40920000012821D1994890F8E01400F5916000EB8101964890F8E10431F810200121099801FB002000B20290904890F8E10404908E4890F8E00403900146049A029811F06E
:409240007DFD0A99087024E00898007A022820D1864890F8E01400F5916000EB8101834890F8E10431F810100122099802FB101000B202907D4890F8E10404907B4890F8CC
:40928000E00403900146049A029811F057FD0A990870012006903DE40898007A032810D1724890F8E1040490704890F8E00403900898808800B20290DDE9031211F0BAFD59
:4092C0004AE00898007A012821D1684890F8E01400F5926000EB8101644890F8E10431F810100122099802FB001000B202905F4890F8E10404905D4890F8E0040390014685
:40930000049A029811F096FD0A99087024E00898007A022820D1554890F8E01400F5926000EB8101514890F8E10431F810100122099802FB101000B202904C4890F8E1042B
:4093400004904A4890F8E00403900146049A029811F070FD0A9908700120069013E40898007A032811D1414890F8E10404903F4890F8E0040390089800790290DDE9031255
:4093800011F096FD0A9908704AE00898007A012821D1364890F8E01400F5906000EB8101324890F8E10431F810100122099802FB001000B202902D4890F8E10404902B4825
:4093C00090F8E00403900146049A029811F070FD0A99087024E00898007A022820D1234890F8E01400F5906000EB81011F4890F8E10431F810100122099802FB101000B244
:4094000002901A4890F8E1040490184890F8E00403900146049A029811F04AFD0A990870012006900CE40898007A03287CD108984068F1280CD112F014FB01460490002073
:409440000FF0A1FE1420DFF828C000DF03DF8AE008984068F22811D10648D0F86801014604900220DFF810C000DF7CE098240020D16C090830320020316D090808984068EB
:40948000F32803D1032019F08BFD6CE008984068F7280AD1FE48D0F86801014604904FF40070DFF8F0C300DF5DE008984068F42809D1F748D0F86801014604908020DFF8D0
:4094C000D4C300DF4FE008984068F5280AD1F048D0F86801014604904FF48070DFF8B4C300DF40E008984068F62809D1E848D0F86801014604900120DFF898C300DF32E003
:4095000008984068F8280BD1E148D0F86801014604904FF48060DFF87CC300DF23E003E006210A9801701EE00898007A012809D1D748D0F86801014604900420DFF854C322
:4095400000DF10E00898007A022809D1D048D0F86801014604900820DFF838C300DF02E007210A9801701420FEF7AEFF0D203EF033FC2EE40898007A012802D1002019F033
:409580000FFD1520FEF7A0FF28203EF025FC20E40898007A032808D10898808800B2049008F0FAFF0A99087022E00898007A01280DD1B948B0F8E2140122099802FB001090
:4095C00000B2049008F0E8FF0A99087010E00898007A02280CD1B048B0F8E2140122099802FB101000B2049008F0D6FF0A9908700120069052E40898007A032808D10898CA
:40960000808880B2049009F03CF80A99087022E00898007A01280DD19F48B0F8EC140122099802FB001080B2049009F02AF80A99087010E00898007A02280CD19648B0F8FE
:40964000EC140122099802FB101080B2049009F018F80A990870012006901FE40898007A032808D10898808880B2049009F038F80A99087022E00898007A01280DD18648A4
:40968000B0F8EE140122099802FB001080B2049009F026F80A99087010E00898007A02280CD17D48B0F8EE140122099802FB101080B2049009F014F80A9908700120069039
:4096C00051E40898007A032812D1734890F8E1040490714890F8E00403900898808800B20290DDE9031208F089FF0A9908704AE00898007A012821D1674890F8E01400F2BB
:40970000E44000EB8101644890F8E10431F810100122099802FB001000B202905E4890F8E10404905C4890F8E00403900146049A029808F063FF0A99087024E00898007AC5
:40974000022820D1544890F8E01400F2E44000EB8101514890F8E10431F810100122099802FB101000B202904B4890F8E1040490494890F8E00403900146049A029808F024
:409780003DFF0A9908700120069051E40898007A032814D10898807A04903F4890F8E10403903D4890F8E004029008980079019002A90EC981F0A9F90A9908704EE00898DC
:4097C000007A012823D1344890F8E01400F5737000EB4101304890F8E104095C0122099802FB001001900898807A04902A4890F8E1040390284890F8E00402900146DDE90E
:409800000323019881F081F90A99087026E00898007A022822D1204890F8E01400F5737000EB41011C4890F8E104095C0122099802FB101001900898807A0490164890F881
:40984000E1040390144890F8E00402900146DDE90323019881F059F90A9908700120069051E40898007A03281BD10898807A0490094890F8E1040390074890F8E004029083
:4098800008980079019002A90EC981F0E3F905E030320020316D0908982400200A9908704EE00898007A012823D1FC4890F8E01400F5747000EB4101F84890F8E104095CE5
:4098C0000122099802FB001001900898807A0490F24890F8E1040390F04890F8E00402900146DDE90323019881F0B4F90A99087026E00898007A022822D1E84890F8E0147A
:4099000000F5747000EB4101E44890F8E104095C0122099802FB101001900898807A0490DE4890F8E1040390DC4890F8E00402900146DDE90323019881F08CF90A9908705E
:409940000120069042E40898007A032814D10898807A0490D14890F8E1040390CF4890F8E004029008980079019002A90EC981F016FA0A9908704EE00898007A012823D157
:40998000C64890F8E01400F5757000EB4101C34890F8E104095C0122099802FB001001900898807A0490BD4890F8E1040390BB4890F8E00402900146DDE90323019881F066
:4099C000EEF90A99087026E00898007A022822D1B24890F8E01400F5757000EB4101AF4890F8E104095C0122099802FB101001900898807A0490A94890F8E1040390A74862
:409A000090F8E00402900146DDE90323019881F0C6F90A990870012006903CE40898007A03280AD10898807A0490089800790390049981F0ECFF0A9908702CE40898007A02
:409A400003280AD10898807A0490089800790390049980F063F80A9908701CE40898007A032806D10898007904901EF064F80A99087010E40898007A03280AD10898807A87
:409A80000490089800790390049980F05EF80A99087063E40898007A03280AD10898807A0490089800790390049980F065F80A99087053E40898007A032811D1089890EDA7
:409AC000010AF8EEC00AB2EE041A80EE810A8DED040A9DED040A81F044FF0A9908702CE00898007A012812D182F032F80122099902FB110000EE100AB8EEC00A8DED040A64
:409B00009DED040A81F02DFF0A99087015E00898007A022811D182F01BF80122099902FB010000EE100AB8EEC00A8DED040A9DED040A81F016FF0A990870012006900DE491
:409B40000898007A032811D1089890ED010AF8EEC00AB2EE041A80EE810A8DED040A9DED040A81F02BFF0A9908702CE00898007A012812D181F0F5FF0122099902FB0100FF
:409B800000EE100AB8EEC00A8DED040A9DED040A81F014FF0A99087015E00898007A022811D181F0DEFF0122099902FB110000EE100AB8EEC00A8DED040A9DED040A81F029
:409BC000FDFE0A990870012006902BE40898007A032818D1089890ED010AF8EEC00AB2EE041A80EE810A8DED040A807A03902B4890F8E104029003999DED040A81F096F911
:409C00000A99087046E00898007A01281FD1234890F8E11400F5777000EB8100D0ED000A9DED090AB8EEC00A30EE800A8DED020A0898807A0490194890F8E1040390049952
:409C40009DED020A81F072F90A99087022E00898007A02281ED1114890F8E11400F5777000EB8100D0ED000A9DED090AB8EEC00A30EEC00A8DED020A0898807A0490074845
:409C800090F8E104039004999DED020A81F04EF90A990870012006906BE40000982400200898007A032818D1089890ED010AF8EEC00AB2EE041A80EE810A8DED040A807A7D
:409CC0000390FE4890F8E104029003999DED040A81F00FFA0A99087046E00898007A01281FD1F64890F8E11400F57B7000EB8100D0ED000A9DED090AB8EEC00A30EE800AE7
:409D00008DED020A0898807A0490EC4890F8E104039004999DED020A81F0EBF90A99087022E00898007A02281ED1E44890F8E11400F57B7000EB8100D0ED000A9DED090A0A
:409D4000B8EEC00A30EEC00A8DED020A0898807A0490DA4890F8E104039004999DED020A81F0C7F90A990870012006900FE40898007A032810D10898807A0490CF4890F899
:409D8000E1040390089800790290DDE9031281F0B0FC0A9908703AE00898007A012819D1C64890F8E11400F20440415C0122099802FB001002900898807A0490BF4890F8A8
:409DC000E10403900146049A029881F092FC0A9908701CE00898007A022818D1B74890F8E11400F20440415C0122099802FB101002900898807A0490B04890F8E104039041
:409E00000146049A029881F074FC0A9908700120069022E40898007A032818D1089890ED010AF8EEC00AB2EE041A80EE810A8DED040A807A0390A14890F8E1040290039994
:409E40009DED040A81F06AFA0A99087046E00898007A01281FD1994890F8E11400F5797000EB8100D0ED000A9DED090AB8EEC00A30EE800A8DED020A0898807A04908F4852
:409E800090F8E104039004999DED020A81F046FA0A99087022E00898007A02281ED1874890F8E11400F5797000EB8100D0ED000A9DED090AB8EEC00A30EEC00A8DED020A96
:409EC0000898807A04907D4890F8E104039004999DED020A81F022FA0A9908700120069053E40898007A032818D1089890ED010AF8EEC00AB2EE041A80EE810A8DED040A61
:409F0000807A03906D4890F8E104029003999DED040A81F0E2FA0A99087046E00898007A01281FD1654890F8E11400F57D7000EB8100D0ED000A9DED090AB8EEC00A30EE81
:409F4000800A8DED020A0898807A04905B4890F8E104039004999DED020A81F0BEFA0A99087022E00898007A02281ED1534890F8E11400F57D7000EB8100D0ED000A9DED9D
:409F8000090AB8EEC00A30EEC00A8DED020A0898807A0490494890F8E104039004999DED020A81F09AFA0A9908700120069057E40898007A032810D10898807A04903F48D1
:409FC00090F8E1040390089800790290DDE9031281F02BFC0A9908703AE00898007A012819D1364890F8E11400F20640415C0122099802FB001002900898807A04902F4809
:40A0000090F8E10403900146049A029881F00DFC0A9908701CE00898007A022818D1274890F8E11400F20640415C0122099802FB101002900898807A0490204890F8E104AC
:40A0400003900146049A029881F0EFFB0A9908700120069004E40898007A032814D10898807A0490154890F8E1040390134890F8E004029008980079019002A90EC980F00F
:40A08000A3FC0A99087052E00898007A012827D10A4890F8E01400F5767000EB4101074890F8E104095C0122099802FB001001900898807A0490014802E0000098240020EB
:40A0C00090F8E1040390F94890F8E00402900146DDE90323019880F077FC0A99087026E00898007A022822D1F04890F8E01400F5767000EB4101ED4890F8E104095C012234
:40A10000099802FB101001900898807A0490E74890F8E1040390E54890F8E00402900146DDE90323019880F04FFC0A9908700120069007E40898007A032808D10898807A4C
:40A14000049008980079039004997EF065F864E40898007A032813D10898807A04900898808880B200EE100AB8EE400A8DED030A04989DED030A7DF02EFD0A9908703CE03D
:40A180000898007A01281AD17EF085FAF0EE400AC74890ED851A9DED090AF8EE401AB0EE410A00EEA10A8DED040A0898807A03909DED040A7DF00FFD0A9908701DE0089854
:40A1C000007A022819D17EF066FAF0EE400AB84890ED851A9DED090AF8EE401AB0EE410A00EEE10A8DED040A0898807A03909DED040A7DF0F0FC0A990870012006900CE4B8
:40A200000898007A03280AD10898807A0490089800790390049984F016F80A9908700CE40898007A03280AD10898807A0490089800790390049984F0C9F80A9908700CE423
:40A240000898007A032803D108980079994908700FE40898007A03281DD1944890F8E11400F5777000EB810090ED000A8DED070A9DED070AB5EEC00AF1EE10FA03D19FED28
:40A280008E0A8DED070A4FF0FF319DED070A08207CF069FA08E00898007A28B900219FED870A08207CF05FFA49E40898007A03280FD181F04DFC00EE100AB8EEC00A8DED6E
:40A2C000040A6FF009019DED040A0A207CF04BFA08E00898007A28B900219FED780A08207CF041FA2BE40898007A032812D16F4890F8E11400F57B7000EB810090ED000A55
:40A300008DED040A6FF001019DED040A08207CF02AFA08E00898007A28B900219FED670A08207CF020FA0AE40898007A03281CD15E4890F8E11400F5797000EB810090ED2B
:40A34000000A8DED070A9DED070AB5EEC00AF1EE10FA03D19FED5A0A8DED070A01219DED070A08207CF0FFF908E00898007A28B900219FED520A08207CF0F5F925E40898A8
:40A38000007A03280ED181F0ECFB00EE100AB8EEC00A8DED040A0A219DED040A08467CF0E2F908E00898007A28B900219FED430A08207CF0D8F908E40898007A032811D114
:40A3C0003A4890F8E11400F57D7000EB810090ED000A8DED040A02219DED040A08207CF0C2F908E00898007A28B900219FED330A08207CF0B8F94FE40898007A032808D194
:40A4000008980079FF2104901AF0CAF80A9908701CE00898007A01280AD117F037F9401CC0B2FF2104901AF0BBF80A9908700DE00898007A022809D117F028F9401EC0B2BA
:40A44000FF2104901AF0ACF80A99087024E40898007A032845D10898406858B9134890F8E1040490114890F8E004039004990AF082FA36E008984068012806D10B4890F8A3
:40A48000E10404900AF093F92BE008984068022818D1064890F8E1040490044890F8E0040390049909F097FF1BE0000098240020D027002055010010CDCCCCBD00000000FB
:40A4C000CDCCCC3D0898406803280AD1F74890F8E1040490F54890F8E004039004990AF0A6F843E40898007A032809D108980079049005F082FA0A990870042004F0AEFE78
:40A5000034E40898007A032859D108984068062846D2DFE800F0030E19242F3A012005F0DEF90A990870002005F0C1F90A99087041E0032005F0D3F90A990870832005F0EE
:40A54000B6F90A99087036E0032005F0C8F90A990870872005F0ABF90A9908702BE0032005F0BDF90A9908708A2005F0A0F90A99087020E0042005F0B2F90A9908707820EE
:40A5800005F095F90A99087015E0042005F0A7F90A9908707E2005F08AF90A9908700AE0012005F09CF90A990870002005F07FF90A99087000BF00BF402004F04FFE28E480
:40A5C0000898007A032809D108980079049005F0BBFA0A990870802004F040FE19E40898007A032809D108980079049005F081FA0A990870022004F031FE0AE409E40898E4
:40A60000007A032807D13C21A94886F088FE4FF05FF9A749086363E40898007A032808D1A448D0F86801014604900220DFF888C200DF55E439F0CBFA0899897A88420FD16D
:40A640009E4890F8D80008B9012000E00020049007F0F2F99A480078A8B11CF05EFD12E008984068012808D1002007F0E5F99448007840B11CF051FD05E00898406810B95C
:40A68000012007F0D9F92BE40898007A012802D1022012F0F4FA23E40898007A03280DD1089890ED010AB8EEC00A8DED040A9DED040A05F044F90A99087026E00898007A2A
:40A6C00001280FD17F4890ED020AF7EE000A30EE200A8DED040A9DED040A05F030F90A99087012E00898007A02280ED1754890ED020AF7EE000A30EE600A8DED040A9DED8D
:40A70000040A05F01CF90A99087050E40898007A03280DD10898807A049008980079039004997FF0BAFE0898007904900FF094FE3DE40898007A032804D106F0AEF820209C
:40A7400004F08CFD33E40898007A032804D108980079049000F00FFF29E40898007A032803D108980079584908701FE20898007A032803D1089800795449087016E2089848
:40A78000007A032804D10898406804901DF09AFB0CE20898007A032804D10898007904901DF0C7FE02E20898007A032804D10898007904901DF0E9FEF8E10898007A03285D
:40A7C00004D10898007904901DF00BFFEEE10898007A032804D10898007904901DF02DFFE4E10898007A032804D10898007904901DF075FFDAE10898007A032804D108986F
:40A80000007904901DF097FFD0E10898007A032804D10898007904901DF0B9FFC6E10898007A032821D108984068052818D2DFE800F003070B0F1300002006F0D2F913E02C
:40A84000012006F0CEF90FE0022006F0CAF90BE0032006F0C6F907E0042006F0C2F903E0002006F0BEF900BF00BF9FE19EE10898007A032818D10D4890F8E004012807D194
:40A880000898807A0146049000200AF0FDFE06E00898807A0146049001200AF0F5FE00214FF4807018F00AFB80E10000982400203C0D001030320020316D0908C81C002079
:40A8C000B01F0010D02B00205D0300105E0300100898007A032809D10898808880B20121049048F078F80A9908701EE00898007A01280BD1FA48B0F85A07401C80B20121F3
:40A90000049048F068F80A9908700EE00898007A02280AD1F248B0F85A07401E80B20121049048F058F80A990870E9E30898007A032809D10898808880B20121049048F0E4
:40A9400087F80A9908701EE00898007A01280BD1E348B0F85C07401C80B20121049048F077F80A9908700EE00898007A02280AD1DB48B0F85C07401E80B20121049048F02B
:40A9800067F80A990870BBE30898007A032809D10898808880B20121049048F096F80A9908701EE00898007A01280BD1CC48B0F85E07401C80B20121049048F086F80A9914
:40A9C00008700EE00898007A02280AD1C448B0F85E07401E80B20121049048F076F80A9908708DE30898007A032809D10898808880B20121049048F0A5F80A9908701EE0A5
:40AA00000898007A01280BD1B548B0F86007401C80B20121049048F095F80A9908700EE00898007A02280AD1AD48B0F86007401E80B20121049048F085F80A9908705FE35E
:40AA40000898007A032808D10898808880B2049048F0B5F80A9908701CE00898007A01280AD19F48B0F86207401C80B2049048F0A6F80A9908700DE00898007A022809D11A
:40AA80009748B0F86207401E80B2049048F097F80A99087034E30898007A032808D10898808880B2049048F0C0F80A9908701CE00898007A01280AD18948B0F86407401C98
:40AAC00080B2049048F0B1F80A9908700DE00898007A022809D18248B0F86407401E80B2049048F0A2F80A99087009E30898007A032808D10898808880B2049010F0C2FC65
:40AB00000A9908701CE00898007A01280AD17448B0F86607401C80B2049010F0B3FC0A9908700DE00898007A022809D16C48B0F86607401E80B2049010F0A4FC0A99087070
:40AB4000DEE20898007A032806D108980079049048F0A1F80A990870D2E20898007A032807D108980079049048F0C9F80A9908701CE00898007A01280AD1594890F869071B
:40AB8000401CC0B2049048F0BAF80A9908700DE00898007A022809D1514890F86907401EC0B2049048F0ABF80A990870A8E20898007A032807D108980079049048F0D3F8E1
:40ABC0000A9908701CE00898007A01280AD1444890F86A07401CC0B2049048F0C4F80A9908700DE00898007A022809D13C4890F86A07401EC0B2049048F0B5F80A9908703E
:40AC00007EE20898007A032806D108980079049048F0E9F80A99087072E20898007A032809D10898808880B20121049048F012F90A9908701EE00898007A01280BD12848C9
:40AC4000B0F86C07401C80B20121049048F002F90A9908700EE00898007A02280AD12048B0F86C07401E80B20121049048F0F2F80A99087044E20898007A032801D111F0D6
:40AC8000FFFD3DE20898007A032810D10898807A0490089890ED010AB8EEC00A8DED030A04989DED030A82F0A2F90A99087027E20898007A032812D10898807A04900898AC
:40ACC000808880B200EE100AB8EE400A8DED030A04989DED030A81F0AEFC0A9908700FE2982400200898007A032812D10898807A04900898808880B200EE100AB8EE400A3D
:40AD00008DED030A04989DED030A82F0D1F80A990870F5E10898007A032805D1089800790121049004F08CFF04F06DFAE8E10898007A032808D10898807A0490089800793B
:40AD4000039004997EF0E2FDDAE10898007A032815D1089890ED010AF8EEC00A9FEDFE1A80EE810A8DED040AFC4890F8E00403909DED040A0FF058FD0A9908703EE008986B
:40AD8000007A01281BD1F54890F8E01400F5F26000EB8100D0ED000A9DED090AB8EEC00A30EE800A8DED030AEC4890F8E00404909DED030A0FF038FD0A9908701EE00898DD
:40ADC000007A02281AD1E54890F8E01400F5F26000EB8100D0ED000A9DED090AB8EEC00A30EEC00A8DED030ADC4890F8E00404909DED030A0FF018FD0A99087080E108983A
:40AE0000007A032818D1D54890F8E104012807D10898807A0146049000200BF06DFA06E00898807A0146049001200BF065FA00214FF4807018F042F862E10898007A03280E
:40AE400008D10898807A0490089800790390049909F0B6F954E10898007A032812D108984068012804D0022805D0032809D105E02EF020FA05E02EF03EFA02E02EF088FA5A
:40AE800000BF00BF3CE10898007A03280ED1089890ED010AB8EEC00ADFEDB10A20EE200A8DED040A9DED040A2EF044FA28E10898007A032836D10898406808282DD2DFE86D
:40AEC00000F004090E13181D22274FF4966004F0E6FD22E04FF4166004F0E1FD1DE04FF4965004F0DCFD18E04FF4165004F0D7FD13E04FF4964004F0D2FD0EE04FF4164067
:40AF000004F0CDFD09E04FF4614004F0C8FD04E04FF4E13004F0C3FD00BF00BF4FF4804004F09CF9ECE00898007A032808D10898807A0490089800790390049983F064FEA1
:40AF4000DEE0DDE00898007A03280AD1089890ED010AB8EEC00A8DED040A9DED040A06F0AEFDCDE00898007A032804D108980079049010F0DCFEC3E00898007A03280AD1CC
:40AF800008980079049005F0F7FC0A9908704FF4007004F063F9B3E011F0F9FA08BB11F01DFBF0B911F00DFBD8B911F0FDFAC0B90898007A032805D108980079049006F009
:40AFC000C7FE26E00898007A01280FD106F0A8FD042807DA06F0A4FD401CC0B2049006F0B7FE16E0012006F0B3FE12E00898007A02280ED106F094FD012807DD06F090FD2D
:40B00000401EC0B2049006F0A3FE02E0042006F09FFE75E00898007A032806D10898007940B204902EF0B6FA20E00898007A01280CD14A4890F89A0741B20122099802FB0F
:40B04000001040B204902EF0A5FA0FE00898007A02280BD1414890F89A0741B20122099802FB101040B204902EF094FA48E00898007A032809D10898807A049008984068F9
:40B08000039004990BF075FA26E00898007A01280FD13248B0F882170122099802FB001003900898807A0146049003980BF061FA12E00898007A02280ED12848B0F8821782
:40B0C0000122099802FB101003900898807A0146049003980BF04DFA0120069010E00898007A03280AD1089890ED010AB8EEC00A8DED040A9DED040A81F0B0F900E000BF52
:40B1000000BF089800780490FDF7DEF906980BB000BD86B04FF6FF7438211248DFF848C000DF0221114880F844110C22842110488BF05CFC00287BD103210C4880F8441164
:40B1400000BF224605A90748DFF828C000DF01285ED0002010E0000000007A44982400206F12833A50070010B96E090830320020CC060010497009088DF800008DF80D00EA
:40B1800001208DF80C0000208DF80E0005980078002838D004AA01210598FDF79BF905469DF8100068B100250599087841F03AF906460598C37A827A9DF81010304641F0C2
:40B1C000E1F911F0E4F908B1002504E00598007A032800D10025B5B19DF80D0098B90598007A80B1059A07CA8DE8070001208DF80D008DF80C004FF47A649DF80E00401CAC
:40B20000C0B28DF80E008D480599FDF78DF898E79DF80000002894DD9DF80E0000283DDD9DF80E00032804D102208DF80C000FE037E09DF80E00052803D106208DF80C00D4
:40B2400006E09DF80E00072802D110208DF80C009DF80E00FF2805DA9DF80E00401CC0B28DF80E009DF80C1004AA6846FDF732F99DF8100078B100208DF80E00059908780A
:40B2800041F0D0F806460598C37A827A9DF81010304641F077F94FF4FA6452E74FF6FF744FE70521664880F844110020DFF894C100DF00BFFEE770B50023002100BF06E061
:40B2C000614830F82100184383B2481CC1B20729F6DB002B55D05C48001F0078401C5A4A121F107010460078CF2801DD002010700CE05548001F0078401C534A121F1070AB
:40B3000010460078CF2801DD002010704E4C241F2278D41702EBD46465114B4C54F82540494D2D1F2878C51700EBD5656D11A0EB45160125B5402C40002CDAD0424C241F70
:40B340002078C41700EBD46465113F4C54F825403D4D2D1F2A78D51702EBD5656D11A2EB45160125B540AC43374D2D1F2878C51700EBD5656E11344D45F82640281F0078B7
:40B3800070BD0020FCE72DE9F04705460E4617469846DDF820904FF0010A2C48DFF8B0C000DFD0B900BF264890F8450140F00201234880F84511B0F850014FF6FF71884265
:40B3C00007DA1F48B0F85001401C81B21C48A0F8501100BF4FF0000A2CE01848FCF794FF04466CB125706660277284F80A8084F80B900A2221461548DFF858C000DF19E0F7
:40B4000000BF0F4890F8450140F004010C4880F84511B0F850014FF6FF71884207DA0848B0F85001401C81B20548A0F8501100BF4FF0000A5046BDE8F0870000CC060010BE
:40B4400030320020717809088C07001050070010B16E0908A56F090810B54FF099F9044655480022D0F8381520464BF000F810BD514890F82903022801D101207047002096
:40B48000FCE74FF6FF764FF071F94FF081F9074649480022D0F8381538464AF0E8FFDFF81CC100DF07466422394608204EF0EFFA38B1DFF808C100DF0746394608204EF00B
:40B4C00015FBDFF8F8C000DF074639460420DFF8F0C000DF00BF002231460D20DFF8E4C000DF0446012CF6D0022CF4D1DFF8D8C000DF054605F0080050B11CF099FC10B170
:40B500001CF0D8FF04E01CF00DFB08B11CF038FA05F004000028DED04EF086FC60B11CF077F820B11CF08CFC1BF094FFD3E71BF0D2FF1CF0F2FCCEE74EF09FFC0028CAD03B
:40B54000FFF796FF30B11CF0BBFA1CF079FCFFF783FFC0E71CF06CFC20B11CF0B1FA1CF0DCFCB8E71CF0DEFA0028B4D01CF068FC1CF0B0FAAFE701B50F4890F829039DF8DD
:40B580000010884216D000BF012269460F480CF0F3FD20B99DF80000074981F8290300BF7420FCF791FF0A48D0F8A8120420DFF810C000DF08BD0000982400202D7A0908E7
:40B5C000316D0908916D0908D96C0908290300683032002070B52DED028B84B004460E461546D0480078B04202D1B5F5FA7F08DDCC4806700020CC49087004B0BDEC028BAA
:40B6000070BDC948007838B9C848D4E9001206C00120C5490870F0E70A2D00DAEDE700EE105AB8EEC00ADFEDC20AC0EE808A94ED010ABE48D0ED010A30EE600A20EE280A21
:40B640008DED030A94ED000AD0ED000A30EE600A20EE280A8DED020A9DED030AB548D0ED010A30EE600A8DED010A9DED020AD0ED000A30EE600A8DED000AAF4890ED000A53
:40B68000B0EEC00ADFEDAD0A30EE200AAC4880ED000A90ED000ADFEDAB0AB4EEE00AF1EE10FA03DD9FEDA70A80ED000AA14890ED010ADDED010AA24890ED001A00EE810A9B
:40B6C0009C4880ED010A90ED000ADDED000A9C4890ED001A00EE810A964880ED000A1FF03FFBB0EE408AB0EE480A10F0BBFE10B1B0EE480A01E09FED940AB0EE408A9FED40
:40B70000930AB4EEC08AF1EE10FA02DD9FED8E0A01E0B0EE480A884880ED000A94ED010A824880ED010A94ED000A80ED000A00BF63E770B52DED048B84B005460E461446A8
:40B7400083480078B04202D1B4F5FA7F08DD8048067000207F49087004B0BDEC048B70BD7C48007838B97C48D5E9001206C0012078490870F0E70A2C00DAEDE700EE104A1F
:40B78000B8EEC00ADFED6A0AC0EE808A95ED010A7148D0ED010A30EE600A20EE280A8DED030A95ED000AD0ED000A30EE600A20EE280A8DED020A9DED030A6848D0ED010A14
:40B7C00030EE600A8DED010A9DED020AD0ED000A30EE600A8DED000A614890ED000AB0EEC00ADFED560A30EE208A9FED560AB4EEC08AF1EE10FA03DD9FED520AB0EE408A56
:40B80000564890ED010ADDED010A00EE880A80ED010A90ED000ADDED000A00EE880A80ED000A1FF09DFAB0EE409AB0EE490A10F019FE10B1B0EE490A01E09FED430AB0EE93
:40B84000409A9FED420AB4EEC09AF1EE10FA02DD9FED3D0A01E0B0EE490A414880ED000A00EE104AF8EEC00A9FED311A81EE200AD0ED000A3B4890ED001A70EEC10A20EE2D
:40B88000200A394880ED000A90ED000A3748D0ED000A70EE600A90ED000AB6EE001A00EE810A80ED000A95ED010A2B4880ED010A95ED000A80ED000A294890ED000A2948B8
:40B8C00080ED000A00BF47E71B4890ED000A7047234890ED000A7047234890ED000A7047224890ED000A704700200F49087070470E4991ED010AD0ED010A30EE200A81ED44
:40B90000010A91ED000AD0ED000A30EE200A81ED000A70470A4890ED000A7047144890ED000A704729000020280000201400002000007A441C00002024000020CDCC4C3EE6
:40B940000C000020CDCC4C3F00000000CDCC32424D0000204C0000202C000020340000203C0000204000002044000020480000201000002010B50220FE49087000200871FA
:40B980004DF0A6FFFB498860002088600120487041F288304880012008750021F54801764DF096FFF349C8610021F248C1610121417541F28831C182152141620220EE4985
:40B9C000087010BD10B5ED480078ED490870ED4800784870EC4800788870EC480078C870FFF7C8FF10BD0421018000214180012181800021C1800181704770B50446042C86
:40BA000001DD002070BD44BBE148B0F87E0728B9DF48B0F8800708B9012523E0D74800784EF096FC00EE100AB8EE400ADFEDD90A20EE200ABCEEC00A10EE106AD448B0F86F
:40BA40007E07B04206D8D248B0F88007B04201D3012000E00020054604E0C949085D4EF0F4FD054694B925B14DF032FFCA4908600CE04DF02DFFC8490968401A41F6583124
:40BA8000884201D2012000E0002005460DB10120B8E70020B6E770B504460025012C11DA84B9B64800784EF053FC00EE100AB8EE400ADFEDB80A20EE200ABCEEC00A10EE26
:40BAC000100A85B2284670BD2DE9F04106463007070E042F02DD0020BDE8F0810025002410E03819042805DAA549085D4EF0ADFD804601E04FF00308610008FA01F00543D6
:40BB0000601CC4B2102CECDB2846E5E72DE9F0470746884615461E464FF00009002448E004EB8400934911F82000B84240D104EB840001EB80000079404539D14FF0010968
:40BB4000012D00D05EB104EB84008A4901EB8000457004EB840001EB8000468028E086480078401EA04206D1002004EB8401814A02F8210017E0804A1278521E02EB8202A1
:40BB80007C4B03EB820104EB840203EB8200142285F069FB002178480078401E00EB8000744A02F8201074480078401E72490870641CB9F1000F03D16F4800788442AFDBFE
:40BBC000B9F1000F2ED16C480078202802D10120BDE8F087012D00D016B36748007800EB8000644901F820706348007800EB800001EB800080F804805F48007800EB8000FA
:40BC000001EB800045705C48007800EB800001EB8000468058480078401C5749087001E00220D5E70020D3E77CB5002600250024CEE0002604EB84004E4911F8200000B9A5
:40BC4000C9E004EB84004B4901EB80004088B0B104EB84020B4603EB8202518804EB840203EB8202D0684DF04DFE40B14DF030FE04EB84013F4A02EB8101C86001263EB9B9
:40BC800004EB84003B4901EB80004078012819D104EB8400374911F82000022809D104EB8401344A02EB81010879FFF70DFF054608E004EB84012F4A02EB81010879FFF74C
:40BCC0009CFE0546A6B904EB84002A4901EB8000407801280CD104EB840001EB80008068A84205D004EB840001EB800085600126F6B304EB84001F4911F82000022816D1C1
:40BD000004EB840001EB800001799DF8000061F387108DF800009DF8000020F03E008DF80000CDF8015068463BF008FF4EE004EB8401104A02EB81010879C11700EB117116
:40BD400009119DF8042061F347128DF8042004EB8401084A02EB81010879C11700EB11710911A0EB01119DF8042061F3440215E02CE00000081E002074000010380600206C
:40BD8000700000103706002036060020390600209824002000404E3F780000108DF804209DF8050065F301008DF8050004EB84000F4901EB8000007C9DF8051060F387015C
:40BDC0008DF8051001A83BF0C1FE00BF601CC4B2202CFFF62EAF00BF7CBDFFF7F3FD05E0FFF722FF2820DFF80CC000DFF8E70000081E0020D16C090888B00168079141684E
:40BE0000069181680591C1680491016903914169029181690191C169009108B07047000000487047A8BD022010B585F0E9FB001D10BD00BFC9BC080020F030BD0000000076
:40BE40000000000000000000000000000000000000000000000000000000000000000000000000000000000000000000526176656E20496E64757374726965732C20496E79
:40BE8000632E000000000000000000004175672D31382D323031380000000000312E332E302E32383000000000000000526176656E2047756964616E636520436F6E74722C
:40BEC0006F6C6C6572000000000000003037373031373134343900000000000000000000000000000000000000000000FFFFFFFFFFFFFFFFFFFFFFFFFFFFFFFFFFFFFFFF30
:40BF0000FFFFFFFFFFFFFFFFFFFFFFFFFFFFFFFFFFFFFFFFFFFFFFFFFFFFFFFFFFFFFFFFFFFFFFFFFFFFFFFFFFFFFFFFFFFFFFFFFFFFFFFFFFFFFFFFFFFFFFFFFFFFFFFF41
:40BF4000FFFFFFFFFFFFFFFFFFFFFFFFFFFFFFFFFFFFFFFFFFFFFFFFFFFFFFFFFFFFFFFFFFFFFFFFFFFFFFFFFFFFFFFFFFFFFFFFFFFFFFFFFFFFFFFFFFFFFFFFFFFFFFFF01
:40BF8000FFFFFFFFFFFFFFFFFFFFFFFFFFFFFFFFFFFFFFFFFFFFFFFFFFFFFFFFFFFFFFFFFFFFFFFFFFFFFFFFFFFFFFFFFFFFFFFFFFFFFFFFFFFFFFFFFFFFFFFFFFFFFFFFC1
:40BFC000FFFFFFFFFFFFFFFFFFFFFFFFFFFFFFFFFFFFFFFFFFFFFFFFFFFFFFFFFFFFFFFFFFFFFFFFFFFFFFFFFFFFFFFF00C00008FFFF170800800008FBBF0008AE3D01CC86
:40C00000012904D002290BD003291BD111E042F2107242436423B2FBF3F2FE4B1A8012E042F2107242436423B2FBF3F2FA4B1A8009E042F2107242436423B2FBF3F2F74B18
:40C040001A8000E000BF00BF704710B50446F44800882044F24908800846008842F21071884202DB0020EE490880ED480088E9490988884205DA0121EA4800784DF05BFF7A
:40C0800004E00021E74800784DF055FFE4480088E1490988884205DA0121E34800784DF04AFF04E00021E04800784DF044FFDC480088DA490988884205DA0121DB480078F5
:40C0C0004DF039FF04E00021D84800784DF033FF10BD70B505464DF0FBFB04460020D44988614FF47A71D248C1614462002180F8281003210020FFF783FF0020CC49C862E3
:40C100004FF47A71CA4801638463002180F83C1002210020FFF774FF0020C54948604FF47A71C348816004610021017501210020FFF766FF0020BE4908644FF47A71BC4895
:40C140004164C464002180F850100020B84948654FF47A71B64881650466002180F86410122D7DD2DFE805F009233D569CC1F1EFEEEDECEBEAE9E8E7E6E54FF4FA70AC499B
:40C1800088610146AA48C1614462012180F82810014691ED080ABCEEC00A10EE101A88B20321FFF72DFF0120A149087007E34FF4FA709F49C86201469D480163846301210B
:40C1C00080F83C10014691ED0D0ABCEEC00A10EE101A88B20221FFF713FF012094490870EDE24FF4FA7092494860014690488160046101210175014691ED030ABCEEC00AE6
:40C2000010EE101A88B20121FFF7FAFE012088490870D4E202208649087032204860322183488160046100210175014691ED030ABCEEC00A10EE101A88B20121FFF7E0FE70
:40C240004FF4FA607A4948650021794881650466012180F864100020FFF7D2FE032100E0ACE20020FFF7CCFE02210020FFF7C8FE02206F4981F8680002216D4880F8691096
:40C2800080F86A1080F86B1080F86C10042180F86D10062180F87710002180F878108EE24FF4FA7062490864014661484164C464012180F85010014691ED080ABCEEC00A0E
:40C2C00010EE101A88B20321FFF79AFE584991ED030ABCEEC00A10EE101A88B20121FFF78FFE01205249087069E264205049086464214F484164C464012180F85010014651
:40C3000091ED080ABCEEC00A10EE101A88B20321FFF776FE464991ED030ABCEEC00A10EE101A88B20121FFF76BFE01204049087045E213E2E1E1AFE169E123E1BDE0EEE04F
:40C3400086E04FE035E01AE0FFE74FF47A703849886100213648C1614462012180F82810014691ED080ABCEEC00A10EE101A88B20321FFF745FE01202D4908701FE24FF406
:40C380007A702B49C8620021294801638463012180F83C10014691ED0D0ABCEEC00A10EE101A88B20221FFF72BFE01202049087005E24FF47A701E49486000211C488160B3
:40C3C000046101210175014691ED030ABCEEC00A10EE101A88B20121FFF712FE012014490870ECE14FF47A7011490864002110484164C464012180F85010014691ED080AA3
:40C40000BCEEC00A10EE101A88B20321FFF7F8FD07490FE0020000200400002006000020080000201A060020350600201B060020A807001091ED030ABCEEC00A10EE101A82
:40C4400088B20121FFF7DCFD0120FE490870B6E10220FC4908704FF4FA7088610021F948C161446280F82810014691ED080ABCEEC00A10EE101A88B20321FFF7C1FD4FF403
:40C48000FA70F049C8620021EE4801638463012180F83C1002210020FFF7B2FD0120E94981F868000021E74880F86910022180F87710002180F8781081E10220E149087061
:40C4C0004FF4FA7088610021DE48C161446280F82810014691ED080ABCEEC00A10EE101A88B20321FFF78CFD4FF4FA70D54948600021D44881600461017501210020FFF7F3
:40C500007FFD0120CF4981F868000221CD4880F8691080F87710002180F878104FE10220C84908704FF4FA70C8620021C54801638463012180F83C10014691ED0D0ABCEE85
:40C54000C00A10EE101A88B20221FFF759FD4FF4FA70BC4948600021BA4881600461017501210020FFF74CFD0020B64981F868000221B44880F8691080F87710002180F8BE
:40C5800078101CE10220AF4908704FF4FA7088610021AC48C1614462012180F82810014691ED080ABCEEC00A10EE101A88B20321FFF726FD4FF4FA70A249C8620021A14869
:40C5C0000163846380F83C1002210020FFF718FD4FF4FA709B49486000219A4881600461017501210020FFF70BFD0120954981F868000021934880F86910022180F86A10C4
:40C60000032180F87710002180F87810D7E002208C49087040F24D10886100218948C1614462012180F82810014691ED080ABCEEC00A10EE101A88B20321FFF7E1FC40F2B6
:40C640004D108049C86200217E480163846380F83C1002210020FFF7D3FC40F24D10794948600021774881600461017501210020FFF7C6FC0120734981F868000021714845
:40C6800080F86910022180F86A10032180F87710002180F8781092E002206A4908704FF4FA70886100216748C161446280F82810014691ED080ABCEEC00A10EE101A88B2E6
:40C6C0000321FFF79DFC4FF4FA705E49086400215C484164C464012180F850100120594981F868000321574880F86910022180F87710002180F8781061E00220514908702B
:40C700004FF4FA70C86200214E480163846380F83C10014691ED0D0ABCEEC00A10EE101A88B20221FFF76CFC4FF4FA7045490864002144484164C464012180F850100020EE
:40C74000404981F8680003213E4880F86910022180F87710002180F8781030E00220394908704FF4FA70486000213648816004610175014691ED030ABCEEC00A10EE101A27
:40C7800088B20121FFF73CFC4FF4FA702D49086400212C484164C464012180F850100220284981F868000321264880F86910022180F87710002180F8781000E000BF00BF6C
:40C7C0002148057070BD20B1012806D002280CD107E01C4981ED0D0A08E01A4981ED080A04E0184981ED030A00E000BF00BF0121164A1170704770B5002515480078E0B92B
:40C800008021104884F08BFD9FED120A0020FFF7DAFF9FED110A0220FFF7D5FF9FED0D0A0120FFF7D0FF0020064981F879000220FFF74FFC0120064908704DF049F80446DC
:40C8400000480BE0A807001000000020010000200A0000200000A0420000C84290F87900002845D14DF0DDFAFF280ED1FD480078022803D1FC480078012805D10220FFF788
:40C8800028FC0020F84908709BE001202EF066FD70B9F4480078052803D1F34800780128F2D10520FFF715FC0020EF49087088E002F011F870B1EB480078042803D1EA4884
:40C8C000007801287DD10420FFF703FC0020E649087076E0E348007818B9E348007801286FD10020FFF7F5FB0020DF49087068E0DE4890F8790001280ED1DA4800780E2886
:40C9000003D1D948007801285BD10E20FFF7E1FB0020D549087054E0D44890F87900022815D1D249C86F4FF47A614CF0EBFF70B9CC480078082803D1CB480078012840D10A
:40C940000820FFF7C6FB0020C749087039E0C74890F87900042815D1C449C86F4FF47A614CF0D0FF70B9BF480078072803D1BE480078012825D10720FFF7ABFB0020BA495A
:40C9800008701EE0B94890F87900032815D1B749C86F4FF47A614CF0B5FF70B9B1480078062803D1B048007801280AD10620FFF790FB0020AC49087003E00020AB4981F8F5
:40C9C0007900AA480078012802D002287DD1F9E0A64890F83C00E0B9A448C06AC8B1A348816B20464CF0BEFFA049096B88422AD301219E4880F83C108463014691ED0D0A45
:40CA0000BCEEC00A10EE101A88B20221FFF7F8FA19E0964890F83C00012814D19348006B88B19248816B20464CF09CFF8F49C96A884208D300218D4880F83C108463022176
:40CA40000020FFF7DDFA8948007DD8B987484068C0B18648016920464CF084FF83498968884227D30121814801750461014691ED030ABCEEC00A10EE101A88B20121FFF79E
:40CA8000BFFA17E07948007D012813D17748806880B17648016920464CF064FF73494968884207D3002171480175046101210020FFF7A6FA6D4890F82800F0B96B4880692E
:40CAC000D8B16A48416A204600E008E24CF04AFF6649C96988422AD30121644880F828104462014691ED080ABCEEC00A10EE101A88B20321FFF784FA19E05C4890F828003D
:40CB0000012814D15948C06988B15848416A20464CF028FF55498969884208D30021534880F82810446203210020FFF769FA4F4890F8500038BB4D48006C20B34B48C16CF6
:40CB400020464CF00FFF4949496C884239D30121464880F85010C464014691ED080ABCEEC00A10EE101A88B20321FFF749FA3F4991ED030ABCEEC00A10EE101A88B2012123
:40CB8000FFF73EFA1DE0394890F85000012818D13648406CA8B13548C16C20464CF0E2FE3249096C88420CD30021304880F85010C46403210020FFF723FA01210020FFF76F
:40CBC0001FFA8CE1294890F878106830405C38BB264890F83C00012817D12448816B20464CF0C0FE2149C96A88420DD300211F4880F83C10846302210020FFF701FA1B48FB
:40CC0000006B002800D10125D2E01848816B20464CF0A8FE1549096B8842F5D30125C7E0124890F878106830405C02282BD10F48007D01281CD10D48016920464CF092FE54
:40CC40000A4949688842DFD3002108480175046101210020FFF7D4F904488068002800D10125A5E00000002001000020A80700109C48016920464CF075FE9A49896888420A
:40CC800000D3012594E0974890F878106830405C012826D1934890F82800012816D19148416A20464CF05EFE8E49896988427FD300218C4880F82810446203210020FFF73D
:40CCC0009FF98848C06990BB012571E08548416A20464CF047FE8349C969884268D3012566E0804890F878106830405C03282AD17C4890F8500001281AD17A48C16C2046DC
:40CD00004CF030FE7749096C884251D30021754880F85010C46403210020FFF771F901210020FFF76DF96F48406C00B901253FE06C48C16C20464CF015FE6A49496C88421D
:40CD400036D3012534E0674890F878106830405C04282DD1634890F8640001281ED16148016E20464CF0FEFD5E49496D88421FD300215C4880F86410046602210020FFF782
:40CD80003FF903210020FFF73BF901210020FFF737F95448806D58B9012509E05148016E20464CF0DFFD4F49896D884200D30125012D28D100254B4890F87800401CC1B237
:40CDC000484880F8781090F8781090F87700814203DB0021434880F87810424890F878106830405C80B901213E4880F83C108463014691ED0D0ABCEEC00A10EE101A88B23B
:40CE00000221FFF7FDF869E0364890F878106830405C02280FD10121324801750461014691ED030ABCEEC00A10EE101A88B20121FFF7E6F852E02B4890F878106830405CD1
:40CE4000012810D10121274880F828104462014691ED080ABCEEC00A10EE101A88B20321FFF7CEF83AE01F4890F878106830405C03281BD101211B4880F85010C46401468C
:40CE800091ED080ABCEEC00A10EE101A88B20321FFF7B6F8134991ED030ABCEEC00A10EE101A88B20121FFF7ABF817E00D4890F878106830405C042810D10121094880F844
:40CEC0006410046602210020FFF79AF803210020FFF796F801210020FFF792F800BF00BF70BD0000A807001013B5044600BFF9490819012201A90BF03FF920B9BDF80400CF
:40CF0000C1B2F548015500BF1CBD13B5044600BFF24901EB4400022201A90BF02DF920B9BDF80410EE4820F8141000BF1CBD13B5044600BFEB496018012201A90BF01CF922
:40CF400018B99DF80410E848015500BF1CBD10B5044600212046FFF7EAFF00212046FFF7D4FF00212046FFF7BFFF10BD2DE9F047DE480078002832D103F07EFB00282ED0A4
:40CF8000DB4890F82180A8F108044FF00009012C00DA0C34002514E0D14810F8150000F00F06A64200DA0C360027301B082800DD012727B12846FFF7CAFF4FF00109681C20
:40CFC000C5B2FF2DE8DBB9F1000F04D001205FF096FB5FF015FD0120C449087000BFBDE8F08770B5A2201CE0C41700EBD4646511C04C54F82540C51700EBD5656D11A0EB3D
:40D0000045160125B5402C40C51700EBD5656D11A0EB45160125B540AC4200D103E0411EC8B20028E0DC00BF70BD10B50024B248006888B14FF47A71AF4800684CF062FC98
:40D0400050B110F09DF838B9AC480078122803D1AB48007800B90124204610BD30B5C31700EBD3635C11A34B303353F824300246C41700EBD4646411A0EB44150124AC4046
:40D0800023430146C41700EBD4646511994C303444F8253030BD9B4A50547047994AFF3A5054704730B50346DA1703EBD2625411904A52F824201946DC1703EBD4646411D6
:40D0C000A3EB44150124AC40A2431846DC1703EBD4646511874C44F82520DA1703EBD2625411844A183252F824201946DC1703EBD4646411A3EB44150124AC40A243DC1737
:40D1000003EBD46465117B4C183444F82520DA1703EBD2625411774A303252F82420DC1703EBD4646411A3EB44150124AC40A243DC1703EBD46465116E4C303444F82520FD
:40D140000020FFF7ABFF30BD30B50146CB1701EBD3635C11674B53F82430CC1701EBD4646411A1EB44150124AC4023400BB1012030BD0020FCE72DE9F0412DED028B04463A
:40D18000614890ED221BB0EE410AF0EE610A51EC100B8AF0EBFC08EE100A9FED5C0AC8EE000ABCEEE00A10EE100AC5B29FED580AC8EE000ABCEEE00A10EE100A80B23C2153
:40D1C00090FBF1F201FB1200C6B26902484890F8200041EA0010464991F82110084387B24148005D401C00F0FF0841462046FFF79EFE39462046FFF788FE31462046FFF7A4
:40D2000073FEBDEC028BBDE8F081014641B1202905D0252902D0262904D100BF00BF00BF002001E0012000BF00BF704701466C2914D006DC592909D0692909D06B2911D124
:40D2400008E0842908D085290CD109E000210BE0112109E0122107E0152105E01C2103E01F2101E0084600BF00BF704770B58CB004460D4621480078122828D1254B26A263
:40D28000232102A8009483F0E3FB02A883F030FF461C314602A873F0CBF92046FFF7C6FF2049087008460078FFF7AFFF40B13DB11C480078FFF75FFF1A4800785FF01EFBE8
:40D2C0008A20FBF701F9C520FBF7FEF800BF0CB070BD0000FE1E006830310020001D0068322F0020001C0068322E002009000010D81B0020000C0010040000104D03001058
:40D30000B01F0010FF040068C81C0020000061450000704268B10908257320636F64653A2025640001000010F948007870472DE9F0412DED028B044600252D2C7ED032DC54
:40D34000172C7CD016DC0B2C5DD006DC052C77D2DFE804F051F2525758000E2C71D004DC0C2C5AD00D2C6BD170E00F2C6AD0162CF9D195E0272C66D00CDC1A2C75D004DC19
:40D38000182C73D0192CEED17BE1232C6FD0242CE9D1CAE0292C6BD02A2C6AD02B2C69D02C2CE0D1E8E03D2C77D00DDCA4F12E000F28CCD2DFE800F0F4F9ECEBEAE94444BC
:40D3C00044E8E74444E6E500482C67D00ADCA4F13E000A28BBD2DFE800F0F1F0EF3333333333EEED4C2C70D04D2C6FD0502C6ED0582CB8D15CE164E14DF095FA80F0010548
:40D400005FE15EE15DE101F0F7FB28B94CF060FAC049884200D9012553E101F0EDFBA0B1BD4890ED1E0ADFEDBD0AB4EEE00AF1EE10FA02DC90F8800038B905E0ABE037E095
:40D440003EE118E02BE076E001253AE101F0D4FB50B1B14890ED1E0ADFEDB10AB4EEE00AF1EE10FA00D201252BE134E028E04EE073E077E07BE001F0BFFB68B1A94890ED13
:40D480000C0ADFEDA90AB4EEE00AF1EE10FA02DC90F8380000B9012513E1D0E0EDE010E103F004F908B9012000E00020054608E102F0EAF9012800D100E00020054600E182
:40D4C00019F062FE20B9012003E0E2E0E6E0EBE000200546F5E00FF0F1FEFA2803D00FF0EDFEFB2812D19148D0ED020A9048B0F8D00000EE100AB8EE400AF4EEC00AF1EE0B
:40D5000010FA01D8012000E000200546D9E0894890F82D01802803D1864890F8F10408B9012000E000200546CBE003F0A5F880F00105C6E000E0C4E012F00EFD50B10FF080
:40D54000BDFEFA2806D07B4890F87B07012801D0012000E000200546B3E003F06AFB00F00105AEE003F065FBC0F34005A9E003F060FBC0F38005A4E003F05BFBC0F3C005B7
:40D580009FE057E051E043E03DE02FE021E01BE015E00AE004E003F04CFBC0F3001590E003F047FBC0F340158BE003F042FBC0F3801586E05CE056E050E04AE044E003F09B
:40D5C00038FBC0F3C0157CE003F033FBC0F3002577E003F02EFB00F4007020B125F055F808B1012000E0002005466AE003F021FB00F4806020B125F048F808B1012000E0DF
:40D60000002005465DE003F014FBC0F3803558E003F00FFB00F4004020B125F028F808B1012000E0002005464BE003F002FBC0F3804546E003F0FDFAC0F3C04541E003F0D5
:40D64000F8FAC0F300553CE003F0F3FAC0F3405537E003F0EEFAC0F3805532E003F0E9FAC0F3C0552DE003F0E4FAC0F3407528E003F0DFFAC0F3807523E003F0DAFAC50FE2
:40D680001FE00FF07DFD08B1012000E00020054617E00AF055FD80F0010512E00125002500BF00BF00BF0CE003F0ACFB054608E019F098FD08B9012000E00020054600BF57
:40D6C00000BF00BF0FF0FAFDFB286ED0194890F87B070128F9D01B2C68D00EDCA4F10500112878D2DFE800F0637B37838BCC7777777777DAF1F0EFEEED004B2C6CD020DC45
:40D70000222C6AD018DC1F2C68D0212C63D135E001000010C0D40100481800200000484300004842D81B002000401C46D02B0020C81C002098240020492C7AD04A2CE5D17E
:40D740006BE1A4F14F000828CBD2DFE800F07644C6CEBF4444F004F0F2FF60B904F0F7FF48B9F84890F89907032802D136F056FA08B9012000E00020054697E1F14890F845
:40D780007D0703280ED0EF4890F87D07022809D0EC4890F87D07012802D112F0ADFC08B9012000E00020054680E105E2F7E005F0D5FE20B106F067F808B1012000E000209B
:40D7C00005463DB1FFF7B0FD052803D000210520FFF74CFD6AE168E134E1FDE0F3E005F007F908B9012000E0002005465EE106F025FB08B1012000E00020054656E1D24882
:40D800001FF0C6F898B9D1481FF0C2F878B9D0481FF0BEF858B9CF481FF0BAF838B9CE481FF0B6F818B9CD481FF0B2F810B1012001E0D9E00020054638E1C3481FF0A8F8D4
:40D84000012818D0C1481FF0A3F8012813D0C0481FF09EF801280ED0BE481FF099F8012809D0BD481FF094F8012804D0BB481FF08FF8012801D1012000E00020054615E1E9
:40D8800006F001F880F001053DB1FFF74DFD0A2803D000210A20FFF7E9FC07E10FF00EFDFA280DD10FF00AFDFB2809D004F014FB20B904F054FF08B1012000E0002005466E
:40D8C000F4E050E043E036E02BE016E004F058FF10B12BF098FE0546E8E004F025F918B12BF09BFE80F00105E0E004F05AFF18B12BF093FE80F00105D8E004F0D4FF78B96D
:40D9000004F0BAFF60B904F0C7FF48B904F0BCFF30B97BF080FF08B9012000E000200546C4E07BF0B7FF012802D0012001E0A9E000200546BAE00FF0C1FCFA2806D10FF0B3
:40D94000BDFCFB2802D00EF0CAFD0546AEE00FF0B5FCFA2806D10FF0B1FCFB2802D00EF0DDFD0546A2E00FF0A9FCFA2816D10FF0A5FCFB2812D00EF09CFD68B90EF007FE5F
:40D9800050B90EF02BFE38B90EF01BFE20B90EF00BFE08B9012000E00020054686E00FF08DFCFA280ED10FF089FCFB280AD06C4890F8D80020B10DF0A3F808B9012000E073
:40D9C0000020054672E07AF038FD012801D0012000E00020054669E012F0BEFA08B9012000E00020054661E004F05DFF80B904F043FF68B904F050FF50B904F045FF38B99F
:40DA000080F082FD08B1012000E00020054603E00B207BF040FA054648E00EF0B8FD40B90EF0DCFD28B90EF0CCFD10B90EF0BCFD38B102F0E8FDB0EE408A0EF013FD80F05B
:40DA4000010533E00FF03AFCFA281AD10FF036FCFB2816D00CF0AAFF78B904F024FF40B904F00AFF28B904F017FF10B904F00CFF28B148207BF00FFA08B1012000E00020EC
:40DA8000054613E00FF01AFCFA280DD10FF016FCFB2809D004F085FE20B135F077F808B9012000E00020054600E000BF00BF04F0FAFE48B904F0E0FE30B904F0EDFE18B947
:40DAC00004F0E2FE002877D0A4F14E00552874D2DFE800F02B73737373734D7373617373777C81868B90959A9FA473A9AEB3F2F7FCEEEDECEBEAE9E8E7E6E5E4E3E2E1E030
:40DB0000DFDEDDDCDBDAD9D8D7D6D5D4D3D2D1D0CFCECDCCCBCAC9C8C7C6C5C4C3C2C1C0BFBEBDBCBBBAB973B8007BF0A2F90D4BC01A71F1000117D205F01DF9A0B10120A5
:40DB400013E000009824002050BF001060BF001070BF001080BF001090BF0010A0BF0010C81C00200E5B637700200546C7E10BF0F8FC06460F467BF028FA301A8F4107D2C2
:40DB800005F0EFF820B14CF078F908B1012000E000200546B3E10BF0E4FC06460F467BF014FA301A8F4109D205F0DBF830B14CF03BF918B1012002E0A2E19FE10020054615
:40DBC0009DE101207BF067F9054698E102207BF062F9054693E103207BF05DF905468EE104207BF058F9054689E105207BF053F9054684E106207BF04EF905467FE10720E7
:40DC00007BF049F905467AE108207BF044F9054675E109207BF03FF9054670E10A207BF03AF905466BE10C207BF035F9054666E10D207BF030F9054661E10E207BF02BF9F7
:40DC400005465CE155E14FE149E143E13DE137E131E12BE125E11FE119E113E10DE107E101E1FBE0F5E0EFE0E9E0E3E0DDE0D7E0D1E0CBE0C5E0BFE0B9E0B3E0ADE0A7E009
:40DC8000A1E09BE095E08FE089E083E07DE077E071E06BE065E05FE059E053E04DE047E041E03BE035E02FE029E023E01DE017E011E00BE005E0FFE70F207BF0ECF8054654
:40DCC0001DE110207BF0E7F8054618E111207BF0E2F8054613E112207BF0DDF805460EE113207BF0D8F8054609E114207BF0D3F8054604E115207BF0CEF80546FFE0162004
:40DD00007BF0C9F80546FAE017207BF0C4F80546F5E018207BF0BFF80546F0E019207BF0BAF80546EBE01A207BF0B5F80546E6E01B207BF0B0F80546E1E01C207BF0ABF82C
:40DD40000546DCE01D207BF0A6F80546D7E01E207BF0A1F80546D2E01F207BF09CF80546CDE020207BF097F80546C8E021207BF092F80546C3E022207BF08DF80546BEE073
:40DD800023207BF088F80546B9E024207BF083F80546B4E025207BF07EF80546AFE026207BF079F80546AAE027207BF074F80546A5E028207BF06FF80546A0E029207BF0CA
:40DDC0006AF805469BE02A207BF065F8054696E02B207BF060F8054691E02C207BF05BF805468CE02D207BF056F8054687E02E207BF051F8054682E02F207BF04CF80546ED
:40DE00007DE030207BF047F8054678E031207BF042F8054673E032207BF03DF805466EE033207BF038F8054669E034207BF033F8054664E035207BF02EF805465FE0362008
:40DE40007BF029F805465AE037207BF024F8054655E038207BF01FF8054650E039207BF01AF805464BE03A207BF015F8054646E03B207BF010F8054641E03C207BF00BF84B
:40DE800005463CE03D207BF006F8054637E03E207BF001F8054632E03F207AF0FCFF05462DE040207AF0F7FF054628E041207AF0F2FF054623E042207AF0EDFF05461EE07A
:40DEC00043207AF0E8FF054619E044207AF0E3FF054614E045207AF0DEFF05460FE046207AF0D9FF05460AE047207AF0D4FF054605E049207AF0CFFF054600E000BF00BF5A
:40DF000055B9F748007838B9F6480078002808DDF4480078844204D10120BDEC028BBDE8F0810020F9E74FF00008C1464FF0500A0321ED4880F8CC10C421EC4883F0EFF9A4
:40DF400000243DE10020EA490855EA48005DC4EB0411E94A02EB810189680870C4EB0410114601EB800080680078002804DCE148FF38005D00287DD0E21704EBD2625311B1
:40DF8000DA4A121D52F823202146E31704EBD3635B11A4EB431C012303FA0CF31A432046E31704EBD3634FEA631CD04B1B1D43F82C20E21704EBD2625311CC4A1C3252F8DF
:40DFC0002320E31704EBD3635B11A4EB431C012303FA0CF31A43E31704EBD3634FEA631CC24B1C3343F82C20C4EB0410C24901EB8000007BE0B1E21704EBD2625311BB4A63
:40E00000343252F823202146E31704EBD3635B11A4EB431C012303FA0CF31A432046E31704EBD3634FEA631CB04B343343F82C204BF04EFCB14941F8240000BFE21704EBE7
:40E04000D2625311A94A4C3252F823202146E31704EBD3635B11A4EB431C012303FA0CF39A432046E31704EBD3634FEA631C9F4B4C3300E002E043F82C2000BFC4EB0410BC
:40E080009D4901EB800090F8300001281CD1E21704EBD2625311954A643252F823202146E31704EBD3635B11A4EB431C012303FA0CF31A432046E31704EBD3634FEA631C24
:40E0C0008A4B643343F82C20C4EB04108A4901EB800090F83000022807D0C4EB041001EB800090F8300003281CD1E21704EBD26253117E4A7C3252F823202146E31704EBA0
:40E10000D3635B11A4EB431C012303FA0CF31A432046E31704EBD3634FEA631C734B7C3343F82C20C4EB0410734901EB800090F8300004281CD1E21704EBD26253116B4AB0
:40E14000943252F823202146E31704EBD3635B11A4EB431C012303FA0CF31A432046E31704EBD3634FEA631C604B943343F82C20C4EB0410604901EB800090F838000128F8
:40E180001CD0E21704EBD2625311584AAC3252F823202146E31704EBD3635B11A4EB431C012303FA0CF31A432046E31704EBD3634FEA631C4D4BAC3343F82C20601CC4B25C
:40E1C000A32CFFF6BFAE5EF01BFC4FF47A60DFF830C100DF4448D0F8F0100120DFF824C100DF4FF47A60DFF818C100DF00BF002251460320DFF810C100DF0646022E50D14A
:40E20000DFF808C100DF074607F0020078B3002442E0E31704EBD3634FEA631C334B1B1D53F82C304FEAE47C04EBDC6C4FEA6C1CA4EB4C1B4FF0010C0CFA0BFC03EA0C0398
:40E240004FEAE47C04EBDC6C4FEA6C1CA4EB4C1B4FF0010C0CFA0BFC634509D10120C4EB0411254A02EB81018968087008E018E00020C4EB0411204A02EB8101896808700A
:40E28000C4EB04111C4A02EB8101896808782146FEF701FF601CC4B2A32CBADB4420FAF713F9002424E22046FFF741F805462046FEF74AFFA8423ED08DB94FF000090C48B9
:40E2C000005D012801D1814627E0C4EB04100A4901EB8000407BD8B94FF001091DE02BE0020000100300001030320020FC0B0010570B0010FF040068348B0908280800102E
:40E30000D16C0908316D0908916D0908D96C0908FE48007808B14FF00109B9F1010F0AD10020FB4908554FF001082046FEF7BAFE4420FAF7C9F8DDE0E31704EBD3634FEADF
:40E34000631CF44B53F82C304FEAE47C04EBDC6C4FEA6C1CA4EB4C1B4FF0010C0CFA0BFC03EA0C034FEAE47C04EBDC6C4FEA6C1CA4EB4C1B4FF0010C0CFA0BFC6345DAD02A
:40E380000020E349085500BF0EF001F940B90EF025F928B90EF015F910B90EF005F9E8B1E21704EBD2625311DA4A483252F823202146E31704EBD3635B11A4EB431C0123EE
:40E3C00003FA0CF31A432046E31704EBD3634FEA631CD04B483343F82C201CE0E21704EBD2625311CB4A483252F823202146E31704EBD3635B11A4EB431C012303FA0CF3D2
:40E400009A432046E31704EBD3634FEA631CC14B483343F82C20E21704EBD2625311BD4A52F823202146E31704EBD3635B11A4EB431C012303FA0CF31A432046E31704EBF4
:40E44000D3634FEA631CB34B43F82C204BF040FAB14941F8240000BF00BF0EF098F840B90EF0BCF828B90EF0ACF810B90EF09CF808B1012000E0002001281DD1E21704EBEF
:40E48000D2625311A34A483252F823202146E31704EBD3635B11A4EB431C012303FA0CF31A432046E31704EBD3634FEA631C994B483343F82C201CE0E21704EBD2625311D4
:40E4C000944A483252F823202146E31704EBD3635B11A4EB431C012303FA0CF39A432046E31704EBD3634FEA631C8A4B483343F82C2000BF002D7DD0E21704EBD26253118D
:40E50000844A183252F82320E31704EBD3635B11A4EB431C012303FA0CF31A40002A4CD1C4EB04107D4901EB8000406AE8BBE21704EBD2625311774A183252F8232021463B
:40E54000E31704EBD3635B11A4EB431C012303FA0CF31A432046E31704EBD3634FEA631C6C4B183343F82C204FF00108C4EB04106A4901EB8000806800787E280DDAC4EB19
:40E58000041001EB800080680078401CC4EB0411624A02EB81018968087021460120FEF77DFDC4EB04115D4A00E007E002EB8101896808782146FEF76EFD53E0C4EB04120F
:40E5C000564B03EB8202516A534A52F824004BF099F9E0B3E21704EBD26253114D4A183252F823202146E31704EBD3635B11A4EB431C00E074E0012303FA0CF31A432046FD
:40E60000E31704EBD3634FEA631C424B183343F82C204FF00108C4EB0410404901EB8000806800787E280DDAC4EB041001EB800080680078401CC4EB0411384A02EB810117
:40E640008968087021460120FEF728FD00E009E0C4EB0411314A02EB8101896808782146FEF719FDC4EB04122C4B03EB8202127BB2B3E21704EBD2625311264A303252F8F9
:40E680002320E31704EBD3635B11A4EB431C012303FA0CF31A401ABB0DF079FF40B90DF09DFF28B90DF08DFF10B90DF07DFFC0B1C4EB0410194901EB8000806A58B1C4EBF8
:40E6C00004120B4603EB8202916A134A52F824004BF018F920B12046FEF7C0FC4FF0010804E02046FEF7BAFC4FF00108601CC4B2A32CFFF6D8ADB8F1010F1AD10848D0F8CB
:40E70000F0100120DFF81CC000DF0DE0B01F0010570B0010000C001028080010348B090830320020316D09084FF000084420F9F7CBFE9548007848B9FEF777FC30B1442024
:40E74000F9F7C2FE01209049087009E00EF018FD30B98E48006818B94BF0BAF88B490860FEF73FFC0446FEF701FC40E5002107E0874850F8210008B101207047481CC1B221
:40E780000629F5DB0020F8E70020002107E0804A303252F8212002B101204A1CD1B20629F5DB704770B5A2201DE0C41700EBD4646511774C303454F82540C51700EBD565D8
:40E7C0006D11A0EB45160125B5402C40C51700EBD5656D11A0EB45160125B540AC4200D103E0411EC8B20028DFDC00BF70BD70B500240DF0CCFE40B90DF0F0FE28B90DF092
:40E80000E0FE10B90DF0D0FE68B3A22428E0E31704EBD3635D115E4B183353F82530E51704EBD5656D11A4EB45160125B5402B40E51704EBD5656D11A4EB45160125B540A1
:40E84000AB420BD1C4EB0413524D05EB83035B7B012B03D1504B1B5D03B903E0601EC4B2002CD4DC00BF204670BD01214A4A1154704701460020FF2906DA474A525C0AB10F
:40E88000012200E000221046704700210CE0404850F821003E4A603252F82120104008B101207047481CC1B20629F0DB0020F8E700210CE0364850F82100354A783252F86B
:40E8C0002120104008B101207047481CC1B20629F0DB0020F8E7002200210CE02C4850F821002B4BA83353F82130184008B101207047481CC1B20629F0DB1046F8E700B589
:40E90000002304E01846FFF7B0FF581CC3B2A32BF8DB00BD1FB5044620A30FCB8DE80F0084B13CF041FC40F014FB00210A2070F0A9F80D226946FF203CF063FB01201B4912
:40E94000087002E00020194908701FBD1748007870470146C1EB01100E4A52F8200070470146C1EB01100B4A02EB8000007970470F490870704710B504460E480470C8201E
:40E98000F9F7A2FD10BD00000800001004000010000C0010348B0908570B00100102050A0B111214181921242B00000000000010030000100200001070B504460025F84873
:40E9C00090F82805012806D002280AD0032803D0052810D10AE000BF204625F0C9FD05460BE0204628F0DDFF054606E0204620F0B3FF054601E0002070BD00BF2846FBE7F8
:40EA000010B5E848007800F0010080B10120FFF7D3FF00280AD0E348006840F00800E14908600846006820F001000860E3E0DD48007800F0020080B10220FFF7BDFF002851
:40EA4000F4D0D848006840F00800D64908600846006820F002000860CDE0D248007800F0400080B14020FFF7A7FF0028DED0CD48006840F00800CB4908600846006820F0F2
:40EA800040000860B7E0C748007800F0800080B18020FFF791FF0028C8D0C248006840F00800C04908600846006820F080000860A1E0BC48007800F0040080B10420FFF704
:40EAC0007BFF0028B2D0B748006840F00800B54908600846006820F0040008608BE0B148007800F0080058B10820FFF765FF002805D0AC48006820F00800AA4908607AE036
:40EB0000A848007800F0100058B11020FFF754FF002870D0A348006820F01000A149086069E0A048007800F0200080B12020FFF743FF00285FD09B48006820F020009949A8
:40EB400008600846006840F40040086053E09548008800F4807058B14FF48070FFF72CFF38B39048006820F480708E49086042E08C48008800F4004058B14FF40040FFF720
:40EB80001BFFB0B18748006820F400408549086031E08448008800F4007058B14FF40070FFF70AFF28B17F48006820F400707D49086020E07B48008800F4804058B14FF490
:40EBC0008040FFF7F9FEB0B17648006820F48040744908600FE07348006800F4803050B14FF48030FFF7E8FE28B16E48006820F480306C49086010BD6B48007B052801D190
:40EC0000012070470020FCE710B56849C86E4AF09AFEB0F5FA7F24D3644890F8800000B30020624981F88000614981F8DA009FED610A084680ED160A00215C4880F84A10D5
:40EC40009FED5C0A80ED130A0020594981F8D5009FED590A554880ED140A002081F8D2000CE05249C86E4AF06EFE5449884205D34E4890F8800008B9FFF7BEFF5049C86A07
:40EC80004AF061FE43F69821884208D34C4890F8380020B100204A4981F838000EE04849C86A4AF050FE4549884207D3444890F8380018B9FFF7A0FF00B100BF4149486CD0
:40ECC0004AF041FE42F21071884208D33D4890F8500020B100203B4981F850000EE03949486C4AF030FE3549884207D3354890F8500018B9FFF780FF00B100BF3249D1F8A9
:40ED000044014AF020FE43F69821884208D32E4890F8500120B100202B4981F850010FE02949D1F844014AF00EFE2449884207D3254890F8500118B9FFF75EFF00B100BF81
:40ED40002249886C4AF0FFFDB0F57A6F08D31F4890F8540020B100201C4981F854000EE01A49886C4AF0EFFD1449884207D3174890F8540018B9FFF73FFF00B100BF1449B6
:40ED8000C86A4AF0E0FD44F62061884222D3104890F83800F0B100200D4981F8380028E0982400201C000010B81D002048180020C81C00200000000000007F43E0930400EE
:40EDC000D81B00209C190020481A0020F01900209C1B0020F749C86A4AF0B5FDF649884207D3F44890F8380018B9FFF705FF00B100BFF24890F8DA0030B918F009FC18B1D6
:40EE00001FED140A18F07EFBED4890ED140A5FED160AB4EE600AF1EE10FA04D1E9A20321543081F015FE10BD10B54AF051FD0446E348C466C06E6438E14988660846C06E53
:40EE4000896E401A00EE100AB8EE400ADC4880ED1E0A0120DA4981F88000DB48C462C06A6438D94988620846C06A896A401A00EE100AB8EE400AD44880ED0C0A0120D249A0
:40EE800081F83800002081F83900D0484464406C6438CE4908640846406C096C401A00EE100AB8EE400AC94880ED120A0120C74981F85000C648C0F84441D0F844016438FB
:40EEC000C349C1F840010846D0F84401D1F84011401A00EE100AB8EE400ABD4880ED520A0120BB4981F85001BA488464806C6438B84948640846806C496C401A00EE100A18
:40EF0000B8EE400AB34880ED130A0120B14981F85400A848C462C06A6438A64988620846C06A896A401A00EE100AB8EE400AA14880ED0C0A01209F4981F8380010BD0021EE
:40EF40009F4880F84A101FED650A80ED130A9FEDA20B80ED0C0B9FEDA00B80ED0E0B80F849101FED6B0A80ED140A704701209C490873704710B54AF0ABFC9149C8664AF0A5
:40EF8000A7FC9149C8628E4890ED140A5FED760AB4EE600AF1EE10FA07D01FED790A80ED140A4FF4A1704BF0F3FC8E4890F8280507287DD2DFE800F09C045B0581309D00FB
:40EFC00000BF8748407B20B9FFF7B9FF002086498880102182481030DFF810C200DF012810D0804B93F830257D4B597B7D4BD3F82C0525F048F87A49487301F11000DFF8C7
:40F00000F0C100DF78488088052804DDFFF7AEFF00207549888070E07148407B20B9FFF78EFF00207049888010216D481030DFF8BCC100DF012810D06A4B93F83025684B36
:40F04000597B684BD3F82C0520F06AFB6449487301F11000DFF898C100DF63488088052804DDFFF783FF00205F49888045E05C48407B30B9FFF763FF27F014FC00205A4967
:40F080008880102156481030DFF860C100DF012812D0544B93F83025514B597B514BD3F82C0528F017FA4E49487301F1100000E01EE0DFF83CC100DF1FE04948407B18B9A6
:40F0C000FFF73DFF21F0F7FE102145481030DFF81CC100DF01280AD04FF4E13021F0F8FE3F49487301F11000DFF804C100DF04E000BF08203A49487300BF00BF10BD10B510
:40F100003748007B06287CD2DFE800F003172438467A4AF089FE60B1364800784BF095FA38B103202E4908734AF0D2FB3249086002E001202A49087363E000212F480078AE
:40F140004AF0F9FE0220264908734AF0C1FB2A49086056E0284800684AF0F5FBB0F57A7F0BD30121254800784AF0E5FE03201C4908734AF0ADFB2049086042E01E48006803
:40F180004AF0E1FB40F6C411884204D30420144908730020487334E0FFF7ECFE1048407B082806D1FFF740FE05200D4908730120487026E09C1B0020E0930400C81C00204D
:40F1C000481800202D2D2D00D81B00209C190020481A0020F01900200000000000000000B81D002098240020A81D0020F971090815710908FE05002028000010200600200C
:40F2000000BF00BF10BD1021FE48DFF8FCC300DF01280AD00020FB491039487304200873F848DFF8E8C300DF17E00421F848DFF8D8C300DF012810D0F548007C40F020002D
:40F24000F3490874F348C16B4FF48060DFF8C8C300DFEF48DFF8B4C300DF7047EF4909680143EE4A1160704710B5ED4991F8281506290ED2DFE801F00D0307040B0900BF2D
:40F2800027F09EFA07E0002005E0002003E0002001E0002000BF00BF10BD10B500244AF0C3FD98B1DE4890F82805012804D0032803D0052807D104E000BF23F04DFA0446F6
:40F2C00003E0002401E0002400BF00BF204610BD10B5D34991F8281506290ED2DFE801F00D0307040B0900BF23F0F5F907E0012005E0002003E0012001E0002000BF00BF64
:40F3000010BD10B5C64991F8281506290ED2DFE801F00D030704090B00BF23F0C3F907E0012005E0012003E0012001E0002000BF00BF10BD70B505460E4636B1012E0DD0CD
:40F34000022E24D0032E3CD113E00DB9002404E0022D01D1032400E0022434E00DB9002406E0022D01D0092D01D1032400E0022429E0FFF7C6FF08B9012407E00DB90024A8
:40F3800004E0052D01D1032400E002241BE0FFF79FFF08B9012413E00DB9002410E0042D09D1FFF77AFF20B1FFF75EFF08B1052406E0032404E0052D01D1042400E0022453
:40F3C00001E0002400BF00BF052C05D0062C03D04AF07EFA93490860924800684AF0B3FA9149C1F89800084680F8D24070BD00208B4991F82815012904D0894991F82815E0
:40F40000032900D10120704710B5874890ED0E1BB0EE410AF0EE610A9FED841B53EC112B51EC100B89F02CF82FD37F4890ED0E1BB0EE410AF0EE610A9FED7E1B53EC112BAF
:40F4400051EC100B88F0E2FE1FD3774890ED0C1BB0EE410AF0EE610A9FED781B53EC112B51EC100B89F00CF80FD36F4890ED0C1BB0EE410AF0EE610A9FED721B53EC112BE3
:40F4800051EC100B88F0C2FE08D20020664981F8D50001205B491039087019E0FFF7A7FF60B16A4890F82C005F4981F8D500674890F82C10664880F8481005E0644890F833
:40F4C0004800594981F8D50000204E491039087010BD10B5544890F8D9005E49097888420BD0514890F8D9005A490870032038F073FC40F275104BF04BFA10BD10B52DED4E
:40F50000028B474890F878430E2C20D2DFE804F01F20212216151407251F1F1F232405F08EFBF0EE408A05F055FBF0EE000A80EE201A38EEC18A15E000BF00BF05F07FFBA6
:40F54000F0EE408A05F046FB38EEC08A0AE000BF00BF00BF00BF00BF00BF05F08BFBB0EE408A00BF00BFB0EE480ABDEC028B10BD10B52DED0A8BF0EE408AF0EE609A9FED05
:40F58000360AF4EEC08AF1EE10FA04D2B0EE680ABDEC0A8B10BD9FED310AB0EE40AAFFF7ADFFB0EE40AA29EE8A0AB0EE409A29EE090AB0EE409A28EEA88AB4EEC89AF1EE9C
:40F5C00010FA0FD238EE490A10EE101A084689F04FF941EC1C0BB0EE4C0AF0EE6C0A86F0ABFB01E09FED1E0BB0EE40BAF0EE60BA51EC1B0B88F0BAFA08EE100AB0EE480A03
:40F60000C6E70000C81D0020F971090815710908D81D002030320020316D09081C0000109824002024000010C81C0020000000000080664000000000008066C000000000B4
:40F640000080564000000000008056C0141C002048180020300000102FDDE43E0000000000000000000000002DE9F0412DED108B05460E461446FE4890F8D80030B195EDA2
:40F68000150ADFEDFC0A30EE200A01E095ED150A10EE107A384689F0EBF841EC1F0BB0EE4F0AF0EE6F0A84F05BFFB0EE40DAF0EE60DA51EC1D0B88F059FA08EE900A3846AC
:40F6C00089F0D6F841EC1F0BB0EE4F0AF0EE6F0A86F006FAB0EE40DAF0EE60DA51EC1D0B88F044FA09EE100A17F054FCF0EE40AA1AEE900A89F0BCF841EC1F0BB0EE4F0A70
:40F70000F0EE6F0A86F0ECF9B0EE40DAF0EE60DA51EC1D0B88F02AFA09EE900A1AEE900A89F0A6F841EC1F0BB0EE4F0AF0EE6F0A84F016FFB0EE40DAF0EE60DA51EC1D0B99
:40F7400088F014FA08EE100A1FED3CAACA4890F88E030A280BD11FED3F0AF0EE409A1FED410AB0EE408A1FED430AB0EE40AA05F0E6FAB1EE40EA05F0BFFAF1EE40EA28EEB0
:40F78000880A69EE0A0A00EEA90A20EE0E0A84ED010A28EEA90A69EE0A0A00EEC80AD4ED010A40EE2E0AC4ED010AB1EE490A20EE080A68EE8A0A00EEA90A20EE0E0A84EDF3
:40F7C000000A29EE290A68EE8A0A00EE880AD4ED000A40EE6E0AC4ED000A94ED000A10EE101A084689F044F841EC1D0B9FEDA30B53EC102B88F046FD41EC1B0B94ED010AC6
:40F8000010EE101A084689F033F841EC1D0B95ED301BB0EE410AF0EE610A53EC102B88F093FA41EC1C0B96ED081BB0EE410AF0EE610A53EC102B51EC1B0B88F0C9F941EC6B
:40F840001B0B96ED0A1BB0EE410AF0EE610A53EC102B51EC1C0B88F0BBF941EC1C0B102105F19C00DFF81CC200DF012808D085ED04BB85ED06CB05F19C00DFF80CC200DF48
:40F88000BDEC108BBDE8F08100B5794890F8D210FFF7B2F900B90021084600BD00B5FFF7F3FF032801D1012000BD0020FCE731B5002400BF012269467448006800F50270E7
:40F8C00008F05AFC28B9BDF80000C1B26A4880F8401500BF6420F8F7F7FD204638BD31B5002400BF012269466848006800F2062008F042FC20B99DF800105F4880F83E15C0
:40F9000000BF6420F8F7E0FD204638BD01205A4991F83015032911D1574991F82815062904D2DFE801F003040605070800BF00BF00BF00BF00BF012000BF00BF704710B5A3
:40F940002DED020B0024DDED000A5148008800EE100AB8EE400AF4EEC00AF1EE10FA08DD4B48008800EE100AB8EE400A8DED000A0224484890ED020ADDED000AB4EE600A1F
:40F98000F1EE10FA14D000BF042269463F48006800F5816008F0F0FB20B99DED000A3D4880ED020A00BF5520F8F78EFDFFF7AEFF20461CBD10B5044654B1012C0DD0022CF7
:40F9C00002D0032C13D10DE07F20314908800FE040F6EC102E4908800AE040F6EC102C49088005E040F2FA202949088000E000BF00BF7320F8F768FD10BD31B500241E48AE
:40FA000090F830059DF8001088421ED000BF012269461E48006800F5FC7008F0ADFB20B99DF80010144880F8301500BF9DF80000FFF7C0FF1648008800EE100AB8EE400ACE
:40FA4000FFF77DFF3D20F8F73FFD204638BD31B5002400BF042269460C48006800F5FA7008F08AFB18B904480099C0F82C1513E0C81C0020DC0F4940982400205D091A3451
:40FA800032DCE23EF9710908157109088400001020000010D02B002000BF204638BD31B5002400BF04226946FE48006800F5007008F062FB18B9FC480099C0F8381500BF95
:40FAC000B220F8F701FD204638BD31B5002400BF02226946F348006800F5017008F04CFB20B9BDF80010F048A0F83C1500BF204638BD31B5002400BF01226946E9480068FB
:40FB000000F5FE7008F038FB20B99DF80010E64880F8341500BF3E20F8F7D6FC204638BD31B5002400BF02226946DE48006800F5FD7008F021FB20B9BDF80010DA48A0F899
:40FB4000321500BF204638BD31B5002400BF01226946D448006800F2114008F00DFB20B99DF80010D04880F8491700BF6620F8F7ABFC204638BD10B50120FFF7B0FE002074
:40FB8000FFF795FE0020FFF7DFFF0420FFF7B1FF4FF6FE70FFF7C4FF0420FFF7AAFF4FF6FE70FFF792FF0120FFF727FF012010BD10B5BD4890F82805012806D0022809D0E9
:40FBC000032803D005280DD108E000BF26F07BFD04460BE028F092FE044607E01FF09EFF044603E0FFF7C7FF044600BF00BF3D20F8F76AFC6420F8F767FC6620F8F764FCFF
:40FC00003E20F8F761FC3F20F8F75EFC0421A748DFF89CC200DF012810D0A448007C40F02000A2490874A348C16B4FF48060DFF888C200DF9D48DFF884C200DF204610BDD4
:40FC400073B50C46002500BF012269469548006800F5F87008F090FA20B99DF80010924880F8281500BFA620F8F72EFC6B20F8F72BFC3CB1FFF79CFFFFF778F94FF4E130AB
:40FC8000FFF70DFF28467CBD2DED048BAAB04FF0C8084FF00009E021894881F040FB582114A881F03CFB0020864908738648DFF81CC200DF8648DFF814C200DF8548DFF81C
:40FCC0000CC200DF8448DFF804C200DF8348DFF8FCC100DF8248DFF8F4C100DF8148DFF8ECC100DF76489C30DFF8E0C100DF6F48DFF8D8C100DF73481030DFF8D0C100DF47
:40FD000049F0E6FD6E49C1F89400002081F8DB0001F1B0001AF086FB01F01EF9624890F88E030A2808D100210620FFF789FF4FF4E130FFF7B4FE21E04AF076F840B10021B0
:40FD40000120FFF77DFF4FF4E130FFF7A8FE15E05548D0F83805B0F5966F05D35248D0F83805B0F5E13F04D94FF4E130FFF797FE04E04D49D1F83805FFF791FE4FF4E1306E
:40FD8000FFF765FE484890F83005052808DB0120FFF733FE0120FFF7A2FD0020FFF787FD0321444880F8401000BF0022414640F2FC70DFF834C100DF0546012D6ED0022DE6
:40FDC0006CD1DFF828C100DF044604F00400002865D0FEF711FF0028FAD010213C48DFF8D0C000DF01285BD058223949103114A881F039FA3648DFF8C4C000DF30481CA9B0
:40FE00004EC94EC09DED200A103880ED170A49F05FFD2F49C866012081F880000A46916ED06E49F09FFD324908602948C06E284988660221264878302D4A92ED000AB8EE9C
:40FE4000400A1AF0DEF82248006F29490968884203D9274800681E4908671D48406F24490968884203D22248006819494867FFF715FDB0B9124890F8C80090B11CAA10495A
:40FE8000B03104A81AF013FB1948016804A80BF018FC1CAA0A49B03104A82BE07CE3DCE10FE13AE08400001098240020D81D0020F971090830320020316D09081571090879
:40FEC000C81C0020B81D0020F01200200571090848180020D01800209C190020F0190020481A00209C1B0020916D0908D96C09080C0000101AF055FB0BF02CFD48B10BF08E
:40FF000032FD0646FBF7F4FC0BF02DFD064601F05FFD00200BF021FD12E00BF021FD78B90BF023FD8DED040ACDED050A04A8FBF7DFFC04A801F04CFD01200BF00EFD00BF80
:40FF4000FD4890F8C800E0B1FB4890F8D700C0B117F036F8A8B104AA14A9F748FFF784FB9DED200AF44880ED180AB9F1000F07D104A8FBF7BDFC04A801F02AFD4FF0010927
:40FF80001CE0ED4890F8C80020B91CA9EA48B0301AF057FAE8481CA94EC910304EC09DED200A203880ED180AE44890F8800018B10120E14981F8DA004FF00009DE4890F82F
:40FFC000C80001287DD1DC49B031A1F1A0001AF0C6FA8246BAF1000F23D1D74A103202F1A00168461AF063FA9DED010AFFEE000A20EE200A8DED010A9DED000AFFEE000A6A
:020000040801F1
:4000000020EE200A8DED000ACB49103101F1A0001AF017FA6846FBF76BFC684601F0D8FC00BF9DED180ADFEDC60A20EE200ABDEEC00AC44880ED000A0068C3490968401A12
:40004000C2490860BF480068BF490860BF480068002807DABD4800684EF660210844BB49086006E0B9480068142802DA1420B74908609DF88860B04A02F1B00104A81AF0F8
:4000800016FAB2483146026804A8FBF752FBAA4A103202F1A00102A81AF009FAAB483146026802A8FBF796FA9FEDA90AB0EE408A16F060FFB0EE409AFBF706FCF0EE409AB9
:4000C00000E0BEE0F0EE490AFFF752FAB0EE408A17F09EFA18B1B0EE480A17F013FA05F04CFA70B1944890ED150AB0EE401A974801683046DDED030A9DED020A01F0F9FA60
:400100000DE08D4890ED150AB0EE401A8F4801683046DDED030A9DED020A01F00BF801F07AFCF0EE408A844890F8D70020B901F0ACFC08B1012000E0002083460C217E4810
:400140009C30DFF810C200DF01286AD001F085FC80F00100784981F8D60001F096FC764981F8D70000F00BFF734981F8D80000F006FF714981F8D9000846C0ED198A80ED30
:400180001A8AFBF7C7FBF7EE000A80EE801AB6EE000A31EE000ABCEEC00A10EE100A87B20A2F00DD0A27C7F10A0163484830B0EE480A19F026FFC7F11E015F484030B0EE7D
:4001C000480A19F01EFFFFF784F949F02DFE78B1FBF782FB584880ED1C0AFBF781FB564880ED1D0AFBF774FB534880ED1B0A0AE09FED570A504880ED1C0A9FED550A80ED5D
:400200001D0A80ED1B8ABBF1000F04D04A48C0ED158A80ED168A48489C30DFF83CC100DF00BF464890F88000012809D1424981F8DA004A48416E4FF48050DFF824C100DFD7
:4002400000BF17F096FEFFF7DFF8464A92F83015394A92F8D500FFF76DF804F0100040B3FEF7CAFC28B349F033FB3F49C862012081F83800084690F8390028B9012081F8B9
:4002800039000004FEF7EAFF374A916AD06A49F069FB36490860012133483030334A92ED000AB8EE400A19F0ACFE2F48C06A2E49886204F02000F0B1FEF79EFCD8B149F03B
:4002C00007FB2B494864012081F850000A46116C506C49F047FB25490860012124484830224A92ED000AB8EE400A19F08AFE2048406C1F49086404F48070E0B1FEF77CFCCE
:40030000C8B149F0E5FA1B49C1F8BC00012081F8C8000A46D2F8B810D2F8BC0049F022FB1249086001211348C030104A92ED000AB8EE400A20E027E0C81C002048180020A5
:4003400000007A4414000010100000101800001000000000F97109081571090830320020316D090898240020D81B00200C0000109C190020D018002019F043FEFA48D0F8D4
:40038000BC00F949C1F8B80004F0400010B3FEF733FCF8B149F09CFAF449C1F84401012081F850010A46D2F84011D2F8440149F0D9FAEF4908600121EE48ED4A92ED000AD7
:4003C000B8EE400A19F01DFEE848D0F84401E749C1F8400104F00800F0B1FEF70DFCD8B149F076FAE449C862012081F838000A46916AD06A49F0B6FADD4908600121DE4848
:400400003030DB4A92ED000AB8EE400A19F0F9FDD948C06AD849886204F40070D0B3FEF7EBFBB8B349F054FAD4498864012081F854000A46516C906C49F094FACC4908606D
:400440000121CE484C30CA4A92ED000AB8EE400A19F0D7FDC948806CC8494864084690ED0D0AC74880ED1E0A084690ED0E0AC44880ED1F0A084690ED0F0AC14880ED200A15
:40048000084690ED100ABCEEC00A10EE100ABC49A1F8D00004F4806000287DD00421B948DFF8E4C200DF012876D0B648007C00F0020070B14120F8F707F85C20F8F704F8DC
:4004C0006B20F8F701F8AF48007C20F00200AD490874AC48007C00F0080040B16E20F7F7F3FFA848007C20F00800A6490874A548007C00F0040080B1A44890F8300503287A
:4005000005D19B20F7F7E0FF1B2037F065FC9D48007C20F004009B4908749A48007C00F0100040B14020F7F7CFFF9648007C20F01000944908749348007C00F0200038B137
:40054000FEF761FE8F48007C20F020008D4908748C48007C00F00100B8B3FEF74DFBA0B310218B48DFF820C200DF01282DD020228749103106A880F076FE8548DFF814C2F5
:4005800000DF834890ED070A7D4880ED1E0A804890ED080A7A4800E01BE080ED1F0A7C4890ED090A764880ED200A794890ED0A0ABCEEC00A10EE100A7149A1F8D0007148BC
:4005C000007C20F001006F4908746E48DFF8C4C100DFFEF794FDFEF717FBFEF70DFB08B1FEF70EFA6649D1F8940042F2107149F089F918B10020624981F8DB004020F7F757
:4006000063FFFFF7D2BB5E4890ED160A70475C48D0ED160AB0EE600A90F8D80028B1FFEE000A60EE200AB0EE600A70475448D0ED100AB0EE600A90F8D80028B1FFEE000A40
:4006400060EE200AB0EE600A70474D4890ED100A70474B48D0ED120AB0EE600A90F8D80028B1FFEE000A60EE200AB0EE600A7047434890ED120A704700B5FFF705F90328D6
:400680000BD0FFF701F9062807D0FFF7FDF8052803D0FFF7F9F8042801D1012200E00022104600BD364890F8D5007047344890F8DA00012804D13848007808B90120704763
:4006C0000020FCE73448007B012800D170470020FCE73148007B032801D1012070470020FCE72D48407B082801D1012070470020FCE710B52DED028B244890F878430E2C1E
:4007000020D2DFE804F01F20212216151407251F1F1F232404F093FAF0EE408A04F05AFAF0EE000A80EE201A38EEC18A15E000BF00BF04F084FAF0EE408A04F04BFA38EE1D
:40074000C08A0AE000BF00BF00BF00BF00BF00BF04F075FAB0EE408A00BF00BFB0EE480ABDEC028B10BD0000D0180020481A00200C000010901B00209C1B0020F01900201E
:40078000C81C0020D81D0020F971090898240020141C002015710908B81D002031B5002400BF01226946FA48006800F2072007F0E3FC20B99DF80010F64880F83F1500BF72
:4007C0006420F7F781FE204638BD31B5002400BF01226946EE48006800F2FD1007F0CCFC20B99DF80010EB4880F8351500BF3F20F7F76AFE204638BD38B50446204680F067
:4008000077FC052848D30522E3A1204680F020FCC0B9E34880F06CFC0546E14B04222121009000206EF0ABF9DEA00BF08AFF002010F031FBA220F7F747FE4FF4D0704AF053
:40084000A7F829E00522D8A1204680F001FC18BB49F072FF054625F0ECFC00BF3C22D1A1D34807F089FC20B9CA48CEA1097880F8C01100BF6B20F7F727FEFF200346032264
:40088000012100903D20FAF77EFD4FF48070FEF7E5FC6B20F7F718FE38BD10B5C548FFF7ABFF30224021C44880F00FFD0622C149C14880F05BFD2C20BF4988710622BD4905
:4008C000C91DBD48C01D80F051FD2C20BA4948730622B8490E31B8480E3080F047FD2C20B54908750622B3491531B348153080F03DFD2C20B049C8760622AE491C31AE480E
:400900001C3080F033FD2C20AB4981F82200A948233080F0EDFBC4B2621CA6492331A648233080F023FDA34890F82E0070B1A24880F0DEFBC4B22C209F490855601CC4B25E
:40094000081907229B492E3180F010FD2020FEF785FC10BD10B504462046FFF74DFF204680F0C6FB402803D82146934880F09CFB2020FEF773FC10BD31B500249DF8000000
:40098000032802DD032000900224824890F898079DF80010884212D000BF012269467C48006800F58C6007F0E7FB20B99DF80010784880F8981700BFC020F7F785FD2046C1
:4009C00038BD7D48704770B50546724890F82805012802D0032806D100E000BF284625F081FD044601E06FA070BD00BF2046FBE770B50546674890F82805062819D2DFE8E8
:400A000000F018030904130E00BF284625F0F8FD044610E0284627F0CBFE04460BE028461FF034F8044606E028461DF082FB044601E05CA070BD00BF2046FBE710B55548FB
:400A400090F82805062808D2DFE800F0070309040A0800BF25F0BBFE05E000BF00BF00BF9FED560A00BF00BF10BD0020704710B5484991F82815012906D0022908D00329D1
:400A800003D005290AD106E000BF25F082FE07E027F0F8FC04E01EF0F6FF01E0002000BF00BF10BD2DE9F04781460D461446C846002600270FE02C21404680F0ADFA0646BA
:400AC00026B9AF4201DA4FF0000806E0AF4201DA06F101087F1CAF42EDDD00BFB8F1000F09D01EB1A6EB0800207006E0404680F0FFFA207001E0002020702078102801DC11
:400B0000207810B94FF0000800244046BDE8F08700B5FFF7CBFD08B9002102E02848B0F8D010084600BD1B4890F85707704701B500BF012269461648006800F21F4007F0B8
:400B40001BFB20B99DF80010124880F8571700BF8520F7F7B9FC002008BD0E48B0F8E20400EE100AF8EE400A9FED161A80EE810A7047134890F8DB007047014605292ED243
:400B8000DFE801F0032224272A00002027E00000840000109824002043455354520000001C260020000000004345475053000000C00100688C1C00204C1C0020000000007E
:400BC000C81C002000007A443C2008E04FF4967005E04FF4167002E04FF4B46000BF00BF704711B583B000BF012203A9C54807F0C3FA20B99DF80C00C34981F8000100BF83
:400C000000200290C04991F80001FFF7B6FF0446E0B28DF80800200A8DF80900022002A903461922CDE90010002108466DF0D5FF1FBDB64840687047B44948607047B3485C
:400C400090ED020A7047B14880ED020A7047AF48407B7047AD48007B7047F0B52DED0C8B85B0B0EE408AF0EE608A01279FEDA80B53EC102B51EC180B87F0C8FA0AD2BF1E8D
:400C8000B0EE480AF0EE680A83F0CEFCB0EE408AF0EE608AB0EE480AF0EE680A83F0D0FCB0EE409AF0EE609A51EC190B87F0E0F944B2204687F039FA53EC182B87F016FCF6
:400CC0009FED950B53EC102B87F0DCFA41EC1A0BB0EE4A0AF0EE6A0A83F0B2FCB0EE409AF0EE609A51EC190B87F0C2F945B2C5EB0511880087F019FA41EC1A0B204687F069
:400D000014FA53EC182B87F0F1FB9FED850B53EC102B87F0B7FA53EC1A2B87F0BFFC86F025FF0646304687F0A3FD41EC190B8DED029B04FB07F37CA20F217E4800957FF060
:400D400087FE7C4805B0BDEC0C8BF0BD10B5044600BF0B2221466B480D3007F00DFA40B97548216801606168416021890181A17A817200BF10BD10B5044600BF0B22214606
:400D80006048801C07F0F8F948B96B480B38216801606168416021890181A17A817200BF10BD10B5584991F8281506290ED2DFE801F00D030704090B00BF25F00CFD07E010
:400DC000002005E0002003E0002001E0002000BF00BF10BD00204C4991F82815022900D1012070470020484991F82815052900D1012070470020444991F82815042900D171
:400E00000120704710B500243F4890F82805062809D2DFE800F0080309040A0B00BF25F0DDFC044604E000BF00BF00BF002400BF00BF204610BD10B50446A068606048F0CC
:400E400047FDA060D4E90110401A206010BD10B5FFF72CFC48B1394890ED140ADFED380AB4EE600AF1EE10FA05D1364A36A137487FF0D8FD06E0314B543333A20C21334868
:400E80007FF0E6FD314810BD10B52C4890ED140ABCEEC00A10EE100A80B2FF2805D1294A29A12B487FF0BEFD0CE0244890ED140ABCEEC00A10EE100A83B226A20421244824
:400EC0007FF0C6FD224810BD00B5FEF790FA00BD00B5FEF78CFA10B9FFF784FF08B1012000BD0020FCE710B5FEF781FA38B1FEF7EFF920B148F098FF08B1012010BD00202A
:400F0000FCE700000001006898240020B81D002000000000000000000000000000004E40000000000020AC4025642A256427252E32662200EC1D0020A525002048180020F7
:400F400000007F43C4F1000825730000FB1D00202C000010257500000020FE490870704710B5FD48007840B14FF47A71FB48006848F0C8FC08B9012010BD0020FCE710B5F7
:400F8000FFF7EEFF10B1F648007810BDF5480078FBE710B50446F048047048F099FCEF49086010BD31B52DED040B2DED028BB0EE408A0446FFF7D4FF10B3EA480078E849AF
:400FC0000978884214D0E848007820B9E748DDE9031206C00CE094ED000ADFEDE50AB4EEE00AF1EE10FA03DDDD480078DD490870DC480078DA4909784840DB4908706BE000
:401000000020FFF7C6FF15F0D5FF022861D0D648007818BBB0EEC80ADFEDD60AB4EEE00AF1EE10FA58DD15F0C5FF08B1012000E00020D149087008460078CA490978884219
:4010400004D0CD480078C749087045E0C748DDE9031206C00120C44908703DE094ED000ADFEDC30AB4EEE00AF1EE10FA12DDB0EEC80ADFEDC00AB4EEE00AF1EE10FA05DD0A
:40108000B848007880F00100B64908700020B649087021E0B0EEC80ADFEDB60AB4EEE00AF1EE10FA18DD15F085FF08B1012000E00020B149087008460078AA4909788842F9
:4010C0000AD0AD480078A74908700020A649087002E00020A3490870BDEC028B05B030BDF0EE401AB0EE610A71EEE02AB0EE622AF0EEC22A9FEDA13AF4EEC32AF1EE10FABF
:4011000017D2B1EE003A21EE033AF0EE432AB7EE003AF4EEC32AF1EE10FA03DDB7EE003AF0EE432AB0EE603A02EE223AB0EE430A00BF7047F3B52DED040B2DED108B8BB00F
:401140000546F0EE41AA0C468D480078A84202D1B4F5FA7F0BD98A48057000207D490870884908700BB0BDEC108B06B0F0BD7948007850BB9FED840A844880ED000A9FED7C
:40118000820A834880ED000A7848DDE91B1206C08048DDE91B1206C000207A490870724908707D4908709FED780A7C4880ED000A9FED750A7A4880ED000A012065490870C7
:4011C00048F086FB65490860CCE79DED1C0A7148D0ED010A30EE609A9DED1B0AD0ED000A70EE608A29EE090A08EEA80A10EE101A084687F03DFB41EC1C0BB0EE4C0AF0EE49
:401200006C0A84F099FDB0EE40BAF0EE60BA51EC1B0B86F0ABFC09905248007810B19FED610A01E09FED600AF0EE40DA9DED090AB4EEED0AF1EE10FA45D2584890ED000A8F
:40124000DFED5A0AB4EEE00AF1EE10FA20DD5448D0ED000A514890ED001AC0EE811AB0EE610A4F4890ED001A00EE904AF8EE600A00EE601A80ED001A484890ED001A00EE9D
:40128000904AF8EE600A71EE600AC0ED000A00BF15F070FEF0EE400A00EE104AB8EE401A3F4890ED000A00EE810A80ED000A3B48D0ED000A00EE104AB8EE400A30EE800ABA
:4012C00080ED000A4EE72848007850B39DED1C0A2648D0ED010A30EE600AB0EE409A9DED1B0AD0ED000A30EE600AF0EE408A29EE090A08EEA80A10EE101A084687F0B8FA5A
:4013000041EC1C0BB0EE4C0AF0EE6C0A84F014FDB0EE40BAF0EE60BA51EC1B0B86F026FC0990B0EEC90ADDED090A80EE201AB0EE41BAB0EE4B0A1AF0B9FDB0EE408AB5EE1B
:40134000C09AF1EE10FA39DBF5EEC08AF1EE10FA34D22DE040000010380000103C0000105700001055000010540000105C0000109A99993ED80FC93F560000103333B33EB7
:4013800064000010410000100000000044000010480000104C000010580000106C000010680000109A99193ECDCCCC3D0000FA439FEDFE0A30EE480AB0EE408AB5EEC09A32
:4013C000F1EE10FA0AD2F5EEC08AF1EE10FA05D29FEDF60A38EE000AB0EE408AB5EEC09AF1EE10FA0AD2F5EEC08AF1EE10FA05DB9FEDEF0A30EE480AB0EE408AFEF77EF897
:401400008DED080AEB48007820B19DED080AB1EE400A01E09DED080AB0EE40AA9FEDE60AB4EEC0AAF1EE10FA0AD29DED091AE348D0ED000AB0EE480AFFF752FEB0EE408A90
:40144000DE4880ED008ADE480078A8BBDD48DE4A06CA06C0DC48DDE91B1206C015F08AFDF0EE400A00EE104AB8EE400A9FEDD71AC0EE011A20EEA10AB0EE40BA9DED080A6F
:401480006BEE000A9DED091A80EE810A38EE400ACF4880ED000AC94880ED008A1FED460ACC4880ED000A1FED480ACB4880ED000A0120C349087055E6FFE7C54890ED00DA24
:4014C00078EE4D9A9FEDB90AF4EEC09AF1EE10FA05DD9FEDB70A39EEC00AF0EE409A9FEDBF0AF4EEC09AF1EE10FA05D29FEDB00A39EE800AF0EE409AAE48067809A89DEDA4
:401500001C1ADDED1B0AB0EE690AFFF74BFDAE48DDE91B1206C0B248007850B11FED660AAC4880ED000A1FED680AAB4880ED000A18E6A0480078864242D0AA48007838B9B3
:401540009FED9A0A3AEE800AA14880ED000A02E09F4880ED008A9E4890ED000ADFED940AB4EEE00AF1EE10FA07DD90ED000ADFED900A30EE600A80ED000A954890ED000AE9
:40158000B5EEC00AF1EE10FA07D290ED000ADFED880A30EE200A80ED000A1FED850A8D4880ED000A1FED880A8B4880ED000AFFF7E6FC074615F001FD00208A490870D1E540
:4015C0009FED7D0AB4EEC0AAF1EE10FA24D215F0D1FCF0EE400A00EE104AB8EE401A7E4890ED000A00EE810ADFED780A80EE201AB0EE41BADDED090A8AEE200A20EE0B0AB4
:40160000B0EE40BAB0EE4B0A1AF050FC38EE400A6F4880ED000A3AE01AEE100A87F028F9CDE9060119EE900A87F022F9CDE900019DED000B84F054FA8DED040B099887F0B8
:4016400017F9CDE902019DED040B53EC102B9DED020B51EC100B86F015FE41EC1C0B9DED060B53EC102B86F06FFB41EC1B0B5848006887F0FDF841EC1E0B53EC1B2B86F0B5
:40168000A7FA41EC1F0B86F071FA514908601FEDC20A514880ED000A1FEDC50A4D4880ED000A08E04A4890ED000ADFED410A30EE600A80ED000A464890ED000ADFED3C0A42
:4016C000B4EEE00AF1EE10FAECDC08E0404890ED000ADFED370A30EE200A80ED000A3C4890ED000AB5EEC00AF1EE10FAEED300BF38E573B52DED040B2DED0C8B0446F0EEC2
:4017000041DA0D4638480078A04202D1B5F5FA7F0AD93548047000203449087028490870BDEC0C8B06B070BD3048007810BB1FEDEA0A274880ED000A1FEDED0A1F4880EDFE
:40174000000A2048DDE90C1206C01F48DDE90C1206C000201A49087021490870214908702349088001202149087048F0B1F821490860D5E79DED0D0A1348D0ED010A30EE35
:40178000609A9DED0C0AD0ED000A70EE609A29EE090A09EEA90A10EE101A084687F068F841EC1C0BB0EE4C0A26E00000DC0F4940DA0FC94055000010CDCCCC3E480000103B
:4017C000410000105C0000104C00001000007A44440000106C00001068000010DC0F49C054000010580000106400001040000010660000103C000010F0EE6C0A84F09CFA26
:40180000B0EE40BAF0EE60BA51EC1B0B86F0AEF90AEE100ADFEDACAAB4EEEAAAF1EE10FA00D27DE7B0EEC90AC0EE0A0AB0EE60BAB0EE4B0A1AF03AFBB0EE408AB5EEC09A8D
:40184000F1EE10FA0ADBF5EEC09AF1EE10FA05D21FED2A0A30EE480AB0EE408AB5EEC09AF1EE10FA0AD2F5EEC09AF1EE10FA05D21FED320A38EE000AB0EE408AB5EEC09AE9
:40188000F1EE10FA0AD2F5EEC09AF1EE10FA05DB1FED390A30EE480AB0EE408A8B48007888B98B488B4A06CA06C08A48DDE90C1206C0894880ED008A884880ED008A012040
:4018C000824908702CE7844890ED00DA78EE4D8A1FED4A0AF4EEC08AF1EE10FA05DD1FED4C0A38EEC00AF0EE408A1FED440AF4EEC08AF1EE10FA05D21FED530A38EE800A82
:40190000F0EE408AB0EEE80ADFED750AB4EEE00AF1EE10FA1DD2B0EE4A0AF7EE000AB4EEE00AF1EE10FA03DDF7EE000AB0EE600A6948D0ED000A40EE280AC0ED000A694853
:401940000088002804DD67480088401E6549088012E06548007880F00100634908705E4880ED008A5F480088401C5E490880FFF706FB064615F021FB5648DDE90C1206C05C
:4019800008E0554890ED000A5FED770A30EE600A80ED000A504890ED000A5FED7B0AB4EEE00AF1EE10FAECDC08E04B4890ED000A5FED810A30EE200A80ED000A464890ED7F
:4019C000000AB5EEC00AF1EE10FAEED300BFA7E63F4991ED010AD0ED010A30EE200A81ED010A91ED000AD0ED000A30EE200A81ED000A384991ED010AD0ED010A30EE200AB7
:401A000081ED010A91ED000AD0ED000A30EE200A81ED000A7047304890ED000A704710B5FFF79EFA28B13048007830490978484010BD2F480078FBE770B50446FFF790FA86
:401A400018B12A480578047006E027480578047085EA04002749087070BD2748007828B11A48007810B12248007808B1012070470020FCE710B5FFF782FA20B9FFF7EDFFA9
:401A800008B9012010BD0020FCE71B48007820B10E48007808B1012070470020FCE713490870704710B5FFF76AFA08B1002400E00124204610BD114890ED000A70470F48B9
:401AC00080ED000A70470000CDCC4C3E410000105C0000104C0000104400001048000010D80FC93F660000105500001057000010540000105800001040000010340000103F
:401B000010B57D231A46D900012032F0FBFB10BD10B57D231A469900012032F0F3FB10BDF94991F89907704700B5FFF7F9FF042801D1012000BD0020FCE7DFEDF40AB0EE99
:401B4000600A04280BDAF24901EB0011497B31B1EF4901EB0011D1ED000AB0EE600A704710B5EC480478FFF7DBFF06287ED2DFE800F00304180524AFAEE000BFE448407FA7
:401B800018B10120E34908700AE0E14890F83D0018B10320DF49087002E00020DD4908709AE0DB4890F82D0018B10220D949087002E00020D74908708EE0D548407F70B3B5
:401BC0000AF0E5FC40B90AF009FD28B90AF0F9FC10B90AF0E9FC18B3CD4890F82D00F8B1CC48007802280DD008F061FE032817D10120FFF7A2FFDFEDC80AB4EEE00AF1EE9D
:401C000010FA0DD20220C3490870C148D0ED040AB0EE600A1921C14818F0F3F956E00EE00120BC490870BA4890ED040ABB48D0ED000A30EE600AB64880ED040A46E0B448C6
:401C400090F83D0078B30AF0A2FC40B90AF0C6FC28B90AF0B6FC10B90AF0A6FC20B3AC4890F82D0000B3AB48007800E02FE002280CD008F01CFE032816D1FFF75EFFDFED63
:401C8000A60AB4EEE00AF1EE10FA0DD20220A14908709F48D0ED0C0AB0EE600A19219F4818F0AFF912E00EE003209A490870984890ED0C0A9948D0ED000A30EE600A94482C
:401CC00080ED0C0A02E000209249087004E000BF00209049087000BF00BF0AF058FC40B90AF07CFC28B90AF06CFC10B90AF05CFCF0B188480078A04222D0FFF715FF80B16B
:401D000084480078012803D082480078032802D1FFF7FEFE05E07F480078022801D1FFF7EFFEC120F6F7D0FB072036F055F807E09FED760A794880ED000A00207749486048
:401D40007748D0F854110120DFF8D8C100DF10BD31B500249DF80000052801DB02241BE09DF80000002801DC032415E000BF012269466D48006800F2614006F0FDF920B9B5
:401D80009DF80010604880F8991700BFC220F6F79BFB072036F020F8204638BD10B51620F6F792FB5320F6F78FFB1720F6F78CFB1820F6F789FB262036F00EF810BD0121B6
:401DC000574880F8541026F0C9FD074627F044F927F018FBFFF7E2FF00204E490870FFF79FFE18B1FFF79CFE052802DB0120FFF7AFFF4A4800210160416000240AE000201D
:401E0000434901EB04110873414901EB04114873601C84B2042CF2DBDFF810C100DF804669224146012047F032FE38B1DFF8FCC000DF80464146012047F058FEDFF8ECC0E5
:401E400000DF804641460220DFF8D8C000DF002F3CD10321324880F8541000BF00224FF6FF710720DFF8C8C000DF0546022DF5D1DFF8C0C000DF0646304626F0C2FD304692
:401E800027F0F5F8304627F0C9FA06F001000028E4D01F4A1832111F081F26F0A5FF1C49487701F138023431081F27F028F9184981F83D0001F128022431081F27F00CFB56
:401EC000134981F82D00FFF74BFEC7E70020DFF868C000DF00BFFEE70E48007808B1012070470020FCE72DE9F05F2DED028BB0EE408A05460F46904699460C9E4FF0000B32
:401F0000DA460FFA88F45FE09824002000000000C00C001050000020BF0E1C3E5400002030320020316D0908840000102D7A0908916D0908D96C090871780908A21905EB73
:401F4000C20105EBC40018F0BFFEF0EE408AF4EEC88AF1EE10FA2FDDC8EE280AB0EE600AA01905EBC000D0ED010A05EBC40090ED011A30EEC11A05EBC400D0ED010A41EE43
:401F8000000AC7ED010AA01905EBC000D0ED000A05EBC40090ED001A30EEC11A05EBC400D0ED000A41EE000AC7ED000AA14678EE680AB0EE608A0EE038EE680AB0EE408A3D
:401FC000A01904B20AF1010A04FB06F0484502DABAF1280FB2D300BFB5EEC08AF1EE10FA01DD4FF0010B5846BDEC028BBDE8F09F2DE9F04F2DED028B83B005460E4691463C
:402000009B46F0EE408ADDE90E4A00200290AAF10100A04201D2044602E0002C00DA002406EBC401284618F04FFEB0EE408AB4EEE88AF1EE10FA28D2109858B9BBF1000F54
:4020400003D000274FF0FF380FE0AAF101074FF001080AE0BBF1000F04D0AAF101074FF0010802E000274FF0FF3838EEC80AF0EE408A3B46224649463046B0EE680ACDF8D0
:402080000080FFF730FF029020E0C8EE880AB0EE600A06EBC400D0ED010A95ED011A30EEC11AD5ED010A41EE000AC9ED010A06EBC400D0ED000A95ED001A30EEC11AD5EDEC
:4020C000000A41EE000AC9ED000A00BF029803B0BDEC028BBDE8F08F2DE9FF4F2DED020B2DED068B8BB00E461746F0EE408A99464FF0000AF2EE020AB2EE040A83F0BCF9C3
:40210000B0EE40AA1FED7F0AB0EE408A07F10C040025B9F1020F02D24FF0010A85E14FF0000B2BE01398D0ED010A06EBCB0090ED011A70EEC10AB0EE600A18F0C3FBB0EEFD
:40214000409A1398D0ED000A06EBCB0090ED001A70EEC10AB0EE600A18F0B4FB39EE000AB0EE408AB4EECA8AF1EE10FA02D25D46B0EE48AA0BF101000FFA80FBCB45D1D324
:40218000A846A9F1010000B205900598804503D1A8F101000FFA80F808F1010206EBC20106EBC80007F1500219F0D6F8B0EE408AB5EEC08AF1EE10FA01D2012000E0002042
:4021C00087F8580097F8580010B14FF0FF3000E001200690B5B96A1C06EBC20106EBC500139A19F0CEF8B0EE408AB5EEC08AF1EE10FA01D24FF0010A97F8580078B3681C90
:4022000005B22CE00598854216D16A1E06EBC20106EBC500139A19F0B4F8B0EE408AB5EEC08AF1EE10FA01D24FF0010A97F85800A8B9681E05B212E0069A2A4406EBC201A8
:4022400006EBC500139A19F09CF8B0EE408AB5EEC08AF1EE10FA02D20698281A05B206EBC50103C9C4E905010698284406EBC00106C9C4E9071204F11C0204F1140104F11C
:40228000240018F0E5FF657094ED090A8DED040A94ED0A0AB1EE400A8DED030A03AA04F11401139819F08AF8B0EEC00AB0EE408A94ED060AD4ED0A0A08EE200A84ED020A58
:4022C00094ED050AD4ED090A08EE200A84ED010AD6E90001CDE90701D6E90201CDE909019DED0A0ADDED080A30EE600A84ED040A9DED090ADDED070A30EE600A84ED030ADF
:40230000D6E90001C4E90B01D6E90212C4E90D12D6E90212C4E90F12B9F1020F7ED9BAF1000F7BD1387A00EE100AB8EE400AF7EE080A20EE200AB0EE409AA8460120CDE9B6
:402340000089029097F85830B0EE490A07AA3146201DFFF74DFE40EA0A0A069828440FFA80F80020CDE90089029097F85830B0EE490A09AA3146201DFFF73AFE40EA0A0AFF
:402380009DED0A0ADDED080A30EE600A84ED040A9DED090ADDED070A30EE600A84ED030AA846787A00EE100AB8EE400AF7EE080A20EE200AB0EE409A0120CDE900890290AD
:4023C00097F85830B0EE490A04F12C023146201DFFF70EFE40EA0A0AD4E90112C4E90D12069828440FFA80F897ED010A20EE280AF0EE409AF4EEC99AF1EE10FA01DDB0EE66
:40240000699A0020CDE90089029097F85830B0EE490A04F13C023146201D00E004E0FFF7E7FD40EA0A0A00BF00BF50460BB0BDEC068B06B0BDE8F08F10B52DED028BF0EEB0
:40244000408A044694ED001AF0EE410A94ED011AB0EE410A18F056FAB0EE408A38EE680AB0EE408A05E09FEDF00A38EE000AB0EE408A9FEDEE0AB4EEC08AF1EE10FAF2D31E
:4024800005E09FEDE90A38EE400AB0EE408A9FEDE80AB4EEC08AF1EE10FAF2DCB0EE480ABDEC028B10BD10B5E248016D012047F053FBE048016D0120DFF87CC300DF10BD50
:4024C000DFEDDE0AB0EE600A04280BDADC4901EB0011497B31B1DA4901EB0011D1ED010AB0EE600A7047DFEDD50AB0EE600A04280BDAD34901EB0011497B31B1D04901EB17
:402500000011D1ED020AB0EE600A704701460020042903DACA4A02EB0112507B70470146C848B0F8E20400EE100AB8EE400ADFEDC60A30EE600ADFEDC40A80EE201A81ED49
:40254000001AC04890F8E02400F2E44000EB8202BC4890F8E10432F8100000EE100AB8EE400ADFEDB90A30EE600A9FEDB71AC0EE010AB0EE000A30EE800A81ED010AB14896
:4025800090F8EC040872AF4890F8EE04487201207047AE480078704731B50024BDF90000B0F57A7F04DD4FF47A700090022406E0BDF90000002802DA00200090032400BFA9
:4025C00002226946A248006800F5D57005F0D4FD28B9BDF8000081B29A48A0F8E21400BF1620F5F771FF262035F0F6FB9148016D0220DFF844C200DF204638BDF7B50C4652
:4026000015460026BDF90000B0F5FA7F04DD4FF4FA700090022606E0BDF90000002802DA0020009003268B4800EB840030F81500BDF90010884222D000BF8549096801F591
:40264000D67101EB840101EB45000222694605F093FD38B9BDF8000081B27E4800EB840020F8151000BF5320F5F72EFF262035F0B3FB7048016D0220DFF8BCC100DF304679
:40268000FEBD31B50024BDF800000A2803DD0A200090022406E0BDF80000012802DA01200090032400BF022269466948006800F5DA7005F061FD20B9BDF800106148A0F81A
:4026C000EC1400BF1720F5F7FFFE262035F084FB5848016D0220DFF860C100DF204638BD31B50024BDF800000A2803DD0A200090022406E0BDF80000012802DA01200090AD
:40270000032400BF022269465148006800F5DB7005F032FD20B9BDF800104A48A0F8EE1400BF1820F5F7D0FE262035F055FB4148016D0220DFF800C100DF204638BD4648CC
:402740008078FE2801D0012070470020FCE743488078FE2801D0012070470020FCE700B5FFF7DEF9042807D0FFF7DAF9032803D0FFF7D6F9012801D1012000BD0020FCE74D
:4027800000B5FFF7CDF9042803D0FFF7C9F9022801D1012000BD0020FCE7314890ED000A704700B5FFF7BCF9022801D1012000BD0020FCE700B5FFF7B3F9022801D10120AC
:4027C00000BD0020FCE700B5FFF7E3FE042801D1012000BD0020FCE701B500BF012269461B48006800F2534005F0C6FC20B99DF80010144880F88B1700BF08BD08B5FFF735
:40280000A6FF38B91748144B01220321009016483AF0D8F908BD00B5FFF7B2FF08B1002200E00022104600BDDC0F4940D80FC9BFD80FC93F30320020316D09080000000000
:40284000C00C0010982400200000C84250000020840000107C290020206E0220E06E022054000020887C02207E030800FE4908707047FE4908707047FD480078092801D1DE
:40288000012070470020FCE7F94800780B2801D1012070470020FCE7F5480078012800D170470020FCE7F2480078062801D1012070470020FCE770B58CB004460D46E217B7
:4028C00004EBD2625311EB4A02EB830212682146E31704EBD3635B11A4EB43160123B3401A432046E31704EBD3635E11E14B03EB86031A60E0480470FFF7D5FF40B9FFF77C
:40290000BBFF28B9FFF7C8FF10B9FFF7BDFF40B1FFF7B2FF28B91E2D03D10120FFF7A9FF13E0D64BD6A2232102A800957EF090F802A87EF0DDFB461C314602A86DF078FE22
:4029400001212846FAF792FC00BF1F2D03D029460C206CF097F8ECB30421CC48DFF830C300DF012818D0C94890F82E1090F82E00401CC64A82F82E0002F1100044541038CE
:4029800090F82E001E2803DB0020114681F82E00BE48DFF800C300DF0421BF48DFF8F0C200DF012818D046F093FFBC4941F83400084600EBC4000079FF2807DA084600EB0A
:4029C000C4000079401C01EBC4010871B248DFF8C4C200E000E000DF1F2035F0FDF90CB070BDAF48807F012800D170470020FCE7AB48C07F08B9012070470020FCE710B59E
:402A000076F048FF01280FD176F005FF60B175F014FD012808D17BF079FE012804D1FFF7E7FF08B1012010BD0020FCE710B5044602F0A3FD08B1022C01D1012010BD00201F
:402A4000FCE770B504460D46607B012824D1A06868B1D4E9010146F055FF002871D000221146204619F097FF0120E07369E02846FFF7DCFF002864D04FF4FA61606846F073
:402A800041FF00285DD00220A0731C210820FFF712FF09F02FFE54E0A07B022802D10020A0734EE0207B01284BD10020E07309F06EFD28B909F078FD10B909F08FFD30B1D8
:402AC00009F018FE1D210320FFF7F5FE39E0FFF796FF58B1FBF758FE40B909F00FFE09F0FDFD20210020FFF7E6FE2AE075F0A5FC012804D01F210420FFF7DDFE1FE076F0B4
:402B0000C9FE012804D012210320FFF7D4FE16E076F081FE20B911210120FFF7CCFE0EE0FBF732FE38B1FBF73DFE064631460920FFF7C1FE03E01E213120FFF7BCFE09F009
:402B4000D9FD207B617B884202D03820F5F7BCFCE07B08B9607B207370BD0020514908707047F0EE400A9FED501A20EE811AB0EE410A9FED4E1A30EE011AB0EE410AB1EE6B
:402B8000001A20EE011AB0EE410AB6EE001A30EE011AB0EE410A9FED461AB4EEC10AF1EE10FA03DD9FED421AB0EE410ABCEEC01A11EE100A80B2704700B52DED028B81B003
:402BC0003C4890F8240001281DD13A4890F82500012818D1FFF767FE40B9FFF74DFE28B9FFF75AFE10B9FFF74FFE38B10120314981F8260046F06CFE2E49486000202D4905
:402C000081F8250080E02B49086846F09CFEB0F57A7F79D3274890F82400012874D1042124480830DFF868C000DF01286CD0DFED220A9FED210A7AF089FDB0EE408AFFF766
:402C400090FF1C494883DFED1C0A9FED1B0A7AF07DFDB0EE408AFFF784FF16490883012081F82200022029E06A0000206B0000205D00002019230020600000207EB10908AE
:402C8000257320636F64653A20256400E8220020F971090815710908D8220020D8200020882000206C00002000007A440000FB4500FF7A47B02000200000000081F82100D4
:402CC00000208877022081F8200091F8200075F021FB0020FA49C8774520F5F7F5FB0020F74981F82400012081F82500FFF735FFF3480830DFF8CCC300DFF348D0F81C121E
:402D00000120DFF8C8C300DFED4890F8260020B3EB49486846F017FE40F6C41188421CD3EB4800680090EB4890F8E024EA4803210368EA4839F046FFE54800680090E548EB
:402D400090F8E124E44803210368E448973039F039FF0020DA4981F8260001B0BDEC028B00BDDF480078C0F380007047DC480078C0F340007047DA48007800F00100704720
:402D8000D7480078072801D1012070470020FCE7D4490870704710B502F0D2FF30B1002213466021D04827F0D4FE3AE003F05EF830B1002213462721CB4827F0CAFE30E0E5
:402DC00002F02DFC30B100221346D221C74827F0C0FE26E003F062F830B1002213460621C14827F0B6FE1CE003F002F830B1002213463121BC4827F0ACFE12E003F005F89D
:402E000030B1002213460621B74827F0A2FE08E002F09EFF28B100221346FC21B24827F098FE10BD10B5002402F08AFF70B902F0DFFF58B902F0E9FF40B902F089FF28B961
:402E400002F0EDFB10B903F029F800B10124204610BD70B504460225112C02DA0025A44804708820F5F730FB284670BD10B502F067FF88B10820FFF7ECFF002213461321F6
:402E80009C4827F066FE9B48934908609A489049086000209649887002F0AFFB88B10D20FFF7D7FF002213461321924827F051FE90488949086090488549086000208C49A0
:402EC000887002F0AFFFC0B10E20FFF7C2FF00221346F021874827F03CFE00221346F0218448C03027F035FE82487B49086082487749086000207E49887002F09BFFA0B102
:402F00000F20FFF7A6FF0022134627217948C03027F01FFE7748C0306F490860764828306B49086001207249887010BD10B50020FFF78FFF01216848006827F025FE02207E
:402F40006B49887010BD10B5002402F0F9FE40B902F070FF28B902F065FF10B902F04DFB00B10124204610BD5E480078704710B50121624827F008FE10BDF0EE400A9FED65
:402F8000601A9FED600A00EE810A70474C48808B00EE100AB8EE400A704710B52DED028B0024FDF730FBB0EE408A09F05BFA98BB08F049FB00B12FE008F03CFBA0B1FFF7F9
:402FC000E5FFB0EE408A05214F4817F01AF84E4890ED000AF6EE000A30EE200ABCEEC00A10EE100A84B217E03548408B00EE900AF8EE600AB0EE600A0521434817F001F8CA
:40300000414890ED000AF6EE000A30EE200ABCEEC00A10EE100A84B235480078112877D2DFE800F0EB3BB0090AEA3C0B0C980D77EA0E100F110000BF00BF00BF00BF00BF35
:4030400000BF00BF00BF09F0A2FA40B909F0C6FA28B909F0B6FA10B909F0A6FAE0B1FDF7D2FAB0EE408A09F0FDF930B9FDF7CBFAB0EE408A72F038FC70B176F002FFDFED44
:40308000230AC0EE208A79F015FA38EE800AB0EE408AFFF766FD0446B2E000BF09F077FA68B1FDF7B0FAB0EE408A09F0DBF930B107F0BCFCB0EE408AFFF753FD04469FE0AA
:4030C000B02000201571090830320020316D0908880400209824002084040020580108006C0000205C000020A0780220E07702205D00002060730220607C02206079022061
:403100000000C84200401C462C02002000007A4572E009F03CFAE0B1FDF775FAB0EE408A09F0A0F9A8B108F078FA38B107F07EFCB0EE408AFFF715FD04460AE007F076FC3D
:40314000B0EE408AFFF719FFBCEEC00A10EE100A84B255E009F01BFA98B1FDF754FAB0EE408A09F07FF960B107F060FCF0EE408A7AF033FF38EE800AB0EE408AFFF7F1FCCD
:4031800004463DE073F0FAFE07280FD2DFE800F00508040F06070B0000BF00BF00BF00BF4FF6FF7426E0FE48048B23E000BF09F0EEF940B909F012FA28B909F002FA10B980
:4031C00009F0F2F9A8B1FDF71EFAB0EE408A09F049F970B176F055FE5FED340AC0EE208A79F068F938EE800AB0EE408AFFF7B9FC044600BF00BF03E000BF4FF6FF7400BFB9
:4032000000BF2046BDEC028B10BD50274FF000084FF000090020E34908700121E24880F88011DF480830DFF884C300DFE048DFF87CC300DFDF48DFF874C300DF08F097FF2C
:403240000020D74981F82400012081F82500002081F82600FFF7FDFD0220D74988700020FFF796FD76F09FFC0020D44908700321CD4880F8801100BF002239460720DFF8CA
:4032800040C300DF84B2022C0DD1DFF838C300DF804608F0020030B1FFF77FFECA490880012034F099FD012C7ED1C84890F88503092803D1502073F0E8FE00E000BF00BFF7
:4032C00002F09BF960B10120C149487071F031FF30B972F082F871F02CFF08B1FFF747FE3BF034FEE0B10CF037FEC8B109F0E6FFFA2803D009F0E2FFFB2811D1FFF734FE0C
:4033000070B9FFF720FE18B1FFF710FEFFF7AEFDFFF788FD08B1FFF73EFD0120FFF738FDFFF7C1FA40B9FFF7A7FA28B9FFF7B4FA10B9FFF7A9FA80B3FFF722FD68BB484610
:4033400046F001FB42F21071884226D3FFF713FD40B9A0480368A048002102684FF6DA602FF073FBFFF702FD40B99A4803689A48002102684FF6C5502FF067FBFFF7F1FC6C
:4033800040B9944803689448792102684FF46F402FF05BFB46F09CFA8146102180480830DFF838C200DF00E0D5E0012809D028227B498B487DF057FF79480830DFF824C221
:4033C00000DFFFF7F9FB76F06AFB76F014FC00218548FFF736FB01218448FFF732FB02218348FFF72EFB03218248FFF72AFB04218148FFF726FB05218048FFF722FB06215A
:403400007F48FFF71EFB73F06BFB09F0C0F840B909F0E4F828B909F0D4F810B909F0C4F808B1012000E000200646002E7BD0012074490870FFF7DCFA30B1FFF7D2FAC0BB6B
:403440007148007814283ADB09F054F976F022FA012804D012213420FFF72DFA79E076F0DAF920B911213420FFF725FA71E074F0E4FF012804D01F213420FFF71CFA68E0DE
:4034800009F092F8B0B909F09CF898B909F0A6F880B9FBF779F968B1FBF784F90546C5EB05115A4A02EB8101887B2946FFF703FA4FE004E01E213420FFF7FDF949E009F049
:4034C00073F828B909F07DF810B909F087F878B14F48406800F48030B0F5803F08D04C48007900F00200022802D009F003F930E009F05AF8C0B909F064F8A8B909F06EF8B0
:4035000090B9FBF741F978B1FBF74CF9054609F0F1F8C5EB05113D4A02EB8101887B2946FFF7C9F915E009E037480078142810DA35480078401C344908700AE03148007887
:4035400038B10020FFF792F900202F4908702D49087008F01FFE4FF000088DE6104890F8240008B9012070470020FCE710B50D2128487DF0D4FE10BD70B50023012152E049
:40358000CC1701EBD4646511224C641C04EB85042468CD1701EBD5656D11A1EB45163BE0B02000206A0000203032002005710908E8220020D82200205D0000206C00002042
:4035C000916D0908D96C09086800002098240020607C02208804002084040020F9710908882000201571090850BF001060BF001070BF001080BF001090BF0010A0BF00102C
:40360000B0BF00102902002028020020348B0908FC0B0010182300200125B5402C4004B10B46481CC1B24029AADB184670BDFC4890F820007047FA4890F821007047F948D1
:403640000078022801D1012070470020FCE710B5FFF7F5FF18B173F097FC044602E0F04890F82340204610BDEF4800887047B0F57B4F01DB4FF6FF2000EE900AF8EE600A0E
:40368000B1EE001AC0EE811AB0EE610ADFEDE70A70EE600AB0EE600ADFEDE50A80EE201AB0EE410A7047E348408B704700B5FFF76DFCDFEDE10A70EE600A9FEDDD1A80EE3E
:4036C000810A00BDF0EE400A9FEDDB0A30EEC01ADFEDDA1A81EE210A704700B5FFF756FCB0EE402AFFF7EEFF00BD10B5D448007808B1FF2010BD08F04AFF40B908F06EFF9E
:4037000028B908F05EFF10B908F04EFF08B1012000E0002020B1CA48007808B9012000E0002040F0FC00E5E7BE4800780D2801D1012070470020FCE7BA4800780E2801D154
:40374000012070470020FCE72DE9F0472DED048B07460C4692469846DDF8309001F05FFF30B1A078FD2803D1BDEC048BBDE8F087FFF7E2FF28B1B3480068C078404500D059
:40378000F2E70025FFF7D0FF18B1204671F006FD0DE0B7F52C4F01D1002508E0B7F56F4F04D12078AC2801D1012500E0DCE75021A0480830DFF890C200DF012861D0615DC9
:4037C000681C205C41EA00269A48068302F0A3FF30B1984886830020964981F822001EE0B6F57B4F15DBFCF712FFF0EE408A13F0C1FBB0EE409AF0EE680A79F0A7FFB0EED2
:40380000408AFFF7AEF98B494883012081F8220005E0884846830020864981F82200A81C205C00F00300834981F82100A81C205CC0F381008877A81C205CC0F3011081F835
:403840002000A81C205C8009C87791F8200074F061FD46F03DF877490860012081F82400E81C205C400981F8230001F10800DFF8DCC100DF7648D0F81C120120DFF8D4C171
:4038800000DF00BF70E76748007808B1012070470020FCE770B5044600256F4890F88E03FF2800D1A3E0092C06D16B4890F88403032801D001259AE0012C06D1664890F8D5
:4038C0008403032801D0012591E0062C06D1624890F88403032801D0012588E0042C14D15D4991F88E0302F016FA07280BD05A4890F87C03172808D1574991F88E0302F014
:403900000AFA012801D1012571E0072C14D1524991F88E0302F0FFF908280BD04E4890F87C03172808D14C4991F88E0302F0F3F9012801D101255AE0022C14D1464991F887
:403940008E0302F0E8F909280BD0434890F87C03172808D1404991F88E0302F0DCF9012801D1012543E00A2C14D13B4991F88E0302F0D1F90B280BD0374890F87C03172837
:4039800008D1354991F88E0302F0C5F9012801D101252CE0032C14D12F4991F88E0302F0BAF90A280BD02C4890F87C03172808D1294991F88E0302F0AEF9012801D1012588
:4039C00015E0102C13D1244991F88E0302F0A3F916280BD0204890F87C03172807D11E4991F88E0302F097F9012800D10125284670BD10B5012402F0A3F900B1002420468D
:403A000010BD70B504460E460025FFF7F2FF00285DD001F0B2FD08B30B2C58D1012556E0882000205D000020680000200000FB4500007A44B020002000401C460000C84217
:403A40006A00002084040020F97109081571090830320020316D090898240020D6B9012C03D0092C01D0062C08D12046FFF712FF054605B30020F749887028E0F548807850
:403A8000C8B12046FFF706FF0546A5B10020F14988701CE0EF48807868B1012C03D0092C01D0062C08D12046FFF7F4FE054615B10120E84988700AE0FFF7E5FE38B9204621
:403AC000FFF7E8FE054615B10120E2498870012D04D1FFF7D8FE08B1FFF728FA284670BD2DE9F0418CB0074688460025002F7CD0F220012102220023CDE90532CDE90710E7
:403B0000042010210193CDE90231049097201A46194600900AA826F02AFE0AA9384626F02EFA044604F0F204384627F05EF80646F22C0BD1022E09D145B941460B20FFF7A5
:403B400060FF18B10B20FFF784F90125F220012102220023CDE90532CDE9071010210193CDE9023197201A461946049300900AA826F0FDFD0AA9384626F001FA044604F097
:403B8000F204384627F031F80646F22C0CD1012E0AD14DB941460920FFF733FF20B10920FFF757F901251BE0F22C0CD1022E0AD14DB941460120FFF724FF20B10120FFF70C
:403BC00048F901250CE0F22C0AD14EB945B941460620FFF716FF18B10620FFF73AF901259A2001210222002300E0E4E0CDE90532CDE9071051210193CDE9023197201A46F7
:403C00001946049300900AA826F0B1FD0AA9384626F0B5F9044604F09A049A2C09D145B941461020FFF7EDFE18B11020FFF711F901259620012100220592CDE9062108905C
:403C400010210192CDE90221392013461146049200900AA826F08BFD0AA9384626F08FF9044604F09604962C09D145B941460420FFF7C7FE18B10420FFF7EBF801259620DF
:403C8000012100220592CDE90621089010210123CDE9013239201346CDE90312009011460AA826F064FD0AA9384626F068F9044604F09604962C09D145B941460720FFF72B
:403CC000A0FE18B10720FFF7C4F801259220012102220023CDE90532CDE9071086210193CDE9023121201A461946049300900AA826F03DFD0AA9384626F041F9044604F07D
:403D00009204922C09D145B941460220FFF779FE18B10220FFF79DF801259A20012102220023CDE90532CDE907108621CDE9013266201A46CDE90313009019460AA826F0CF
:403D400016FD0AA9384626F01AF9044604F09A049A2C09D145B941460320FFF752FE18B10320FFF776F801259A20012102220023CDE90532CDE9071086210193CDE90231F5
:403D800066201A461946049300900AA826F0EFFC0AA9384626F0F3F8044604F09A049A2C09D145B941460A20FFF72BFE18B10A20FFF74FF8012515B16A20F4F785FB2846E9
:403DC0000CB0BDE8F08123480078102801D1012070470020FCE71F480078082801D1012070470020FCE71B4800780F2801D1012070470020FCE717480078032801D10120B9
:403E000070470020FCE7134800780A2801D1012070470020FCE70F480078042801D1012070470020FCE70B480078072801D1012070470020FCE7074800787047064890F873
:403E400022007047044890F8240008B1012070470020FCE75D000020B02000207748704710B5774890F87C03122805D100221346D721744826F06DFE10BD00B5FFF7C3FF75
:403E800010B9FFF7DCFB08B1012000E000200146084600BD6C49097801436B4A117070472DE9F04781460C4692461D46DDF8208066480068C078A84240D100232022644968
:403EC00020463DF0A0F818B9202161487DF005FA012320225E49203120463DF094F820B920215B4820307DF0F8F9022320225849403120463DF087F820B9202154484030D7
:403F00007DF0EBF9032320225149603120463DF07AF828B920214E4860307DF0DEF90AE010214B48603005F0A8F8064674F0A6FF0120FFF7AFFF4220F4F7C6FABDE8F087F6
:403F40002DE9F04107460C4690461D46069E3F480068C078A8425ED1002320223D4920463DF0B8F818B920213A487DF0B6F9012320223849203120463DF0ACF820B92021D7
:403F8000344820307DF0A9F9022320223149403120463DF09FF820B920212E4840307DF09CF9032320222B49603120463DF092F820B92021274860307DF08FF904232022A7
:403FC0002449803120463DF085F820B92021214880307DF082F9052320221E49A03120463DF078F820B920211A48A0307DF075F9062320221749C03120463DF06BF820B921
:4040000020211448C0307DF068F90220FFF742FF4220F4F759FABDE8F0810F480078704710B501F0AAFA20B1054890F88603012801D0012010BD0020FCE700008820002054
:4040400098240020607902206C0000208404002032230020B22300206B0000200021FE4A1180FE4A1180FE4A1170704770B5FD4890F88E4390F88453C4EB041101EB4101D9
:40408000F94A02EB011101F5F471C5EBC50231F8220001213EF09FFCC4EB041101EB4101F14A02EB011101F5F471C5EBC50201EB8201488801213EF0CBFCC4EB041101EBB2
:4040C0004101E94A02EB011101F5F471C5EBC50201EB8201888801213EF0F7FCC4EB041101EB4101E04A02EB011101F5F471C5EBC50201EB8201C88801213EF023FDC4EBED
:40410000041101EB4101D84A02EB011101F5F471C5EBC50201EB820108893EF050FDC4EB041101EB4101D04A02EB011101F5F471C5EBC50201EB820148893EF076FDC4EB61
:40414000041101EB4101C84A02EB011101F5F471C5EBC50201EB8201087B3EF09CFDC4EB041101EB4101C04A02EB011101F5F471C5EBC50201EB8201887B3EF0F4FDC4EB53
:40418000041101EB4101B84A02EB011101F5F471C5EBC50201EB8201487B3EF0B0FDC4EB041101EB4101B04A02EB011101F5F471C5EBC50201EB8201C87B3EF014FE70BD00
:4041C00033B581B00C460025A64890F88403032815D100BF012201A9A44800684D3003F0CBFF20B99DF804109E4880F8851300BFAF20F4F769F92D2033F0EEFD5CE0BCB9A8
:40420000FEF751FB40B9FEF737FB28B9FEF744FB10B9FEF739FB58B195480068009095489DF8042003210368934838F0CBFC43E0FCB190480068C078A0421AD0FEF733FB12
:4042400058B9FEF719FB40B9FEF726FB28B9FEF71BFB10B9FEF710FB58B185480068009084489DF8042003210368834838F0AAFC22E0FEF718FB40B9FEF7FEFA28B9FEF71F
:404280000BFB10B9FEF700FBB0B17A480068C078A04211D100BF012201A9744800684D3003F06AFF20B99DF804106E4880F8851300BFAF20F4F708F928463EBD31B50024FA
:4042C00000BF012269466948006800F2454003F053FF20B99DF80010624880F87D1700BF204638BD70B55F4890F88E5390F88443C5EB051101EB41015B4A02EB011101F5F8
:404300001D7104EB440211F81200FFF7D7FFC5EB051101EB4101544A02EB011101F51D7104EB440201EB42014878012138F052FEC5EB051101EB41014B4A02EB011101F582
:404340001D7104EB440201EB42018878002138F041FE00209FED490A78F049FE00209FED480A78F0A5FD00209FED460A78F063F9032C01D0042C2DD1C5EB051101EB41012B
:40438000394A02EB011101F2922111F83400002175F0BCFAC5EB051101EB4101324A02EB011101F2922101EBC4014878002173F033FFC5EB051101EB41012B4A02EB0111B8
:4043C000383104EB440202EBC40211F822000021FFF7F6FE70BD2DE9F04104460F462FF0F6FB804656F093F91E4890F88E5390F88463C5EB051101EB41011B4A02EB0111E5
:4044000001F58A7106EBC60201EB8201891C085D3A46214606F016FCC5EB051101EB4101114A02EB011101F58A7106EBC60201EB8201091D085D3A46214606F041FCC5EBAE
:40444000051101EB4101084A02EB011101F58A7106EBC60218E000003C0200203E02002040020020982400208CB609088400001088040020840400208C000800F966DFBE3E
:4044800000000000F966DF3E01EB8201891D085D3A46214606F090FCC5EB051101EB4101FE4A02EB011101F58A7106EBC60201EB82010831085D3A46214606F03FFCC5EBE3
:4044C000051101EB4101F54A02EB011101F58A7106EBC60201EB82010A31085D3A46214606F0A8FCC5EB051101EB4101EB4A02EB011101F58A7106EBC60201EB82010C3182
:40450000085D3A46214606F0D3FCC5EB051101EB4101E24A02EB011101F58A7106EBC60201EB82010E31085D3A46214606F0FEFCC5EB051101EB4101D84A02EB011101F5AC
:404540008A7106EBC60201EB82011031085D3A46214606F034FDC5EB051101EB4101CF4A02EB011101F58A7106EBC60201EB8201085D3A46214606F0DDFAC5EB051101EB74
:404580004101C64A02EB011101F5E47106EB460201EB4201891C31F8141008B23A462146FEF72CF8C5EB051000EB4000BB4901EB001000F58A7006EBC60100EB8100143004
:4045C00000EB8400D0ED000AB0EE600A204606F02BF9C5EB051101EB4101B04A02EB011101F58A7106EBC60201EB820191ED070ABCEEC00A10EE101A88B206F043FFC5EBAA
:40460000051101EB4101A54A02EB011101F5E47106EB460231F8121008B2FDF7BDFF0220FEF75EF80220FEF72CF8BDE8F0812DE9F84304460F46FEF736F940B9FEF71CF93A
:4046400028B9FEF729F910B9FEF71EF998B19448006800909348002203210368924838F0B1FA924890F88403042803D10021012079F0E9FD99E08D4890F88E5390F8846377
:4046800090F8C80308B1012000E000208046B8F1000F0DD08649C85D0022394677F029F88349891CC85D0022394677F0BEF827E0C5EB051101EB4101784A02EB01113831DC
:4046C00006EB460202EBC60201EB82010931085D0022394677F00DF8C5EB051101EB41016E4A02EB0111383106EB460202EBC60201EB82010B31085D0022394677F095F80A
:40470000C5EB051101EB4101644A02EB0111383106EB460202EBC60201EB8201C91C085D00233A46214676F0F0F9C5EB051101EB41015A4A02EB0111383106EB460202EB49
:40474000C60201EB8201491D085D00233A46214676F080FAC5EB051101EB41014F4A02EB0111383106EB460202EBC60201EB8201C91D085D00233A46214676F010FBC5EB85
:40478000051101EB4101454A02EB0111383106EB460202EBC60201EB8201491C085D00233A46214676F010F900BFBDE8F883F8B50446FEF778F840B9FEF75EF828B9FEF7C9
:4047C0006BF810B9FEF760F850B13548006800903448002201210368334838F0F3F9C9E0324890F88E5390F8846390F8C80308B1012000E000200746002120469FED2D0A51
:4048000076F077FC002120469FED2B0A76F065FE87B32748203800EB8400D0ED000AB0EE600A0021204676F081FB2148103800EB8400D0ED000AB0EE600A0021204676F00A
:4048400058FC1B48183800EB8400D0ED000AB0EE600A0021204676F061FD1548083800EB8400D0ED000AB0EE600A0021204676F034FE7EE0FFE7C5EB051000EB400007492A
:4048800001EB0010383006EB460101EBC60100EB81000E3030F9140010E000008CB60908880400208404002072000800982400205C2800200000C8C20000C84200EE900A15
:4048C000F8EEE00AB0EE600A0021204676F02EFBC5EB051000EB4000FD4901EB0010383006EB460101EBC60100EB8100163030F9140000EE900AF8EEE00AB0EE600A0021D5
:40490000204676F0F6FBC5EB051000EB4000F04901EB0010383006EB460101EBC60100EB8100123030F9140000EE900AF8EEE00AB0EE600A0021204676F0F0FCC5EB051059
:4049400000EB4000E24901EB0010383006EB460101EBC60100EB81001A3030F9140000EE900AF8EEE00AB0EE600A0021204676F0B4FD00BFF8BD70B505460C462046FFF70F
:4049800016FF21462846FFF752FE21462846FFF722FD70BD70B500240BE0002505E029462046FFF718FD681CC5B2022DF7DB601CC4B2022CF1DB70BDF8B5FDF774FF40B970
:4049C000FDF75AFF28B9FDF767FF10B9FDF75CFF98B1C04800680090BF48002203210368BE4838F0EFF8BE4890F8840304284DD10021012079F027FC48E0B94890F88E6332
:404A000090F8847300241FE0002505E029462046FFF70DFE681CC5B2022DF7DBC6EB061101EB4101AA4A02EB0111383107EB470202EBC70201EB82012431085D0022214603
:404A400079F0DAFD601CC4B2022CDDDBC6EB061000EB40009E4901EB0010383007EB470101EBC70100EB8100D0ED080AB0EE600A002077F07FF876F02CFE0021084679F04A
:404A8000E2FB0021084679F0A1FC00BFF8BD38B5FDF709FF40B9FDF7EFFE28B9FDF7FCFE10B9FDF7F1FE50B18A48006800908A48002201210368894838F084F808E0002425
:404AC00004E02046FFF773FE601CC4B2022CF8DB38BD10B5FFF7DBFFFFF76EFFFFF75AFF10BD2DE9F0417E48B0F85A77B0F85C47B0F85E57B0F86067B0F86C8790F87803CE
:404B00000A2827D1A74206DB002C04DD611E88B200213DF060FFAE4204DA691C88B200213EF010F8BD4203DA002138463DF0CDFFA64203DD002120463EF004F8B04503DD68
:404B4000002130463EF086F9A84503DA002128463EF080F9BDE8F08110B5012038F0C9FA0146604880F83910002038F0C2FA5D494874012038F0BDFA04462146012025F00D
:404B8000EFF9002038F0B5FA04462146002025F0E7F910BD10B5FFF7A5FBFDF76DFE18B10021012038F05DF9FFF793FFFFF7D4FF012074F08FFE10BD10B50CF064FD0128C5
:404BC00003D14748B0F8BC4402E04548B0F88C43204610BD10B5FFF7EFFF00EE100AF8EE400A9FED411A80EE810A10BD10B53F48007801280AD1FFF7DFFF00EE100AF8EE79
:404C0000400A9FED3B1A80EE810A10BDFFF7D4FF00EE100AF8EE400A9FED331A80EE810AF3E710B50CF02FFD012803D12C48D0F8C04402E02A48D0F89043204610BD10B5C5
:404C40002DED028BFFF7EDFF00EE100AB8EEC00AB0EE408A2748B0F9000000EE100AB8EEC00A78EE000A9FED201A80EE810ABDEC028B10BD10B52DED028BFFF7D2FF00EEE8
:404C8000100AB8EEC00AB0EE408A1848007801280DD1FFF791FF00EE100AF8EE400AB0EE001A80EE810A38EE400AB0EE408A1148B0F9000000EE100AB8EEC00A78EE000AF2
:404CC0009FED091A80EE810ABDEC028B10BD00008CB6090888040020840400207200080098240020607C022000007A44400200200000FA443E020020FE48B0F89403FE4984
:404D0000B1F90010084400EE100AF8EEC00A1FED0A1A80EE810A704710B52DED028B0CF0B2FC012803D1F54890ED638A02E0F14890EDE68AB0EE480ABDEC028B10BD10B55B
:404D4000FFF7EAFF1FED181AC0EE010AB0EE600A10BD2DE9F04104460D460026E848B0F90000844204D1E748B0F90000854221D0E3480480E3480580FFF753FFE049B1F900
:404D80000010E04AB2F90020891A01EB8101490000FB01F7FFF710FF97FBF0F0D949098801EB810100EB410000B2D34908800020D54908803046BDE8F08177B581B00C4686
:404DC00015460026BDF8040041F65831884202DD084601900226012D03D00CF054FC01280FD100BF022201A9C848006800F5C27003F0C2F920B9BDF80410BE48A0F8BC14C9
:404E00000EE000BF022201A9C0480068543003F0B3F920B9BDF80410B648A0F88C1300BF0220F3F751FB202032F0D6FFACB1B8480068C078A04210D0AE4890F88403032850
:404E40000BD0B44800680090B148BDF8042003210368B14837F0B6FE17E0B4B9FDF723FD40B9FDF709FD28B9FDF716FD10B9FDF70BFD50B1A74800680090A548BDF8042068
:404E800003210368A44837F09DFEA448D0F854110220DFF88CC200DF00214FF480700EF00DF8304604B070BD73B50C4600250098B0F5FA4F04DD4FF4FA400090022506E0A8
:404EC000009810F5FA4F02DA964800900325012C03D00CF0D8FB01280ED100BF042269468A48006800F5C47003F046F918B981480099C0F8C0140DE000BF0422694683484F
:404F00000068583003F038F918B97A480099C0F8901300BF0620F3F7D7FA202032F05CFF7E48D0F854110220DFF8F4C100DF00214FF480700DF0C2FF28467CBD31B5002436
:404F4000BDF8000041F65831884202DD08460090022400BF022269466C4800685C3003F00BF920B9BDF800106248A0F8941300BF0720F3F7A9FA202032F02EFF204638BDFA
:404F800031B52DED020B044600259DED000ADFED660AB4EEE00AF1EE10FA05DD9FED620A8DED000A02250DE09DED000ADFED5F0AB4EEE00AF1EE10FA04D29FED5C0A8DED3E
:404FC000000A0325012C03D00CF05DFB01280FD100BF042269464D48006800F5C67003F0CBF820B99DED000A444880ED630A0EE000BF0422694645480068603003F0BCF82F
:4050000020B99DED000A3B4880EDE60A00BF0520F3F75AFA202032F0DFFE28463EBD31B5002400BF0422694638480068403003F0A3F818B92F480099C0F8781300BF0920C9
:40504000F3F742FA202032F0C7FE204638BD31B5002400BF022269462C480068563003F08BF820B99DF800102248A0F88E1300BF0820F3F729FA5D20F3F726FA202032F016
:40508000ABFE204638BD31B5002400BF042269461E480068443003F06FF818B915480099C0F87C1300BF0A20F3F70EFA202032F093FE204638BD33B581B00C4600259DF856
:4050C000040003284AD100BF012201A90F4800684C3003F051F820B99DF80410054880F8841300BF0B20F3F7EFF92D2032F074FE00491DE0982400203C020020D027002051
:4051000042020020440200203E02002084000010840400208804002004FA070030320020316D09080083FFFF0000FA460000FAC691F88E13C1EB011101EB4101FB4A02EB5E
:40514000011101F51D71FA4A92F8842302EB420201EB4201487905F0DBFCBFE0E4BBFDF7A2FB40B9FDF788FB28B9FDF795FB10B9FDF78AFB80B300BF012201A9ED480068F5
:405180004C3002F0F9FF20B99DF80410E84880F8841300BFE84800680090E8489DF8042003210368E64837F00DFDE14991F88E13C1EB011101EB4101DC4A02EB011101F5AF
:4051C0001D71DB4A92F8842302EB420201EB4201487905F09DFC81E0FFE7FCB1D7480068C078A0421AD0FDF75EFB58B9FDF744FB40B9FDF751FB28B9FDF746FB10B9FDF700
:405200003BFB58B1CC4800680090CC489DF8042003210368CA4837F0D5FC5FE0FDF743FB40B9FDF729FB28B9FDF736FB10B9FDF72BFB68B3C1480068C078A04228D100BFF4
:40524000012201A9BB4800684C3002F095FF20B99DF80410B64880F8841300BFB44991F88E13C1EB011101EB4101B04A02EB011101F51D71AE4A92F8842302EB420201EBD0
:405280004201487905F044FC0B20F3F71DF925E024BB00BF012201A9A64800684C3002F06BFF20B99DF80410A14880F8841300BF9F4991F88E13C1EB011101EB41019B4AD0
:4052C00002EB011101F51D71994A92F8842302EB420201EB4201487905F01AFC28463EBD31B5002400BF012269469248006800F23E4002F041FF20B99DF800108C4880F839
:40530000761700BF204638BD31B5002400BF012269468848006800F23F4002F02DFF20B99DF80010824880F8771700BF204638BD01460020704710B5044628228149204655
:405340007BF04CFF10BD70B50446C4EB041000EB4000764901EB001090F83550FF2D00D10025C4EB041101EB4101704A02EB0110FFF7DEFFC4EB041101EB41016B4A02EB52
:405380000111887FFFF74BFEC4EB041101EB4101664A02EB0111088D00221146FFF70DFDC5EB051101EB4101604A02EB0111088D01220021FFF701FDC4EB041101EB41018A
:4053C0005A4A02EB0111C86A0021FFF76DFDC5EB051101EB4101554A02EB0111C86A0121FFF762FDC4EB041101EB41014F4A02EB0111088EFFF7A2FDC4EB041000EB400079
:405400004A4901EB0010B0F9320000EE900AF8EEE00AB0EE600A0020FFF7B2FDC5EB051000EB4000414901EB0010B0F9320000EE900AF8EEE00AB0EE600A0120FFF7A0FD78
:40544000C4EB041101EB4101384A02EB011191F82000FFF7FCFDC4EB041101EB4101334A02EB0111C87FFFF70EFE44F0DDFC80B1002108460FF094F8C4EB041101EB410140
:405480002A4A02EB011191F8360001210FF088F81AE044F0F2FCB8B1C4EB041101EB4101224A02EB011191F8340000210FF078F8C4EB041101EB41011C4A02EB011191F80A
:4054C000360001210FF06CF8FEF7D0FD002010F0BBF870BD01B500BF012269461548006800F5886002F048FE20B99DF80010104880F8781700BF08BD31B582B000BF0122B3
:4055000002A9114802F038FE20B99DF80800084981F8010100BF064890F8010120B1012818D0022818D000BF08A417E08CB6090898240020840000108804002084040020F9
:4055400056010800E82700200101006874726163746F7200FCA401E0FEA400BF00BF20467BF0C6FD401CC5B20123232200210846CDE9004569F031FB3EBDF84890F8781386
:40558000082905D0092903D00A2901D00E2901D1012070470020FCE7F04890F87813082903D0092901D00E2901D1012070470020FCE7EA4890F878130A2901D101207047A0
:4055C0000020FCE7E54890F87813082901D1012070470020FCE7E14890F87813092901D1012070470020FCE7DC4890F878130E2901D1012070470020FCE70020D74991F88B
:405600008E13432909D0D54991F88E13452904D0D24991F88E13472900D1012070470020CE4991F88E13422909D0CC4991F88E13442904D0C94991F88E13462900D10120DA
:4056400070470020C54991F88E13412900D10120704770B504460025C1480078844211D0012C01DD02250DE0BD480470BD48D0F854110220DFF8F0C200DF00214FF48070A4
:405680000DF01CFC284670BD33B581B00D4600249DF80400012802DD012001900224AF4890F8E0049DF8041088420FD000BF012201A9AE48006800F5D47002F05DFD20B934
:4056C0009DF80410A54880F8E01400BF8920F2F7FBFEA448D0F854110220DFF88CC200DF05F0AAFC9F48D0F808120120DFF878C200DF76F02FFB9B48016D0220DFF868C2A6
:4057000000DFFCF74BFB9A480068009099489DF8042003210368984837F054FA2820F2F7D3FE20463EBD8D4890F88E03C0EB001000EB4000914901EB0010408C704787489A
:4057400090F88E03C0EB001000EB40008B4901EB0010808C704770B50124894889490978455C88480078652827DA864800785C2823DAC5EB051101EB4101804B03EB01122B
:40578000C5EB051101EB410103EB0111888C1E212FF0AFFF044024B17A480078401C7949087001207849087040F2B91045F0F0F840F20B3045F0ECF805E0012071490870BC
:4057C000002071490870204670BD70B501246F4800781E2833DA6D4800781D282FDA6B49097801EB01116A4A02EB4101081D7BF07FFC85B26549097801EB0111644B03EB5B
:4058000041010A1D6149097801EB011103EB4101488829462FF06DFF044024B15B480078401C5A49087001205749087040F2B91045F0AEF84FF4437045F0AAF805E001204F
:4058400052490870002050490870204670BD51480078704770B501254F48007812286FD14E48007800286CD148F642604C490880012005E04FF6FF71494A22F81010401C61
:405880001D28F7DB002403E1C4EB041000EB40003A4901EB001090F87402032852D0C4EB041000EB400001EB001090F87402022848D0C4EB041000EB400001EB001090F875
:4058C0007A0203283ED0C4EB041000EB400001EB001090F87A02022834D0C4EB041000EB400001EB001090F8800203282AD0C4EB041000EB400001EB001090F880020228A0
:4059000020D0C4EB041000EB400001EB001090F88602032816D0C4EB041000EB400001EB001090F88602022878D0C4EB041000EB400001EB001090F88C0203286ED031E086
:40594000E6E0ADE06AE00000696D706C656D656E7400000066656E6474000000982400204002002030320020316D0908840000108804002084040020580108008CB60908A3
:40598000F4B1090838020020720300103902002050B209083A0200204D03001046020020000D0010C4EB041000EB400001EB001090F88C02022831D00AF09EFB002866D087
:4059C000C4EB041000EB4000F74901EB001090F8740218BBC4EB041000EB400001EB001090F87A02D0B9C4EB041000EB400001EB001090F8800288B9C4EB041000EB400012
:405A000001EB001090F8860240B9C4EB041000EB400001EB001090F88C0298B3E34890F87803C4EB041101EB4101DF4A02EB0111897F88422BD1012126E0C4EB041000EB2A
:405A40004000D94A02EB0010C07F01EB0112D84B13F81220904216D1FFF7F9FE40B1FFF7F6FE01EB0112D24B13F8122090420AD101EB0110CE4A02EB40004088CD4A22F866
:405A8000110003E003E0491C1D29D6DB00BF641C6F2CFFF6F9AE0120C7490870C7490870C54800781E282DDCC248C349097830F811004FF6FF71884210D0BF4800781D2845
:405AC0000CDABC48BC49097830F81120BA48017842F218702FF009FD054008E04FF6FF72B548017842F218702FF0FFFC054025B1B1480078401CB049087040F20A3044F059
:405B000047FF05E00120AC4908700020AB490870284670BD70B5AA48AA490978445C0125A948007812287DD1A648007865287ADCA44800785C2877DA9C4890F87C03C4EB27
:405B4000041101EB4101984A02EB0111C97F88426AD1964890F87803C4EB041101EB410102EB0111897F88425ED10AF0C5FA88B3C4EB041000EB40008B4901EB001090F8A7
:405B80007402002851D1C4EB041000EB400001EB001090F87A02002847D1C4EB041000EB400001EB001090F8800200287CD1C4EB041000EB400001EB001090F8860200286C
:405BC00072D1C4EB041000EB400001EB001090F88C0250BBC4EB041000EB4000724901EB001090F8740203285ED0C4EB041000EB400001EB001090F87402022854D0C4EB76
:405C0000041000EB400001EB001090F87A0203284AD0C4EB041000EB400001EB001090F87A0203E075E06AE04EE03DE002283BD0C4EB041000EB400001EB001090F88002FC
:405C4000032831D0C4EB041000EB400001EB001090F88002022827D0C4EB041000EB400001EB001090F8860203281DD0C4EB041000EB400001EB001090F88602022813D0CA
:405C8000C4EB041000EB400001EB001090F88C02032809D0C4EB041000EB400001EB001090F88C0202280FD1C4EB041000EB40003D4901EB0010428C4248017842F21970D8
:405CC0002FF013FC054008E04FF6FF723D48017842F219702FF009FC054025B139480078401C3849087001203849087040F2B91044F04EFE40F2093044F04AFE09E00120C5
:405D00003049087000203149087040F2B91044F03FFE284670BD0146C1EB011000EB4000214A02EB001090F8BC0070470120704700207047264800687047254908607047FE
:405D400000201A4991F87C13102900D1012070470020164991F88E13142901D1012100E00021124A92F88E23152A01D1012200E0002211430D4A92F88E23162A01D10122E3
:405D800000E000221143094A92F88E23172A01D1012200E000221143044A92F88E23182A18D1012217E000008CB609089824002050B20908000D0010390200204602002083
:405DC000F4B10908380200204D030010720300103402002000221143FE4A92F88E23192A01D1012200E00022114301B1012070470020F84991F87813042905D1F54991F808
:405E00007C13022900D1012070470020F14991F87813042905D1EF4991F87C130C2900D1012070470020EB4991F87C13112900D1012070470020E74991F88E13652913D026
:405E4000E44991F88E1366290ED0E24991F88E13672909D0DF4991F88E13682904D0DD4991F88E13692900D1012070470020D94991F87C13152900D1012070470020D549DF
:405E800091F87C130F2900D1012070470020D14991F87C13122900D1012070470020CD4991F87C13132900D1012070470020C94991F87C13162900D101207047014601EB1B
:405EC0000110C54A12F8100070470246012109E001EB0110C04B13F81000904201D1C8B27047491C1D29F3DB0020F9E72DE9F0410124B84991F87C03FFF7E7FF00EB0010A1
:405F0000B54901EB4000051DB24991F87C03FFF7DCFF00EB0010B04901EB4000071D38467BF0E6F886B22A46314649F2FC102FF0E0FB04462046BDE8F08170B5A54890F876
:405F40008E4390F884530A20DFF890C200DFC4EB041101EB4101A24A02EB011101F2922101EBC5014878002172F056F90A20DFF86CC200DF00209FED9B0A71F02CFE0A20E4
:405F8000DFF858C200DFC4EB041101EB4101944A02EB0111383105EB450202EBC50211F822000021FEF70CF90A20DFF830C200DFC4EB041000EB4000894901EB00103830B2
:405FC00005EB450101EBC50100EB8100B0F90E0000EE900AF8EEE00AB0EE600A0021084674F0A4FF0A20DFF8F4C100DFC4EB041000EB40007A4901EB0010383005EB4501E0
:4060000001EBC50100EB8100B0F9160000EE900AF8EEE00AB0EE600A0021084675F069F80A20DFF8B8C100DFC4EB041000EB40006B4901EB0010383005EB450101EBC501A7
:4060400000EB8100B0F9120000EE900AF8EEE00AB0EE600A0021084675F060F90A20DFF87CC100DFC4EB041000EB40005C4901EB0010383005EB450101EBC50100EB810004
:40608000B0F91A0000EE900AF8EEE00AB0EE600A0021084675F021FA0A20DFF840C100DFC4EB041101EB41014D4A02EB0111383105EB450202EBC50201EB8201C87800233F
:4060C0001A46194674F021FD0A20DFF810C100DFC4EB041101EB4101414A02EB0111383105EB450202EBC50201EB8201487900231A46194674F0AEFD0A20DFF8E0C000DF3D
:40610000C4EB041101EB4101354A02EB0111383105EB450202EBC50201EB8201C87900231A46194674F03BFE0A20DFF8B0C000DF75F0CFFA0A20DFF8A4C000DFC4EB0411E6
:4061400001EB4101264A02EB0111383105EB450202EBC50201EB8201487A0022114675F0C8FA0A20DFF874C000DFC4EB041101EB41011B4A02EB0111383105EB450202EB66
:40618000C50201EB8201C87A0022114675F04DFB0A20DFF848C000DFC4EB041101EB41010F4A02EB0111383105EB450202EBC50201EB8201487800231A46194674F004FC46
:4061C0000A20DFF818C000DFC4EB041000EB4000034909E09824002050B20908D16C09088CB609080000000001EB0010383005EB450101EBC50100EB8100D0ED080AB0EE0F
:40620000600A002075F0B6FC0A20DFF8F0C300DF00209FEDFB0A76F080FF0A20DFF8DCC300DF00209FEDF70A76F014FC0A20DFF8CCC300DFC4EB041101EB4101F24A02EB68
:406240000111088DFF220021FEF7B7FD0A20DFF8ACC300DF70BD10B50124EC48007810282ADAEA48007800EB4000E94901EB4000007970B1E548007800EB400001EB400075
:406280004288E248017842F210702FF02EF9044008E04FF6FF72DD48017842F210702FF024F90440D9480078401CD849087040F20F3044F06DFB02E00020D449087020462B
:4062C00010BD10B5002413E004EB4400D14A02EB8000411CD0487BF075F838B904EB4400CC4911F82000CD49087003E0601CC4B2082CE9DB00BF10BD33B581B00D46002414
:406300009DF80400012802DD012001900224C44890F8E1049DF8041088420FD000BF012201A9C048006800F2A91001F025FF20B99DF80410BA4880F8E11400BFAE20F2F7F6
:40634000C3F8B948D0F854110220DFF8E0C200DF04F072FEB448D0F808120120DFF8CCC200DF75F0F7FCB048016D0220DFF8BCC200DFFBF713FDAE4800680090AD489DF885
:40638000042003210368AC4836F01CFC20463EBDF8B5FCF788FA40B9FCF76EFA28B9FCF77BFA10B9FCF770FA58B1A14800680090A04803221146036840F2762036F002FC0D
:4063C000ACE0974890F88E4390F884530026A1E0C4EB041000EB40008B4901EB0010383005EB450101EBC50100EB81000E308C4991F8E01430F9110000EE900AF8EEE00A37
:40640000B0EE600A30466DF0CEF8C4EB041000EB40007D4901EB0010383005EB450101EBC50100EB810012307D4991F8E01430F9110000EE900AF8EEE00AB0EE600A3046BA
:406440006DF0C9F8C4EB041000EB40006E4901EB0010383005EB450101EBC50100EB810016306F4991F8E01430F9110000EE900AF8EEE00AB0EE600A30466DF015FFC4EBF6
:40648000041000EB4000604901EB0010383005EB450101EBC50100EB81001A30604991F8E01430F9110000EE900AF8EEE00AB0EE600A30466DF0DFFEC4EB041101EB410190
:4064C000514A02EB0111383105EB450202EBC50201EB82010931524A92F8E024885C31466DF0B6FEC4EB041101EB4101464A02EB0111383105EB450202EBC50201EB82012B
:406500000B31474A92F8E024885C31466DF08EFE701CC6B2022EFFF65BAF00BFF8BD10B52DED020B002400BF042269463D48006800F24C4001F020FE20B99DED000A3F4803
:4065400080ED130A00BFB120F1F7BEFF20461CBD10B50024FFF711F808B1012405E0FFF770F808B1022400E000242046FEF7B2FF10BD33B581B00C460025294890F8840348
:40658000032816D100BF022201A92648006800F24A4001F0F1FD20B9019881B22048A0F8821700BFC620F1F78FFF2D2031F014FC95E014BBFCF777F940B9FCF75DF928B96A
:4065C000FCF76AF910B9FCF75FF9B0B10198322802DD3220019004E00198002801DA0020019013480068009012480368032112488D38019A36F0E6FA71E021E0D16C09084E
:40660000B81E05BFB81E053F8CB60908470200202AB6090894B10908D86F00083A020020982400208400001030320020316D09088804002084040020EF010800D02B0020F0
:406640004CB340480068C078A04224D0FCF72BF958B9FCF711F940B9FCF71EF928B9FCF713F910B9FCF708F9A8B10198322802DD3220019004E00198002801DA0020019019
:406680003148006800902F48036803212F48019A36F098FA23E0FCF706F940B9FCF7ECF828B9FCF7F9F810B9FCF7EEF8B8B125480068C078A04212D100BF022201A9244839
:4066C000006800F24A4001F057FD20B9019881B22048A0F8821700BFC620F1F7F5FE28463EBD00201B4991F88E13622904D0194991F88E13632900D101207047154890F897
:40670000BE0420B1134890F8BE04012801D1012070470020FCE70F4890F8BE04022804D00C4890F8BE04032801D1012070470020FCE7084890F8BE04042801D101207047C6
:406740000020FCE784040020880400206201080084000010982400201FB5012108466BF036FA012104206BF032FA012108206BF02EFA012110206BF02AFA0020009001906C
:40678000029003460122FE490390104643F0B0FC002000900190029003460222F9490390104643F0A5FC002000900190029003460246F5490390052043F09AFC0020022226
:4067C0000123CDE90120009303900346EF49062043F08EFC002002220123CDE90120009303900346EA49072043F082FC002002220123CDE90120009303900346E549082057
:4068000043F076FC002000900190029001230222E1490390092043F06BFC00200323CDE90030029003460222DC4903900A2043F05FFC00200121CDE9000103460A46CDE935
:406840000210D7490B2043F053FC002000900190029003460322D3490390112043F048FC002000900190029003460322CE490390122043F03DFC00200323CDE9003002905A
:4068800003460222C9490390182043F031FC002000900190029003460122C5490390192043F026FC002000900190029003460122C04903901A2043F01BFC00200222CDE967
:4068C000000202900346BC4903901B2043F010FC00200222CDE9000202900346B74903901F2043F005FC00200222CDE9000202900346B3490390202043F0FAFB00200121BC
:406900000090CDE9010103460A46AE490390212043F0EEFB002001210090CDE9010103460A46A9490390242043F0E2FB002000900190029003460246A4490390252043F037
:40694000D7FB002000900190029003460246A0490390262043F0CCFB002001210090CDE9010103460A469B490390292043F0C0FB00200090019002900123022296490390C7
:406980002A2043F0B5FB00200121CDE9000103460A46CDE9021091492D2043F0A9FB0020009001900290034602228D490390312043F09EFB0020009001900290034602224C
:4069C00088490390322043F093FB00200121CDE9000103460A46CDE902108349332043F087FB00200121CDE9000103460A46CDE902107E49342043F07BFB00200121CDE9DC
:406A0000000103460A46CDE902107949352043F06FFB00200121CDE9000103460A46CDE902107449362043F063FB00200121CDE9000103460A46CDE902106F49372043F0A6
:406A400057FB00200121CDE9000103460A46CDE902106A49382043F04BFB002001210090CDE9010103460A4665490390392043F03FFB002001210090CDE9010103460A4699
:406A8000604903903B2043F033FB002001210090CDE9010103460A465B4903903C2043F027FB00200121CDE9000103460A46CDE9021056493D2043F01BFB00200121CDE93C
:406AC000000103460A46CDE9021051493E2043F00FFB002001210090CDE90101034602224C490390402043F003FB00200090019002900346022248490390412043F0F8FA65
:406B000000200090019002900346022243490390422043F0EDFA0020009001900290034602463F490390432043F0E2FA0020009001900290034601223A490390462043F09B
:406B4000D7FA00200222CDE900020290034636490390472043F0CCFA00200090019002900346022231490390482043F0C1FA0020009001900290034602222D49039059E0D6
:406B8000FA05002025060020FB05002012060020130600201406002015060020FC0500202D0600200206002042060020FD0500201A0600201B0600201C0600201D06002039
:406BC0001E060020200600200E060020FE05002036060020260600202306002027060020180600201906002028060020290600202A0600202B060020070600200806002060
:406C0000090600200A0600200B0600200C0600200D06002040060020300600203106002041060020350600200F060020FF05002000060020492043F05BFA00200121009048
:406C4000CDE9010103460A46FE4903904A2043F04FFA00200222CDE9000202900346FA4903904D2043F044FA00200222CDE9000202900346F54903904E2043F039FA0020DC
:406C800000900190029003460322F1490390512043F02EFA002000900190029003460322EC490390522043F023FA002000900190029003460322E8490390532043F018FA92
:406CC0000021E648007843F036F90021E448007843F031F90021E348007843F02CF90121E148007843F027F90021E048007843F022F90021DE48007843F01DF90021DD48BA
:406D0000007843F018F90121DB48007843F013F90121DA48007843F00EF90121D848007843F009F90021D748007843F004F90021D548007843F0FFF80021D448007843F006
:406D4000FAF81FBD1FB5012108466AF040FF012104206AF03CFF012108206AF038FF012110206AF034FF002000900190029003460322C7490390012043F0BAF90020009038
:406D80000190029003460322C2490390022043F0AFF9002000900190029003460322BE490390104643F0A4F9002000900190029003460322B9490390042043F099F90020C7
:406DC0000222CDE90002029003460322B4490390052043F08DF9002002220123CDE90120009303900346AF49062043F081F9002002220123CDE90120009303900346AA492F
:406E0000072043F075F9002002220123CDE90120009303900346A549082043F069F9002000900190029001230222A1490390092043F05EF900200090019002900346024682
:406E40009C4903900A2043F053F900200121CDE9000103460A46CDE902108A490B2043F047F9002001210090CDE9010103460A46814903900C2043F03BF900200121CDE91B
:406E8000000103460A46CDE902107B490C2043F02FF900200090019002900346012272490390192043F024F90020009001900290034601226B4903901A2043F019F90020EA
:406EC00002220092CDE9012003467B4903901B2043F00EF9002000900190029003460246764903901C2043F003F9002002220092CDE901200346724903901F2043F0F8F829
:406F0000002002220092CDE9012003466D490390202043F0EDF800200090019002900346032269490390212043F0E2F800200090019002900346032264490390242043F0EE
:406F4000D7F8002001210090CDE9010103460A465F490390252043F0CBF8002001210090CDE9010103460A465A490390262043F0BFF8002000900190029003460122564942
:406F80000390272043F0B4F800200090019002900346012251490390292043F0A9F80020009001900290012302224D4903902A2043F09EF8002000900190029003460222F8
:406FC000484903902B2043F093F8002000900190029003460222444903902C2043F088F80020009001900290034601223F490390312043F07DF8002001210090CDE9010128
:4070000003460A463A490390322043F071F800200121CDE9000103460A46CDE902101749332043F065F800200121CDE9000103460A46CDE902101449342043F059F8002067
:40704000012157E00E06002010060020110600203D0600203E0600203F060020FA0500202D0600201A0600201B060020350600203B0600203C06002026060020280600203F
:407080002A06002027060020290600202B0600200106002002060020030600200406002038060020120600201306002014060020150600202F0600201C0600203A060020B6
:4070C0001D0600201E0600201F06002005060020200600202106002022060020060600202306002031060020300600201806002019060020CDE9000103460A46CDE902100D
:40710000FE49352042F0F4FF00200121CDE9000103460A46CDE90210F949362042F0E8FF00200121CDE9000103460A46CDE90210F449372042F0DCFF00200121CDE900018F
:4071400003460A46CDE90210EF49382042F0D0FF002001210090CDE9010103460A46EB490390392042F0C4FF002000900190029003460122E64903903A2042F0B9FF002080
:4071800001210090CDE9010103460A46E14903903B2042F0ADFF002001210090CDE9010103460A46DC4903903C2042F0A1FF00200121CDE9000103460A46CDE90210D74953
:4071C0003D2042F095FF00200121CDE9000103460A46CDE90210D2493E2042F089FF002000900190029003460122CE4903903F2042F07EFF01200021009101910B460246EA
:40720000CDE90210C849402042F072FF002000900190029003460222C4490390412042F067FF002000900190029003460222C0490390422042F05CFF0020009001900290FB
:4072400003460122BB490390432042F051FF002000900190029003460122B7490390442042F046FF002000900190029003460122B2490390452042F03BFF0020009001909A
:40728000029003460122AE490390462042F030FF002002220092CDE901200346A9490390472042F025FF002001210090CDE9010103460A46A4490390482042F019FF0020D2
:4072C0000222CDE900020290034602469F4903904A2042F00DFF00200222CDE900020290034602469A4903904B2042F001FF002000900190029003460246964903904C20F8
:4073000042F0F6FE002002220092CDE901200346914903904D2042F0EBFE002002220092CDE9012003468D4903904E2042F0E0FE01200021009101910B460246CDE9021099
:4073400087494F2042F0D4FE01200021009101910B460246CDE902108249502042F0C8FE0020009001900290034603227E490390512042F0BDFE00200090019002900346BC
:4073800003227A490390522042F0B2FE00200090019002900346032275490390532042F0A7FE00215F48007842F0C5FD00215E48007842F0C0FD00216E48007842F0BBFD87
:4073C00001216D48007842F0B6FD00215C48007842F0B1FD00216248007842F0ACFD00216048007842F0A7FD01216448007842F0A2FD01216248007842F09DFD0121614815
:40740000007842F098FD01215F48007842F093FD01213A48007842F08EFD00215B48007842F089FD00215A48007842F084FD00213348007842F07FFD1FBD1FB5002000902D
:40744000019002900346024652490390012042F04FFE0020009001900290034602464D490390022042F044FE00200090019002900346024647490390032042F039FE002034
:407480000090019002900346024642490390042042F02EFE0020009001900290034602463C490390052042F023FE00200090019002900346024637490390062042F018FE0F
:4074C00000200090019002900346024631490390072042F00DFE0020009001900290034602462C490390082042F002FE00200090019002900346024626494DE02A060020A1
:407500002B0600200706002008060020090600202C0600200A0600200B0600200C0600200D0600202E0600202D060020250600202406002032060020330600203406002011
:40754000350600200F0600200E06002036060020370600203906002010060020110600203B0600203C0600203D0600203E0600203F0600201A0600201B060020210600200B
:407580002206002026060020280600202706002029060020F90500200390092042F0A8FD002000900190029003460246FE4903900A2042F09DFD002000900190029003464C
:4075C0000246F94903900B2042F092FD002000900190029003460246F34903900C2042F087FD002000900190029003460246EE4903900D2042F07CFD002000900190029094
:4076000003460246E8490390112042F071FD002000900190029003460246E3490390122042F066FD002000900190029003460246DD490390172042F05BFD0020009001901B
:40764000029003460246D8490390182042F050FD002000900190029003460246D2490390192042F045FD002000900190029003460246CD4903901B2042F03AFD002000905C
:407680000190029003460246C74903901C2042F02FFD002000900190029003460246C24903901F2042F024FD002000900190029003460246BC490390202042F019FD0020A1
:4076C00000900190029003460246B7490390212042F00EFD002000900190029003460246B1490390222042F003FD002000900190029003460246AC490390232042F0F8FC7B
:40770000002000900190029003460246A6490390242042F0EDFC002000900190029003460246A1490390252042F0E2FC0020009001900290034602469B490390262042F07B
:40774000D7FC00200090019002900346024696490390272042F0CCFC00200090019002900346024690490390282042F0C1FC0020009001900290034602468B490390292004
:4077800042F0B6FC002000900190029003460246854903902A2042F0ABFC002000900190029003460246804903902B2042F0A0FC0020009001900290034602467A4903906A
:4077C0002C2042F095FC002000900190029003460246754903902D2042F08AFC0020009001900290034602466F4903902E2042F07FFC0020009001900290034602466A49FF
:4078000003902F2042F074FC00200090019002900346024664490390302042F069FC0020009001900290034602465F490390312042F05EFC00200090019002900346024659
:4078400059490390322042F053FC00200090019002900346024654490390332042F048FC0020009001900290034602464E490390342042F03DFC002000900190029003463A
:40788000024649490390352042F032FC00200090019002900346024643490390362042F027FC0020009001900290034602463E490390372042F01CFC002000900190029086
:4078C0000346024638490390382042F011FC00200090019002900346024633490390392042F006FC0020009001900290034602462D4903903A2042F0FBFB0020009001901C
:40790000029003460246284903903B2042F0F0FB002000900190029003460246224903903C2042F0E5FB0020009001900290034602461D4903903D2042F0DAFB0020009067
:407940000190029003460246174903903E2042F0CFFB002000900190029003460246124903903F2042F0C4FB0020009001900290034602460C490390402042F0B9FB0020B2
:407980000090019002900346024607490390412042F0AEFB00200090019002900346024601490390422001E0F905002042F0A0FB002000900190029003460246FE490390B7
:4079C000432042F095FB002000900190029003460246F9490390442042F08AFB002000900190029003460246F3490390452042F07FFB002000900190029003460246EE492F
:407A00000390462042F074FB002000900190029003460246E8490390472042F069FB002000900190029003460246E3490390482042F05EFB0020009001900290034602460D
:407A4000DD490390492042F053FB002000900190029003460246D84903904A2042F048FB002000900190029003460246D24903904B2042F03DFB002000900190029003466A
:407A80000246CD4903904C2042F032FB002000900190029003460246C74903904D2042F027FB002000900190029003460246C24903904E2042F01CFB0020009001900290B6
:407AC00003460246BC4903904F2042F011FB002000900190029003460246B7490390502042F006FB002000900190029003460322B2490390512042F0FBFA0020009001906E
:407B0000029003460322AE490390522042F0F0FA002000900190029003460322A9490390532042F0E5FA1FBD1FB50024FFF785FC0CE00020A44901EB041189680870A2494A
:407B400001EB0411C9680870601CC4B2542CF0DB42F0ADF842F09EF9012102206AF037F800200090019002900346012297490390162042F0BDFA002001210090CDE9010156
:407B800003460A46924903901E2042F0B1FA002001210090CDE9010103460A468D4903901A2042F0A5FA42F0C4FDFF281CD042F038F90C2816D2DFE800F015060A070B0E8B
:407BC0000C0D0F10111200BFFFF7BCF80BE000BF00BF00BF00BF00BF00BF00BF00BFFEF7BBFD00E000BF00BF1FBD10B500207A49087041F031FEFA2041F097FEFFF794FF0E
:407C0000F0F774FB002211467448DFF8D4C100DF002010BD38B50446002560680090009D206880F3088800BFA84738BD10B501206949087041F04CFE67494860012069F0A5
:407C400077FE1CE0612069F015FE78B145F25550644908600120486040F6B83088604CF6CC40086002205C49087008E05A49486841F069FE642802D90320574908705648B5
:407C800000780128DED010BD10B572B66FF0040000F039FA6FF0010000F035FA4FF0FF3000F031FA042000F02EFA052000F02BFA062000F028FA072000F025FA082000F031
:407CC00022FA092000F01FFA0A2000F01CFA0B2000F019FA0C2000F016FA0D2000F013FA0E2000F010FA0F2000F00DFA102000F00AFA112000F007FA122000F004FA13209B
:407D000000F001FA142000F0FEF9152000F0FBF9162000F0F8F9172000F0F5F9182000F0F2F9192000F0EFF91A2000F0ECF91B2000F0E9F91C2000F0E6F91D2000F0E3F9A4
:407D40001E2000F0E0F91F2000F0DDF9202000F0DAF9212000F0D7F9222000F0D4F9232000F0D1F9242000F0CEF9252000F0CBF9262000F0C8F9272000F0C5F9282000F0DF
:407D8000C2F9292000F0BFF92A2000F0BCF92B2000F0B9F92C2000F0B6F92D2000F0B3F92E2000F0B0F92F2000F0ADF9302000F0AAF9312018E00000F90500203D060020EE
:407DC0003E0600203F06002094060B0816060020170600201A060020480200205F1102087D7509080030004000F08DF9322000F08AF9332000F087F9342000F084F93520E9
:407E000000F081F9362000F07EF9372000F07BF9382000F078F9392000F075F93A2000F072F93B2000F06FF93C2000F06CF93D2000F069F93E2000F066F93F2000F063F9D0
:407E4000402000F060F9412000F05DF9422000F05AF9432000F057F9442000F054F9452000F051F9462000F04EF9472000F04BF9482000F048F9492000F045F94A2000F068
:407E800042F94B2000F03FF94C2000F03CF94D2000F039F94E2000F036F94F2000F033F9502000F030F9512000F02DF96FF0040000F032F96FF0010000F02EF94FF0FF3049
:407EC00000F02AF9042000F027F9052000F024F9062000F021F9072000F01EF9082000F01BF9092000F018F90A2000F015F90B2000F012F90C2000F00FF90D2000F00CF9C1
:407F00000E2000F009F90F2000F006F9102000F003F9112000F000F9122000F0FDF8132000F0FAF8142000F0F7F8152000F0F4F8162000F0F1F8172000F0EEF8182000F039
:407F4000EBF8192000F0E8F81A2000F0E5F81B2000F0E2F81C2000F0DFF81D2000F0DCF81E2000F0D9F81F2000F0D6F8202000F0D3F8212000F0D0F8222000F0CDF82320DB
:407F800000F0CAF8242000F0C7F8252000F0C4F8262000F0C1F8272000F0BEF8282000F0BBF8292000F0B8F82A2000F0B5F82B2000F0B2F82C2000F0AFF82D2000F0ACF8EB
:407FC0002E2000F0A9F82F2000F0A6F8302000F0A3F8312000F0A0F8322000F09DF8332000F09AF8342000F097F8352000F094F8362000F091F8372000F08EF8382000F0DD
:408000008BF8392000F088F83A2000F085F83B2000F082F83C2000F07FF83D2000F07CF83E2000F079F83F2000F076F8402000F073F8412000F070F8422000F06DF84320DA
:4080400000F06AF8442000F067F8452000F064F8462000F061F8472000F05EF8482000F05BF8492000F058F84A2000F055F84B2000F052F84C2000F04FF84D2000F04CF80A
:408080004E2000F049F84F2000F046F8502000F043F8512000F040F862B610BD00BFBFF34F8F2248006800F4E06021490843001D1E490860BFF34F8F00BF00BFFEE74AF642
:4080C000AA201C49086070472DE9FC4106460C4617469846089D0020009001902078B0280DD16078102802D0112805D103E0142004F06FFC01E000E000BF00BF00E000BF8D
:4081000000BFBDE8FC8100F01F02012191400A4A430942F82310704700F01F0201219140064A430942F82310704700000CED00E00000FA050030004080E100E080E200E007
:40814000FE480078704710B541F06EFE40B1FC4890F83503012803D001200AF012FF0AE042F0F3FB38B1F64890F83503022802D002200AF006FF10BD2DE9F04104460E464B
:4081800017460025B4F1D04F0FD3E019401EED4988420AD8A4F1D0483A464146304610F01DFE00B102E0102500E0082525B1E64800882843E44908802846BDE8F0812DE9FE
:4081C000FE4F06468946174698460020009083464FF4807200233846414678F077FB05464FF4807200233846414678F06FFB924615B9BAF1000F2AD0ADB1002411E006EBF4
:408200000420029009EB042001904FF48072DDE90110FFF7B1FF009000984BEA000B601CC4B2AC42EBD3BAF1000F12D006EB0520029009EB052001901FFA8AF2DDE90110CD
:40824000FFF79AFF009000984BEA000B01E04FF0400B5846BDE8FE8F10B5044600BF10222146BA48FFF788FF20B910222146B84878F0B4FF00BF10BD70B504460D46B5490D
:40828000611A75F1000009D20C2016F0AFF8032016F0C4F840F2E27016F0D0F870BD70B504460D46AB491439611A75F1000001D20FF054FD70BD2DE9F84305460E46A549B3
:4082C0003239691A76F100002BD203F0CAFB8046012423E0062C0CD2DFE804F00B0C090705039D4F08E09D4F06E09D4F04E09D4F02E000BF9C4F00BF00BF0020009001224D
:40830000694607F5C370FFF737FF444504D19DF800108B4880F8BE14601CC4B2052CD9DD00BFBDE8F8832DE9F04180460C4615460026B4F1D04F0FD36019401E814988426A
:408340000AD8A4F1D0472A463946404610F0DBFD00B102E0102600E0082606B103DF3046BDE8F0812DE9FF5F86B007468846DDF850B0DDE90801381A78EB01007ED203F0C4
:4083800070FB814601257DE3062D0CD2DFE805F00B0C09070503704E08E0704E06E0704E04E0704E02E000BF6F4E00BF00BF012206F1560105A8FFF7B6FF9DF814006F287A
:4083C00001DB00200590012206F14C0104A8FFF7AAFF9DF81000052801DB002004909DF8140058457DD19DF8100003287AD10024F4E04FF0000AC8E09DF81400C0EB0010DC
:4084000000EB4000594901EB001038309DF8101001EB410202EBC10100EB8100C01C005D029006F1940101EB440101EB0A00012202A9FFF7A1FE4D4506D19DF808104C4881
:4084400000EB440000F80A109DF81400C0EB001000EB4000454901EB001038309DF8101001EB410202EBC10100EB8100401D005D029006F1980101EB440100E006E301EB79
:408480000A00012202A9FFF777FE4D4507D19DF808103748001D00EB440000F80A109DF81400C0EB001000EB4000304901EB001038309DF8101001EB410202EBC10100EB9B
:4084C0008100C01D005D029006F19C0101EB440101EB0A00012202A9FFF74EFE4D450AD101E0CDE2BEE09DF808102148083000EB440000F80A109DF81400C0EB001000EBEB
:4085000040001A4901EB001038309DF8101001EB410202EBC10100EB8100401C005D029006F1A00101EB440101EB0A00012202A9FFF722FE4D4524D11CE000008000001034
:4085400098240020FF1F00688A00001018010068B0250020BA91C83B901700682C130068C80E0068640A0068000600688CB60908642800209DF80810FE4800EB440000F8EA
:408580000A100AF1010000F0FF0ABAF1020FFFF633AF9DF81400C0EB001000EB4000F64901EB001038309DF8101001EB410202EBC10100EB81002430005D029006F192011B
:4085C0000819012202A9FFF7D7FD4D4504D19DF80810E8480E380155601CC4B2022CFFF608AF9DF81400C0EB001000EB4000E24901EB001038309DF8101001EB410202EB27
:40860000C10100EB810090ED080A8DED030A042203A906F1C400FFF7AFFD4D4504D19DED030AD64880EDFF0A01200290012202A906F21920FFF7A0FD4D4504D19DF80810DC
:40864000CE4880F8511500200290012202A906F24140FFF791FD4D4504D19DF80810C74880F879170024CBE14FF0000A99E19DF81400C0EB001000EB4000BF4901EB001038
:4086800000F58A709DF8101001EBC10100EB8100801C005D019006F5987101EB840101EB4A00022201A9FFF767FD4D4507D1BDF80410B048903000EB840020F81A109DF86E
:4086C0001400C0EB001000EB4000AB4901EB001000F58A709DF8101001EBC10100EB8100001D005D019006F59C7101EB840101EB4A00022201A9FFF73FFD4D4507D1BDF8F9
:4087000004109C48983000EB840020F81A109DF81400C0EB001000EB4000974901EB001000F58A709DF8101001EBC10100EB8100801D005D019006F5A07101EB840101EBAB
:408740004A00022201A9FFF717FD4D4507D1BDF804108848A03000EB840020F81A109DF81400C0EB001000EB4000834901EB001000F58A709DF8101001EBC10100EB81003E
:408780000830005D019006F5A87101EB840101EB4A00022201A9FFF7EFFC4D4507D1BDF804107448B03000EB840020F81A109DF81400C0EB001000EB40006F4901EB001066
:4087C00000F58A709DF8101001EBC10100EB81000A30005D019006F5AC7101EB840101EB4A00022201A9FFF7C7FC4D4507D1BDF804106048B83000EB840020F81A109DF844
:408800001400C0EB001000EB40005B4901EB001000F58A709DF8101001EBC10100EB81000C30005D019006F5A47101EB840101EB4A00022201A9FFF79FFC4D4507D1BDF881
:4088400004104C48A83000EB840020F81A109DF81400C0EB001000EB4000474901EB001000F58A709DF8101001EBC10100EB81000E30005D019006F5B47101EB840101EB45
:408880004A00022201A9FFF777FC4D4507D1BDF804103848C83000EB840020F81A109DF81400C0EB001000EB4000334901EB001000F58A709DF8101001EBC10100EB810016
:4088C0001030005D019006F5B07101EB840101EB4A00022201A9FFF74FFC4D4507D1BDF804102448C03000EB840020F81A109DF81400C0EB001000EB40001F4901EB001045
:4089000000F58A709DF8101001EBC10100EB8100005D019006F5947101EB840101EB4A00022201A9FFF728FC4D4507D1BDF804101048883000EB840020F81A109DF814005F
:40894000C0EB001000EB40000B4901EB001000F5E4709DF8101001EB410100EB4100801C30F81400019006F5D67101EB840101EB4A0005E0702800208CB60908982400204B
:40898000022201A9FFF7F8FB4D4506D1BDF80410FD4800EB840020F81A100AF1010000F0FF0ABAF1020FFFF662AE9DF81400C0EB001000EB4000F54901EB001000F58A706A
:4089C0009DF8101001EBC10100EB8100143000EB840090ED000A8DED030A06F58B6101EB8400042203A9FFF7C7FB4D4506D19DED030AE74800EB840080ED000A601CC4B2FF
:408A0000022CFFF631AE9DF81400C0EB001000EB4000DE4901EB001000F5E4709DF8101001EB410130F811000190022201A906F5D570FFF7A1FB4D4504D1BDF80410D5489F
:408A4000A0F8E21402200190022201A906F5DB70FFF792FB4D4504D1BDF80410CD48A0F8EE1402200190022201A906F5DA70FFF783FB4D4504D1BDF80410C648A0F8EC142F
:408A8000681CC5B2052D7FF77FAC00BF0AB0BDE8F09F38B504460D461420BF4A0023009020462946FFF75EFC1520BB4A0023009020462946FFF756FC1620B74A00230090A8
:408AC00020462946FFF74EFC1720B34A0023009020462946FFF746FC1820AF4A0023009020462946FFF73EFC1920AB4A0023009020462946FFF736FC38BDF8B505460E4665
:408B0000A649691A76F1000038D2012433E0062C0CD2DFE804F00B0C09070503A04F08E0A04F06E0A04F04E0A04F02E000BFA04F00BF00BF012207F117016846FFF7F3FBDF
:408B400002F08FFFA0420ED100BF02226946994800685630FFF710FB20B99DF800108D48A0F88E1305E00222694607F15600FFF703FB601CC4B2052CC9DD00BFF8BD70B56A
:408B800005460E468C49691A76F100001ED2814890F8300540B1012809D0022802D003280BD107E07F2409E040F6EC1406E040F6EC1403E040F2FA2400E000BF00BF00EEA7
:408BC000104AB8EE400AF6F7BAFE00BF70BD2DE9FE4306460F4670494539711A77F1000057D202F03EFF804601244FE0062C0CD2DFE804F00B0C09070503694D08E0694DB8
:408C000006E0694D04E0694D02E000BF684D00BF00BF012205F1560102A8FFF784FB9DF808006F2801DB00200290012205F14C0101A8FFF778FB9DF80400052801DB00209F
:408C400001909DF80800C0EB001000EB40004F4901EB001038309DF8041001EB410202EBC10100EB810090ED080A8DED000A0422694605F1C400FFF77FFA444504D19DEDF8
:408C8000000A444880EDFF0A601CC4B2052CADDD00BFBDE8FE8301B500BF012269464748FFF76AFA20B99DF800003A4981F8300300BF08BD2DE9FC4104460D4616461F4614
:408CC0003F490020891BB84114D23D490020091BA8410FD30020FFF7DEFF3A4903C9CDE900019DF8070000F00F0010B10120FFF7D2FF00BFBDE8FC812DE9FE4F0646894618
:408D0000174698460020009083464FF4807200233846414677F0DAFD05464FF4807200233846414677F0D2FD924615B9BAF1000F4AD0ADB1002411E006EB0420029009EB7E
:408D4000042001904FF48072DDE90110FFF7EBFA009000984BEA000B601CC4B2AC42EBD3BAF1000F32D006EB0520029009EB052001901FFA8AF2DDE90110FFF7D4FA009083
:408D800000984BEA000B21E07C2900208CB60908282C002098240020C64EB93B3A91C83B901700682C130068C80E0068640A006800060068840000102514AA3B3003006817
:408DC000D2D19A3BF86F00084FF0400B5846BDE8FE8F70B505460E46FE49691A76F100003DD2012002F00CFE04F068FAFA2803D004F064FAFB2819D102F033FE0446F648BC
:408E000090F88E03C0EB001000EB4000F34901EB00121521204602F028FEEF4991F87807FCF76AFB0120F8F793FF02E00020FCF763FB022404E0204602F079FF601CC4B2EC
:408E4000052CF8DD40F264420023E5480168E548FFF752FFE04991F85807F7F7C2FE70BD2DE9F84305460E46DA492731691A76F1000047D24FF00708D6491331691A76F1F2
:408E8000000001D24FF00908FF200090012436E0062C0CD2DFE804F00B0C09070503D24F08E0D24F06E0D24F04E0D24F02E000BFD14F00BF00BF022207F156016846FFF71F
:408EC00032FA9DF800004044C0B200909DF80000132812DD9DF800006F280EDA0222694607F15600FFF748F902F0BBFDA04204D19DF80010B848A0F88E13601CC4B2052C9E
:408F0000C6DD00BFBDE8F8832DE9F04105460E46B0491739691A76F1000022D2AE4890F88E7390F88483002418E0C7EB071000EB4000AA4901EB001000F58A7008EBC801EA
:408F400000EB8100143000EB8400D0ED000AB0EE600A204601F068FC601CC4B2022CE4DB00BFBDE8F08170B504460D46A349611A75F100000AD2984890F8C90318B1032009
:408F8000FBF79CF902E00020FBF798F970BD7FB505460E469A49691A76F1000017D2002003F017FD002003F030FD10229549684678F014F96846FFF74FF9012404E02046FA
:408FC00002F0B5FE601CC4B2052CF8DD03DF7FBD2DE9FC4705460E468B49691A76F1000049D24FF014084FF0150900200190009001243DE0062C0CD2DFE804F00B0C0907B8
:409000000503794F08E0794F06E0794F04E0794F02E000BF784F00BF00BF042239466846FFF781F90098142802D1FA20019007E00098152802D1FB20019001E0002001908E
:4090400002F00FFDA0420CD100BF042201A964480068FFF791F818B95F490198C1F8380304E0042201A93846FFF786F8601CC4B2052CBFDD00BFBDE8FC872DE9F34F82B035
:40908000844600BF00210A460B460E460F46002001908046009063E09CF80000A0F13004E5179CF800002E2838D1B8F1000F0CD156494FF00009A2FB010A03FB01A102FB69
:4090C0000919861949EB07071FE0B8F1010F0CD14F494FF00009A2FB010A03FB01A102FB0919861949EB07070FE0B8F1020F0CD14FF47A714FF00009A2FB010A03FB01A16C
:4091000002FB0919861949EB070708F1010000F0FF0800200090002213461BE09CF80000C0B1009810B922462B460FE0009801280CDB0A214FF0000B9146A9FB010E03FB45
:4091400001E102FB0B19021949EB05030098401CC0B200900CF1010C0198401CC0B2019003990198884297DBB6185F413046394604B0BDE8F08F10B50446102225492046DC
:4091800078F02CF810BD73B50C46204602F022FC05460222694605F11000FEF7EDFF20B99DF800100C48A0F848137CBDFEB50020029001900090012540F69851064878F0E2
:4091C000AEF80122144902A8FFF7ADF89DF80800401C23E06D0CAA3B982400208CB6090884000010D0270020901700682C130068C80E0068640A006800060068ECCD9A3B0A
:4092000034CB9A3B9CBE0008B891C83B00CA9A3B40420F00B02500202C010068C0B20190012201A9D048FEF7A7FF002002900122CD4902A8FFF777F89DF808009DF804102F
:40924000884206D0C948008840F08000C7490880AFE00122C449C91E6846FFF764F89DF8000013284CD04FF44E71C14878F057F840F26441BF4878F052F84FF4FF71BE48D0
:4092800078F04DF840F2FE31BC4878F026F84FF44E720023B6494FF0D040FEF790FF01240BE0204602F096FB064640F264420023B049FEF784FF601CC4B2052CF1DD4FF439
:4092C000FF720023AC49AE48FEF779FF40F2FE320023AA49AB48FEF772FF1320009001226946A148C01EFEF747FF002405E021460620FFF748FF601CC4B2052CF7DD58E018
:409300004FF44E7200234FF0D0419948FFF7F4FC02F0A7FB044602F073FB00219448A0F84813022298480168103192481030FEF7FAFF8F48B0F84803062823D040F264414A
:409340008C4877F0ECFF4FF4FF718B4877F0E7FF40F26442002387498B480068FEF72FFF4FF4FF72002384498548FEF728FF012405E021460620FFF706FF601CC4B2052C89
:40938000F7DD16E0022540F2644200237E4801687848FFF7B1FC4FF4FF72002378497648FFF7AAFC40F2FE32002376497348FFF7A3FC2846FEBD70B590B000BF182102A879
:4093C00077F0ADFF01206949088000206F4908706F480FF08FFC10B100206449088063480088002812D1FFF7E1FE6A490880102269490CA877F0F2FE66480088012806D1E5
:409400000020624908700CA8FEF726FFA0E001205E49087010210CA8FFF72FFE5F4A03C208A8FFF7A8FE102108A8FFF726FE0D4604465A48D0E90021101BA94121D200205D
:4094400003F0C7FA002003F0E0FA002007F043FD102251490CA877F0C1FE0CA8FEF7FCFE182102A877F05BFF012604E0304602F05EFC701CC6B2052EF8DD0EF06FFC03DFE3
:4094800064E0464903C9201A75EB01005ED220462946FFF79DFD20462946FFF778FD20462946FFF760FD20462946FFF72DFD20462946FFF7D5FC20462946FFF78AFC374814
:4094C0000CC820462946FFF7F5FB1E20344A0023009020462946FEF745FF20462946FFF776FB20462946FFF74AFB20462946FFF704FB20462946FFF7CCFA20462946FEF7EF
:40950000DAFE20462946FEF7CAFE20462946FEF7B3FE002003F05DFA002003F076FA002007F0D9FC10221C490CA877F057FE0CA8FEF792FE40F2FE31104877F0CEFE40F20F
:40954000FE3200230D490F48FEF739FEFEF7FBFD0020FCF7F2FB10B070BD054890F8300370470E4903C970472C0100688A00001098240020D0270020342C0020322E00202A
:4095800000040068001C0068840000108000001000300140880000109CBE000890000010B20CAA3B10B52DED088B0446FE4890F83800002840D1FD4890F83800D8BB94F8CA
:4095C0000001032829D103F0A0F842F21071884223D9F549086B4FF4FA6140F093F938B9F249086B4FF4FA6140F08CF9002813D00120ED4981F83800EC4981F8380040F019
:4096000067F9E949086340F063F9E849086340F05FF9E749C1F8E40FFEE340F059F9E249086340F055F9E149086340F051F9E049C1F8E40FF0E7FFE794F8000138B90020EB
:40964000D94981F83800D94981F83800E4E70120D54981F83800D54981F83800F6F7D3FFF0EE408A02F0FEFE00287CD0D4ED3A0AB0EE600A4FF0FF31CB48083010F0C1FC6D
:4096800094ED3A0AC848D0ED020A30EE600AB0EE408A28EE080AB0EE408A4FF0FF311030B0EE480A10F0ADFCBF4890ED040A10EE101A08467FF0DCF841EC1B0BB0EE4B0AB3
:4096C000F0EE6B0A7CF038FBB0EE40AAF0EE60AA9FEDB80B53EC102B51EC1A0B7EF0D2FD41EC190B7EF042FAAF498862084690ED020AB0EEC00AD0ED0A0A30EE200A80EDFE
:409700000A0AD4ED3B0AB0EE600A4FF0FF31183010F077FC94ED3B0AA348D0ED060A30EE600AB0EE408A28EE080AB0EE408A4FF0FF312030B0EE480A10F063FC9A4890ED72
:40974000080A10EE101A08467FF092F841EC1B0BB0EE4B0AF0EE6B0A7CF0EEFAB0EE40AAF0EE60AA00E0FCE39FED920B53EC102B51EC1A0B7EF086FD41EC190B7EF0F6F9A8
:409780008949C862084690ED060AB0EEC00AD0ED0B0A30EE200A80ED0B0AD4ED3E0AB0EE600A4FF0FF3110F02CFC7F49086B40F0CAF87D49496B08447B49486340F088F814
:4097C00079490863D4ED3A0AB0EE600A4FF0FF317648083010F015FC94ED3A0A7348D0ED020A30EE600AB0EE408A28EE080AB0EE408A4FF0FF311030B0EE480A10F001FC54
:409800006A4890ED040A10EE101A08467FF030F841EC1B0BB0EE4B0AF0EE6B0A7CF08CFAB0EE40AAF0EE60AA9FED620B53EC102B51EC1A0B7EF026FD41EC190B7EF096F92F
:409840005A498862084690ED020AB0EEC00AD0ED0A0A30EE200A80ED0A0AD4ED3B0AB0EE600A4FF0FF31183010F0CBFB94ED3B0A4E48D0ED060A30EE600AB0EE408A28EEC8
:40988000080AB0EE408A4FF0FF312030B0EE480A10F0B7FB454890ED080A10EE101A08467EF0E6FF41EC1B0BB0EE4B0AF0EE6B0A7CF042FAB0EE40AAF0EE60AA9FED3D0B63
:4098C00053EC102B51EC1A0B7EF0DCFC41EC190B7EF04CF93549C862084690ED060AB0EEC00AD0ED0B0A30EE200A80ED0B0AD4ED3E0AB0EE600A4FF0FF3110F082FB2B494A
:40990000086B40F020F82949496B0844274948633FF0DEFF25490863D4ED3A0AB0EE600AC821264810F09EFB94ED3A0A2348D0EDC90A30EE600AB0EE408A28EE080AB0EE87
:40994000408AC82100F54B70B0EE480A10F08AFB1B4890EDC90A10EE101A08467EF088FF41EC1B0BB0EE4B0AF0EE6B0A7CF0E4F9B0EE40AAF0EE60AA9FED0E0B53EC102B80
:4099800051EC1A0B7EF07EFC41EC190B7EF0EEF80749C1F8DC0F094890EDC90AB0EEC00A00F6D4000EE000003C0D0010780D0010B40D00100000000000000040E010001004
:4099C0000C140010D0EDF70A30EE200A80EDF70AD4ED3B0AB0EE600AC821A0F51F7010F041FB94ED3B0AFE48D0EDC90A30EE600AB0EE408A28EE080AB0EE408AC82100F572
:409A00004B70B0EE480A10F02DFBF64890EDC90A10EE101A08467EF02BFF41EC1B0BB0EE4B0AF0EE6B0A7CF087F9B0EE40AAF0EE60AA1FED200B53EC102B51EC1A0B7EF041
:409A400021FC41EC190B7EF091F8E749C1F8E00FE34890EDC90AB0EEC00A00F51F70D0EDF80A30EE200A80EDF80AD4ED3E0AB0EE600AC821DC4810F0F5FADB49D1F8E40FDF
:409A80003FF061FFD849D1F8E81F0844D649C1F8E80F3FF01DFFD449C1F8E40F00BF0422D249D348006800F51470FEF765FB30B9CE48083890ED020ACE4880ED940A00BFFE
:409AC00000BF0422C949091DC948006800F51570FEF752FB28B9C5480838C168C648C0F88C1500BF00BF0422C0490831C048006800F51670FEF740FB30B9BC48083890EDAB
:409B0000040ABC4880ED960A00BF00BF0422B7490C31B748006800F51770FEF72DFB28B9B24808384169B448C0F8941500BF00BF0422AE491031AE48006800F51870FEF757
:409B40001BFB30B9A948083890ED060AA94880ED980A00BF00BF0422A4491431A448006800F51970FEF708FB28B9A0480838C169A148C0F89C1500BF00BF04229B49183132
:409B80009B48006800F51A70FEF7F6FA30B99748083890ED080A974880ED9A0A00BF00BF042292491C319248006800F51B70FEF7E3FA28B98D480838416A8F48C0F8A41526
:409BC00000BF00BF0422894908398948006800F51C70FEF7D1FA30B98448083890ED000A844880ED9C0A00BF00BF04227F49091F7F48006800F51D70FEF7BEFA28B97B4843
:409C0000083841687C48C0F8AC1500BF00BF042276492C317648006800F51E70FEF7ACFA28B972480838416B7348C0F8B01500BF6E480838406B714988427CD96B4808380F
:409C400090ED0A0ADFED6E0A20EE200A80ED0A0A90ED0A0ADFED6B0AB4EEE00AF1EE10FA03DD9FED680A80ED0A0A6048083890ED0B0ADFED650A20EE200A80ED0B0A90EDC4
:409C80000B0ADFED620A20EE200A80ED0B0A90ED0B0ADFED5C0AB4EEE00AF1EE10FA03DD9FED580A80ED0B0A5048083890ED000ADFED530A20EE200A80ED000A90ED000A56
:409CC000DFED500AB4EEE00AF1EE10FA03DD9FED4D0A80ED000A4E480078401C4C49087008460078322801DB0020087000BF012247493F48006800F20C40FEF73DFA20B9E0
:409D0000434801783C4880F8441700BF00BF3849096801F2AE213E4A12788818012233492031FEF729FA70B93048083890ED0A0ABCEEC00A00E029E110EE100AC1B2354804
:409D4000334A1278815400BF00BF2949096801F538712F4A12788818012224492431FEF70BFA68B92148083890ED0B0ABCEEC00A10EE100AC1B227483230254A127881548B
:409D800000BF00BF1A49096801F51F71204A12788818012215490839FEF7EEF968B91348083890ED000ABCEEC00A10EE100AC1B218483238164A1278815400BF3C210B485F
:409DC000083877F0ACFA3FF083FD08490839086300BF042208310648006800F514701CE038170010641A0010B40D0010800D001084000010D02700209824002080EE36009B
:409E000000007A4400007F43E12E65420000C842940200207E2A0020C9E0FEF7ADF928B9FE4890ED020AFE4880ED940A00BF00BF0422FA490C31FB48006800F51570FEF7E1
:409E40009BF920B9F548C168F748C0F88C1500BF00BF0422F1491031F248006800F51670FEF78AF928B9ED4890ED040AEC4880ED960A00BF00BF0422E8491431E94800682E
:409E800000F51770FEF778F920B9E4484169E648C0F8941500BF00BF0422E0491831E148006800F51870FEF767F928B9DB4890ED060ADB4880ED980A00BF00BF0422D74982
:409EC0001C31D848006800F51970FEF755F920B9D248C169D448C0F89C1500BF00BF0422CE492031CF48006800F51A70FEF744F928B9CA4890ED080AC94880ED9A0A00BF8B
:409F000000BF0422C5492431C648006800F51B70FEF732F920B9C148416AC348C0F8A41500BF00BF0422BD49BE48006800F51C70FEF722F928B9B94890ED000AB84880ED3B
:409F40009C0A00BF00BF0422B449091DB548006800F51D70FEF710F930B9B0484168B24800E017E0C0F8AC1500BF00BF0422AB493431AC48006800F51E70FEF7FDF820B91C
:409F8000A648416BA848C0F8B01500BF4920EEF79BFA0CE03FF09CFCA44908633FF098FC9E4908633FF094FCA149C1F8E40FBDEC088B10BD10B52DED028B04460320F8F7B2
:409FC000A5FA50B10320F7F7B8FDF0EE408A0320F8F776FAB0EE408A09E00120F7F7ADFDF0EE408A0120F8F76BFAB0EE408A02F0CEFA18B9002084F800013AE0B0EEE80A70
:40A00000DFED8C0AB4EEE00AF1EE10FA10D2B0EEC80ADFED890AB4EEE00AF1EE10FA07D2032084F8000100212520F3F71FF920E0B0EEE80AF7EE000AB4EEE00AF1EE10FA4E
:40A0400010D2B0EEC80ADFED7D0AB4EEE00AF1EE10FA07D2022084F8000100212620F3F705F906E000212620F3F700F9012084F8000194F8010194F80011884206D094F8DA
:40A08000000184F801011320EEF71EFABDEC028B10BD70B50446F6F7B6FA84ED040AF8F778FA0546F8F71FFA84ED030AF8F771FA0546F8F705FA84ED010AF8F76AFA054684
:40A0C000F7F73BFD84ED000A70BD574A92F878130F297DD2DFE801F07CF608437DF5F4F3F2F1F0EF090AEE0000BF00BF9FED540A80ED060A9FED530A80ED070A9FED520A90
:40A1000080ED080A9FED510A80ED090A9FED490A80ED0A0A9FED4E0A80ED0B0A9FED4D0A80ED0C0A9FED4C0A80ED0D0A9FED4B0A80ED0E0A9FED4A0A80ED0F0A9FED490AFC
:40A1400080ED100A9FED480A80ED110A9FED470A80ED120AB5EE000A80ED130A42E19FED440A80ED060A9FED430A80ED070A9FED310A80ED080A9FED400A80ED090A9FED5C
:40A180003F0A80ED0A0A9FED3E0A80ED0B0A9FED3D0A80ED0C0A9FED3C0A80ED0D0A9FED3B0A80ED0E0A9FED3A0A80ED0F0A9FED390A80ED100A9FED380A80ED110A9FEDEF
:40A1C000370A80ED120A9FED360A80ED130A09E1C8E09FED340A80ED060A9FED320A80ED070A9FED310A80ED080A9FED300A80ED090A9FED2F0A80ED0A0A9FED140A80ED37
:40A200000B0A9FED0C0A80ED0C0A9FED110A80ED0D0A9FED130A80ED0E0A54E0780D0010D027002084000010982400203C0D0010B40D00109A99993E295C0F3D0E2DB23D0C
:40A24000EC51183F46B6F33E5C8FC23EC3F5A83E295C8F3E713D8A3E14AE873EDD24863EB81E853E9318843E6F12833E2506813E713D0A3F83C0CA3E5C8F823EEDD46C3EF6
:40A280002366563E24ED463E74B73B3EC329333EA6422C3E0D6F263E06A0213E707C1D3E9A99193E9A99193F8FC2F53E3D0AD73EA470BD3E58E01CE058E056E053E056E05E
:40A2C00056E056E014E0B5EE000A80ED0F0A9FEDFE0A80ED100A9FEDFD0A80ED110A9FEDFC0A80ED120A9FEDFB0A80ED130A79E000BF9FEDF90A80ED060A1FED130A80EDA5
:40A30000070A9FEDF60A80ED080A9FEDF50A80ED090A9FEDF40A80ED0A0A9FEDF30A80ED0B0A9FEDF20A80ED0C0A9FEDF10A80ED0D0A9FEDF00A80ED0E0A9FEDEF0A80EDCD
:40A340000F0A9FEDEE0A80ED100A9FEDED0A80ED110A9FEDEC0A80ED120A9FEDEB0A80ED130A3FE000BF00BF00BF00BF00BF00BF00BFB7EE000A80ED060AB7EE000A80EDF8
:40A38000070AB7EE000A80ED080AB7EE000A80ED090AB7EE000A80ED0A0AB7EE000A80ED0B0AB7EE000A80ED0C0AB7EE000A80ED0D0AB7EE000A80ED0E0AB7EE000A80ED19
:40A3C0000F0AB7EE000A80ED100AB7EE000A80ED110AB7EE000A80ED120AB7EE000A80ED130A00BF00BFB0EE000A80ED140AB7EE000A80ED150AB7EE000A80ED160AB7EE99
:40A40000000A80ED170AB7EE000A80ED180AB7EE000A80ED190AB7EE000A80ED1A0AB7EE000A80ED1B0AB7EE000A80ED1C0AB7EE000A80ED1D0AB7EE000A80ED1E0AB7EE18
:40A44000000A80ED1F0AB7EE000A80ED200AB7EE000A80ED210A704710B50446AB4804705720EEF731F86020EEF72EF810BD10B52DED068B3C21A64876F051FF3C21A548EA
:40A4800076F04DFF4FF47F61A34876F048FFFF21A1480FF03BFEFF21A0480FF037FEFF219F480FF033FEFF219E480FF02FFEFF219D480FF02BFE9D4890F844079C49087007
:40A4C0009C4890ED940A934880ED020A9748D0F88C159048C160974890ED960A8D4880ED040A9248D0F894158A484161914890ED940A884880ED060A8C48D0F88C15854872
:40A50000C1618C4890ED960A824880ED080A8748D0F894157F484162864890ED9C0A7D4880ED000A8148D0F8AC057A4948607F48D0F8B0054863084690ED040A10EE101A4B
:40A5400008467EF095F941EC1A0BB0EE4A0AF0EE6A0A7BF0F1FBB0EE409AF0EE609A9FED760B53EC102B51EC190B7DF08BFE41EC180B7DF0FBFA67498862084690ED020A53
:40A58000B0EEC00AD0ED0A0A30EE200A80ED0A0A90ED080A10EE101A08467EF069F941EC1A0BB0EE4A0AF0EE6A0A7BF0C5FBB0EE409AF0EE609A9FED600B53EC102B51EC05
:40A5C000190B7DF05FFE41EC180B7DF0CFFA5149C862084690ED060AB0EEC00AD0ED0B0A30EE200A80ED0B0A4920EDF76DFFBDEC068B10BD4FF6FF760121514880F858112E
:40A600000020504981F800019FED4F0A084680ED410ABFEE000A4D4880ED000A00204C49088090214B4876F07AFEFFF720FF0120FFF712FF4748303847490860001D474901
:40A640000860001D46490860001D46490860001D45490860083045490860001D44490860DFF810C100DF074639460220DFF808C100DF0421324880F8581100BF002231462B
:40A680004CF20300DFF8F4C000DF85B2012DF5D0DFF8ECC000DF044604F4004028B14FF416760321264880F8581104F4804028B14FF6FF760421224880F8581104F0020015
:40A6C00000286ED001215DE08FC2753ED7A3703E1F856B3ED578693ECDCCCC3E7B14AE3E52B89E3E745F8E3E28636C3E4E9D473E97FD2A3E520E163EF967063E07EAF43D6A
:40A70000C6BEE43D08ACDC3D3D0AD73D780200203C0D0010780D0010B40D0010E01000100C14001038170010641A00109824002094020020D02700200000000000000040ED
:40A7400030320020A41D0010000000008402002096020020BC1E0010580200205C020020600200206402002068020020700200206C0200202D7A0908316D0908916D09081E
:40A78000D96C0908FA4880F8FC10FA4890F8BE74012F0CD0022F05D0032F0DD0042F15D10FE029E036F0F8FCF349086013E037F095F8F14908600EE036F082FEEE49086015
:40A7C00009E037F0DBFEEC49086004E037F00AFAE949086000BF00BFE74800680168E4488847E348FFF771FC9FEDE40A72F0FCF8E34880ED000A00BF04F0010000283FF4A2
:40A800003DAFDB48E830FFF744FCD948FFF7D2FBD9480068DB494268D5489047D448FEF7C1FE71F0C6FA29E731B52DED020B04460225022C39DA9DED000ADFEDD30AB4EEED
:40A84000E00AF1EE10FA04DD9FEDCF0A8DED000A0CE09DED000ADFEDCD0AB4EEE00AF1EE10FA03D29FEDC90A8DED000A00BFC849096801F58B6101EB840004226946FDF78F
:40A880007BFC30B99DED000AC24800EB840080ED000A00BFC048D0F854110220DFF8FCC200DFAB20EDF710FE002528463EBDB04890F800017047B34800797047F0EE400A54
:40A8C00090ED010AB0EE401A9FEDB50AF4EEC00AF1EE10FA03D29FEDB20AF0EE400A81EE200A7047F0EE400A90ED220AB0EE401A9FEDAB0AF4EEC00AF1EE10FA03D29FED63
:40A90000A80AF0EE400AB6EE080A61EE001AB6EE080A30EE802A81EE820A7047A14800787047B0EE401AF0EE601AB0EE410A914991F83015022902D19FED9B2A01E09FED39
:40A940009B2AB4EEE12AF1EE10FA0BDD894991F83015022902D19FED942A01E09FED932AF0EE421A90ED262A61EEA12AC2EE220AB4EEE01AF1EE10FA05DDB0EE600A0121F4
:40A980008B4A117011E0B1EE602AB4EEC21AF1EE10FA07D2B1EE602AB0EE420A0121844A117002E00021824A1170704780480078704700207E4908707047F0EE401AB0EE79
:40A9C000612A6C4890F83005022802D19FED760A01E09FED760AB4EEE00AF1EE10FA22DD72EE412AB0EE620A6548D0ED002AB4EEE20AF1EE10FA05DDD0ED002A71EE222A9D
:40AA0000B0EE622A5E48D0ED002AF1EE622AB4EEE20AF1EE10FA05D2D0ED002A71EE622AB0EE622A00BFB0EE420A70475FEDBA0AB0EE600A5348007920B15248D0ED000AEC
:40AA4000B0EE600A704710B50246F0EE400AB7EE000AB0EE401A5348007888B3F2EE0A1AF4EEE10AF1EE10FA03DBDFED521AF0EE610AFDEEE01A11EE903A18B201EE900AD3
:40AA8000F8EEE11A30EEE10A01291AD102F15003441C03EB8403D3ED001A02F1500303EB800393ED002A31EEC22A02F1500303EB8003D3ED001A40EE021AB0EE611A19E049
:40AAC00019E002F11803441C03EB8403D3ED001A02F1180303EB800393ED002A31EEC22A02F1180303EB8003D3ED001A40EE021AB0EE611A00BF92ED240A20EE010A10BD5E
:40AB000000201C4991F87813042900D00120704701B500BF012269461D48006800F5C370FDF72AFB20B99DF80010124880F8BE1400BF08BDF7B50C461546FAF71EFD08B18E
:40AB4000642000E0C82006460027BDF90000B04202DD0096022744E0FAF70FFD38B1BDF90000012828DA01200090032739E023E0A41D0010982400209802002044D8F03B40
:40AB8000740200208C020020003C1C46003C1CC684000010282C002030320020316D0908CDCCCC3F780200200AD7A33C9A99193E880200200AD74F41FA48007838B1BDF960
:40ABC0000000322803DA32200090032709E0F548007830B9BDF90000012802DA012000900327022C2BDA00BFEF49096801F5947101EB840101EB450002226946FDF7BCFA40
:40AC000038B9BDF8000081B2E84800EB840020F8151000BF0D20EDF757FC22202DF0DCF8E348D0F854110220DFF888C300DFE048D0F808120120DFF87CC300DF00E0022765
:40AC40003846FEBDF7B50C4615460026BDF90000FF2803DDFF200090022606E0BDF90000002802DA002000900326022C25DA00BFCD49096801F5987101EB840101EB4500FB
:40AC800002226946FDF778FA40B9BDF8000081B2C648083000EB840020F8151000BF0E20EDF712FC22202DF097F8C148D0F854110220DFF800C300DF00E002263046FEBDB1
:40ACC000F7B50C4615460026BDF90000FF2803DDFF200090022606E0BDF90000002802DA002000900326022C25DA00BFAE49096801F59C7101EB840101EB450002226946FC
:40AD0000FDF73AFA40B9BDF8000081B2A748103000EB840020F8151000BF0F20EDF7D4FB22202DF059F8A248D0F854110220DFF884C200DF00E002263046FEBDF7B50C4672
:40AD400015460026BDF90000FF2803DDFF200090022606E0BDF90000002802DA002000900326022C25DA00BF8F49096801F5A87101EB840101EB450002226946FDF7FCF9A3
:40AD800040B9BDF8000081B28848283000EB840020F8151000BF8C20EDF796FB23202DF01BF88348D0F854110220DFF808C200DF00E002263046FEBDF7B50C461546002639
:40ADC000BDF90000FF2803DDFF200090022606E0BDF90000002802DA002000900326022C25DA00BF7049096801F5A07101EB840101EB450002226946FDF7BEF940B9BDF85B
:40AE0000000081B26948183000EB840020F8151000BF1020EDF758FB22202CF0DDFF6448D0F854110220DFF88CC100DF00E002263046FEBDF7B50C4615460026BDF900006E
:40AE4000FF2803DDFF200090022606E0BDF90000002802DA002000900326022C25DA00BF5149096801F5AC7101EB840101EB450002226946FDF780F940B9BDF8000081B2AE
:40AE80004A48303000EB840020F8151000BF8D20EDF71AFB23202CF09FFF4548D0F854110220DFF810C100DF00E002263046FEBDF7B50C4615460026BDF90000FF2803DDBA
:40AEC000FF200090022606E0BDF90000002802DA002000900326022C25DA00BF3249096801F5A47101EB840101EB450002226946FDF742F940B9BDF8000081B22B482030D7
:40AF000000EB840020F8151000BF1120EDF7DCFA22202CF061FF2648D0F854110220DFF894C000DF00E002263046FEBDF7B50C4615460026BDF90000C82803DDC820009080
:40AF4000022606E0BDF90000012802DA012000900326022C30DA00BF1349096801F5B47101EB840101EB450002226946FDF704F940B9BDF8000081B20C48403000EB8400D5
:40AF800020F8151000BF0C20EDF79EFA23202CF023FF0748D0F854110220DFF818C000DF0BE000007802002084000010F828002030320020316D090802263046FEBDF7B5B1
:40AFC0000C4615460026BDF90000642803DD64200090022606E0BDF90000012802DA012000900326022C24DA00BFFE49096801F5B07101EB840101EB450002226946FDF782
:40B00000BBF838B9BDF8000081B2F74800EB840020F8151000BF4D20EDF756FA23202CF0DBFEF248D0F854110220DFF8C4C300DF00E002263046FEBD10B50E20EDF744FAED
:40B040000F20EDF741FA1020EDF73EFA8C20EDF73BFA8D20EDF738FA1120EDF735FA0D20EDF732FA0C20EDF72FFA4D20EDF72CFA22202CF0B1FE23202CF0AEFE10BDF0B5F3
:40B080002DED0E8B97B00446F0EE408AB6EE000AF4EEC08AF1EE10FA03D2B6EE000AF0EE408A94ED260A68EEA80A80EE209A94ED280AB4EEC90AF1EE10FA06D2FAF75DFAA4
:40B0C00018B994ED280AB0EE409AB7EE000AC0EE09EA0121B0EE680A2046FFF7B4FCD4ED270A20EE208AC34890F8D80050B1C24890F8E004012805D0B6EE000A28EE000A6E
:40B10000B0EE408AB0EE000A30EE480A60EE2E9A89EE88EA20210FA876F001F9CDED0F9A9FEDB60A29EE800A8DED110A9FEDB30A2EEE000A20EE080A8DED140A8DED16EAB2
:40B14000002661E00127002537E000EE105AB8EE400AB2EE041AC0EE010A9FEDA90A30EE800AF0EE40AADFEDA70A7AEEE00AB0EE600A01A90FA810F05EFB03A9B0EE6A0A47
:40B180000FA810F058FBDFED9F0A7AEEA00AB0EE600A05A90FA810F04EFB01A810F0D1F9B0EE40BAB0EECB0AB4EEC90AF1EE10FA01DD002703E0681C85B2032DC5DB00BF3A
:40B1C00007B123E09DED0F0ADFED8F0A20EE200A8DED0F0A9DED110ADFED8B0A20EE200A8DED110A9DED140ADFED870A20EE200A8DED140A9DED160ADFED830A20EE200ADE
:40B200008DED160A701C86B20A2E9BDB00BF9DED120ADDED100A30EE600AF0EE080A20EE200A8DED0A0A9DED110ADDED0F0A30EE600AF0EE080A20EE200A8DED090A9DED2C
:40B24000140ADDED120A30EE600AF0EE080A20EE200A8DED0C0A9DED130ADDED110A30EE600AF0EE080A20EE200A8DED0B0A9DED160ADDED140A30EE600AF0EE080A20EEA7
:40B28000200A8DED0E0A9DED150ADDED130A30EE600AF0EE080A20EE200A8DED0D0ABDEEE80A10EE100A00B2584908800846B0F90000042801DA042008805448B0F9000082
:40B2C0000C2802DD0C20514908805048B0F90000800000EE100AB8EEC00AF7EE000A80EE80AA002575E000EE105AF8EE400A4748B0F9000000EE100AB8EEC00A80EE801A73
:40B30000F0EE41AA3AEE8A0AF0EE40AA07A9B0EE6A0A0FA810F08FFA9DED070A05EB450104F58C7000EB810080ED000A07A9B0EE6A0A09A810F0E7FA9DED070ADDED080A4A
:40B3400080EE201A11EE106A30467DF091FA41EC1D0BB0EE4D0AF0EE6D0A78F0D1FDB0EE40CAF0EE60CA9FED2A0B53EC102B51EC1C0B7CF087FF41EC1B0B7CF0F7FB05EB87
:40B38000450204F58C7101EB820148607AEECA0AB0EE600A01A90FA810F04DFA03A9B0EE6A0A0FA810F047FA7AEE8A0AB0EE600A05A90FA810F03FFA01A810F0C2F805EBA2
:40B3C000450104F58C7000EB810080ED020A681C85B20E48B0F90000401EA84283DC9FED0E0A1BE0840000103029002030320020316D0908C81C0020982400206666E63E1F
:40B400009A99993ECDCC4C3DCDCC8C3F96020020000000000000F0BF000000009348B0F90000401E00EB400104F58C7000EB810080ED000A1FED080A8C48B0F90000401E36
:40B4400000EB400104F58C7000EB810080ED010A1FED0F0A8548B0F90000401E00EB400104F58C7000EB810080ED020A94ED480AF6EE000A20EE200A84ED480A17B0BDEC9C
:40B480000E8BF0BD31B50024BDF80000642803DD64200090022406E0BDF80000002802DA0020009003247248B0F86607BDF8001088420FD000BF022269466E48006800F28C
:40B4C0002E40FCF759FE20B9BDF800106848A0F8661700BF9520ECF7F7FF6748D0F854110220DFF898C100DF204638BD70B52DED048BB0EE409A04460D46B5EEC09AF1EEBD
:40B5000010FA04DD94ED370A30EE098A03E094ED350A30EE098A94ED380AB4EEC80AF1EE10FA03D294ED380AB0EE408A94ED360AB4EEC80AF1EE10FA03DD94ED360AB0EEDC
:40B54000408A95ED440ABCEEC00A10EE100A3EF0FAF900EE100AF8EE409A94ED390A60EE298A94ED370AB4EEC80AF1EE10FA08D895ED450AD4ED370AB4EEE00AF1EE10FAB0
:40B580000FD394ED350AB4EEC80AF1EE10FA14DB95ED450AD4ED350AB4EEE00AF1EE10FA0BDD94ED350AB0EEC00AD4ED370A30EE200A30EE280AF0EE408A95ED450A38EE0E
:40B5C000400AB4EEE80AF1EE10FA06DD95ED450A30EE280AB0EE408A10E095ED450A38EE400AF1EE680AB4EEE00AF1EE10FA05D295ED450A30EE680AB0EE408A3EF068F9F2
:40B6000000EE100AB8EE400A85ED440A85ED458AB0EE480ABDEC048B70BD154890F8BE0420B1134890F8BE04012801D1012070470020FCE70E4890F8BE04022801D101200C
:40B6400070470020FCE70A4890F8BE04032801D1012070470020FCE7054890F8BE04042801D1012070470020FCE7000096020020982400208400001030320020316D0908D3
:40B680000021C74A1170C74A117090ED010AC64981ED010A90ED000A81ED000A90ED010AC24981ED010A90ED000A81ED000A9FEDC00AC04981ED010A9FEDBD0A81ED000A88
:40B6C000704730B52DED028B87B004460D46BA48007830B92046FFF7D3FF07B0BDEC028B30BD00EE105AB8EE400ADFEDB40A80EE208A9FEDB30AB4EEC08AF1EE10FA00D2EE
:40B70000EBE7A94890ED010AAA48D0ED010AB6EE001A60EE810A00EE880AA34880ED010A90ED000AA348D0ED000AB6EE001A60EE810A00EE880A9C4880ED000A94ED010A53
:40B740009A48D0ED010A30EE600AC0EE080ACDED060A94ED000AD0ED000A30EE600AC0EE080ACDED050A9DED060A9248D0ED010A30EE600A8DED040A9DED050AD0ED000AFE
:40B7800030EE600A8DED030A94ED010A8648D0ED010A30EE600A8DED020A94ED000AD0ED000A30EE600A8DED010A9DED040A20EE000ADDED030A9DED031AF0EE408A40EEE7
:40B7C000818AB3EE090AF4EEC08AF1EE10FA7DDD744800787249087001207249087070480078E0B3704890ED010A7648D0ED010A30EE200A6C4880ED010A90ED000A714823
:40B80000D0ED000A30EE200A674880ED000A94ED010AD0ED010A30EE600A8DED020A94ED000AD0ED000A30EE600A8DED010A9DED020ADFED650A20EE200A80ED010A9DED07
:40B84000010ADFED610A20EE200A80ED000A94ED010A564880ED010A94ED000A00E002E080ED000A67E09DED060A20EE080A554880ED010A9DED050A20EE080A80ED000A2B
:40B88000494890ED010A4B48D0ED010AB6EE001A60EE810A00EE880A434880ED010A90ED000A4448D0ED000AB6EE001A60EE810A00EE880A3C4880ED000A90ED010A3B4803
:40B8C00080ED010A384890ED000A00E003E0374880ED000A2FE0002032490870304908709DED040ADFED390A20EE200A314880ED010A9DED030ADFED350A20EE200A80EDE6
:40B90000000A9DED020ADFED300A20EE200A264880ED010A9DED010ADFED2B0A20EE200A80ED000A94ED010A204880ED010A94ED000A80ED000A1C4890ED010A84ED010A28
:40B9400090ED000A84ED000A00BFC6E600201A49087070471248007870471D49087070471B4800787047174870470CB50F4890ED010A0D48D0ED010A30EE600A8DED010A18
:40B980000A4890ED000A0848D0ED000A30EE600A8DED000A9DED000ADDED010A0CBD0000C1020020C0020020A8020020A002002000000000B00200209C02002000007A44BA
:40B9C0000AD7233CB8020020CDCCCC3DCDCC4C3EC20200200146EE48062904D2DFE801F0030406080A0C00BFEA4807E0EA4805E0EA4803E0EA4801E0E54800BF00BF7047A6
:40BA000001B59DF80000012802DA0120009005E09DF80000052801DD052000909DF80000FFF7D8FFDF49086040F26442002308460168DD48FDF760F99DF80000DB49087084
:40BA400000BF01226946DA48FCF796FB20B99DF80000D84981F82A0100BFB820ECF734FD08BDD44890F82A01704770B504460D461646062C53D2DFE804F052031222324239
:40BA800000BF1E223146CC48FCF776FB28B92A463146C848283075F0A1FB00BF40E000BF1E223146C4481E30FCF766FB28B92A463146C048463075F091FB00BF30E000BF9F
:40BAC0001E223146BC483C30FCF756FB28B92A463146B848643075F081FB00BF20E000BF1E223146B4485A30FCF746FB28B92A463146B048823075F071FB00BF10E000BFFE
:40BB00001E223146AC487830FCF736FB28B92A463146A848A03075F061FB00BF00E000BF00BFB820ECF7D0FC70BD70B504460D46062C27D2DFE804F026030A11181F15221A
:40BB40009C492831284675F049FB1CE0152299494631284675F042FB15E0152295496431284675F03BFB0EE0152292498231284675F034FB07E015228E49A031284675F0DE
:40BB80002DFB00E000BF00BF70BDF8B504460025062C63D2DFE804F0620316293C4F0120FFF718FF0646042231466846FCF7BBFB0098C0B2FA2803D00098C0B2FB2800D1FA
:40BBC00001254CE00220FFF705FF0646042231466846FCF7A8FB0098C0B2FA2803D00098C0B2FB2800D1012539E00320FFF7F2FE0646042231466846FCF795FB0098C0B241
:40BC0000FA2803D00098C0B2FB2800D1012526E00420FFF7DFFE0646042231466846FCF782FB0098C0B2FA2803D00098C0B2FB2800D1012513E00520FFF7CCFE064604227A
:40BC400031466846FCF76FFB0098C0B2FA2803D00098C0B2FB2800D1012500E000BF00BF2846F8BD70B50625012406E02046FFF78CFF00B92546601CC4B2052CF6DD2846D4
:40BC800070BD10B5044649480470B820ECF71CFC10BD46480078704710B5012407E02046FFF773FF08B1012010BD601CC4B2052CF5DD0020F8E710B50446152221463F4878
:40BCC00075F08CFA3D4811F087FB00203B49087540F261103EF05CFE10BD384870472DE9F04106460D4601241DE0AC4219D034492046FFF71AFF304675F0FAF907463A4695
:40BD00002F49304675F0A4F958B9304675F0F0F907462B4875F0ECF9874202D10120BDE8F081601CC4B2052CDFDD0020F7E770B504461521234875F0D0FA224A152120463D
:40BD4000FFF793FE40F26441174875F0E8FA2046FFF740FE054640F264421349FCF70CFA21460620FDF70FFA40F2644200230D4801680D48FCF7C0FF70BD10B504462046C1
:40BD800075F0B6F908B9012010BD0020FCE700009017006800060068640A0068C80E00682C13006884000010D0270020C30200202A01006898240020280000684C1F00107B
:40BDC000611F0010761F001000B587B003A804A905AB06AACDE90010CAA1CD4874F0A8FF4FF44051049841EA00200399084380B207B000BD2DE9F0432DED028B83B0054663
:40BE00000C4616464FF00008C146002002902868B0F56F4F06D0BF490844002875D0FF286ED14AE1686804286CD14FF0080920700BF0B0F8DFEDB80A30EE200ADFEDB70A1A
:40BE400020EE200ABCEEC00A10EE100A80B20290BDF808006070BDF808000012A0700BF09DF8DFEDAD0A30EE200ADFEDAC0A20EE200ABCEEC00A10EE100A80B20290BDF8B4
:40BE80000800E070BDF80800001220710BF0A0F80746012F06DD072F04DA0BF0A4F8B0EE408A18E09E4890ED158A90F8D80090B19FED990A38EE000AB0EE408A9FED990A33
:40BEC000B4EEC08AF1EE10FA05DD9FED960A38EE400AB0EE408A9FED910A28EE000ABCEEC00A10EE100A80B20290BDF808006071BDF808000012A071FF20E07103E004E04B
:40BF0000F5E0FFE700BF00BFF2E04FF00809002020706868B0F57A4F6CD00CDC7B283AD004DC652827D0682872D117E0CA283FD0CB28F9D14DE04FF60322811A904268D0BF
:40BF400007DC6FF47A410844002863D00128EBD16EE006297CD00729E6D19EE0032060706820A0700020E07020716071A07105F08DFBE0719FE0132060706520A070002093
:40BF8000E070FFF721FF0290BDF80800A0800020A071E0718FE0332060707B20A0700020E07005F0E2FB8DED010A0198606082E00B206070CA20A0700020E0705A48B0F8BC
:40BFC0007E070290BDF80800E08000202071607171E00B206070CB20A0700020E0705248B0F880070290BDF80800E08000202071607160E0132060700020A070FA20E070FD
:40C000003DF00FFF207100206071A071E07152E050E01EE0132060700120A070FA20E07000202071102060710020A071E07142E0132060700220A070FA20E070FFF7C4FE36
:40C040000290BDF80800A0800020A071E07132E016E0132060700320A070FA20E07000202071324890F8420000F01F0060712F4890F84100A0712D4890F84000E0711AE079
:40C08000132060700920A070FA20E0700120207100206071A071E0710DE0132060700A20A070FA20E070AA20207100206071A071E07100E000BF00BF1AE04FF008090120CA
:40C0C00020700AF08CFF0290BDF808006070BDF808000012A0700AF07BFFE07054202071C82060718420A0710020E07100E000BF00BFA6F80090404603B0BDEC028BBDE8E5
:40C10000F083000025642E25642E25642E2564009CBE00080011E7FFDC0F494000401C46C81C0020DA0FC94098240020607C02202DE9FF413DF083FD002605463DF038FDC9
:40C14000B0460746FD4874F0D3FFC4B2012340222146FA48CDE90078CDE902560DF069FC18B1012004B0BDE8F0810020FAE710B50020F3490870F3490870F34908703DF0DB
:40C18000A7FBF2490860FFF7D3FF10B9002004F082FE10BD10B5EE48007A062870D2DFE800F0035B3490AA76F2F7EEFA90B969F073FB78B96AF038FC60B968F089FD48B9D2
:40C1C00001F07CF8FB2805D00020E14948720220087219E068F07CFD28B10020DC4948720120087210E069F057FB28B10020D84948720520087207E06AF016FC20B10020B3
:40C20000D34948720320087207E1F2F7BDFAE8B969F042FBD0B96AF007FCB8B968F058FDA0B901F04BF8FB2810D0C548007848B10220C7494872042008726DF05EFB00205A
:40C24000BF4908700020BF49087004E00220C049487200200872E0E068F03AFD88B1B848007848B10120BA494872042008726DF044FB0020B24908700020B249087005E01F
:40C28000C7E00120B249487200200872C5E069F003FB80B1AA48007848B10520AC494872042008726DF029FB0020A54908700020A449087004E00520A5494872002008728E
:40C2C000ABE06AF0B1FB80B19D48007848B103209F494872042008720020994908706DF00CFB00209749087004E00320984948720020087291E09648407A02282BD1F2F719
:40C3000043FA00BB69F0C8FAE8B96AF08DFBD0B968F0DEFCB8B900F0D1FFFB2813D089480078002874D0002086490870844908700120854908700420854948720220087265
:40C340006DF0CEFA64E0042081494872002008726DF0C6FA5CE07E48407A01281BD168F0B7FC80B177480078002851D00020754908707349087004207549487201200872A7
:40C380006DF0AEFA44E0042071494872002008726DF0A6FA3CE06E48407A03281AD16AF043FB78B16748007850B300206549087063490870042066494872032008726DF0A7
:40C3C0008FFA25E0042062494872002008726DF087FA1DE05E48407A052819D169F05CFA78B15848007858B100205649087054490870042056494872052008726DF070FA12
:40C4000006E0042052494872002008726DF068FA03E000204E49087200BF00BF4C48807A4B49097A884206D14FF47A71474800683DF068FA68B14648007A454988723DF0E2
:40C4400047FA4249086007202BF0C6FC2E20ECF73BF83F48007A042803D03DF039FA3C49486010BD3B4890F83005022802D19FED3A1A01E09FED391AF0EE410AB0EEC01A48
:40C48000B4EEE01AF1EE10FA01DD012070470020FCE7304890F87803072804D02D4890F87803062802D19FED2E0A01E09FED2D0A704710B52DED028BF4F7A5F8B0EE408ACC
:40C4C000FFF7E7FFF0EE408AB4EEE88AF1EE10FA03D20120BDEC028B10BD0020FAE710B52DED028B1B4890F87803072804D0194890F87803062802D19FED1A8A01E09FEDEA
:40C500001A8AF4F780F8B4EEC80AF1EE10FA03DD0120BDEC028B10BD0020FAE710B52DED028B0C4890F87803072804D0094890F8780306281CD19FED0D8A1BE01C260020DD
:40C54000C5020020C6020020C7020020C8020020A41F0010982400200AD7A33C9A99193EE3A5AB4083C00041B81E41413D0A0F419FEDE88AF4F747F8B4EEC80AF1EE10FAB5
:40C5800003DD0120BDEC028B10BD0020FAE7E249097A042905D1E049497A022901D1012100E0002108467047DB49097A042905D1D949497A052901D1012100E000210846B4
:40C5C0007047D549097A042905D1D349497A032901D1012100E0002108467047CE49097A042904D1CC49497A012900D100E0002108467047C849087A704710B50024FFF73D
:40C60000C6FF28B9FFF7DDFF10B9FFF7CDFF30B1F2F74EF908B1062421E004241FE0FFF7DDFF08B101241AE0BB48007A01280BD0B948007A022807D0B748007A052803D0BB
:40C64000B548007A032806D1F2F732F908B1052405E0022403E0B148007800B10324204610BD10B5AC48007A092831D2DFE800F0061B1D1A24193031050000BF00F080FD9C
:40C6800008B108240CE0A648007830B9A548C06B00F08060B0F1806F01D1012400E0002419E000BF00BF012415E0F2F701F908B1052400E002240EE0FFF790FF08B101243A
:40C6C00005E0F2F7F5F808B1062400E0042402E000BF072400BF00BF204610BD10B503F03BFC18B101208D49087002E000208B49087010BD01208C490870704700208B49BC
:40C700000870704789480078704710B5824948683DF019F910BD70B50446002500BF3C2221468348FBF728FD40B9204674F0E0FC461C324621467F4874F050FD00BF2846FF
:40C7400070BD70B50446002500BF3C22214678487838FBF711FD48B9204674F0C9FC461C324621467348783874F038FD00BF9E20EBF7AAFE284670BD2DE9FF4704464FF0A8
:40C7800000093DF05CFA002605463DF011FAB0460746204674F0ACFC00F0FF0A0123402251462046CDE90078CDE902560DF041F901281BD10220604908702046FFF7C1FF2C
:40C7C000012004F068FBA220EBF77EFE4FF4D0703EF0DEF8204674F08BFC05462346032221210090002062F0CAF924E03DF027FA002605463DF0DCF9B0460746204674F017
:40C8000077FC00F0FF0A0123402251462046CDE90078CDE902560DF00CF9022803D12046FFF779FF07E09E20EBF74EFE0120424908704FF0FF39484604B0BDE8F08770B508
:40C8400004460D4630222946204674F03EFD05223A49204674F08AFD2D20607104223749891DA01D74F082FD2D20A0720C2233490B3104F10B0074F079FD0020E07570BD8F
:40C8800000B587B0182101A8FFF7D9FF01A8FFF773FF07B000BD2848007870472DE9F04781460F461446C8460025484674F020FC08B9A8462BE000260FE02D21404674F0AD
:40C8C000ABFB054625B9022E01DA4FF0000806E0BE4201DA05F10108761CBE42EDDD00BFB8F1000F09D01DB1A5EB0800207006E0404674F0FDFB207001E000202070207834
:40C900000C2801DC207810B94FF0000800244046BDE8F0878B6C4F41A41F0010C5020020B01F0010FC0B0010C6020020C7020020FC01006894260020C40200208C1F001090
:40C9400001B500BF04226946FE48FBF715FC18B9FD490098C1F8FC0000BF08BD1CB53CF0B7FFB0F57A7F19D93CF0B2FF4EF66021884205D963F0B1FE044663F0B1FE02E07F
:40C98000012063F0ADFE002063F066FE00200090034601220146019062F014F81CBD70B504460D46002620790A2810DB002020716079401C60710DB1FFF7D0FF60793C2841
:40C9C00005DB002060712068401C00B10126304670BD01B500BF04226946DA48E838FBF7CBFB10B9D8490098486100BF08BD01B500BF04226946D348EC38FBF7BDFB10B918
:40CA0000D1490098086100BF08BD01B500BF04226946CE48FBF7B0FB18B9CB490098C1F82C0300BF08BD01B500BF04226946C548F038FBF7A1FB10B9C3490098C86000BF10
:40CA400008BD10B52DED028B04469FEDC10AB0EE408AC0480078844212D1BE4800783DF077FC00EE100AB8EE400ADFEDBB0A20EE200AF7EE000A80EE201AB0EE418A2CE068
:40CA8000B6480078844212D1B44800783DF060FC00EE100AB8EE400ADFEDAF0A20EE200AF7EE000A80EE201AB0EE418A15E0AC480078844211D1AA4800783DF049FC00EED2
:40CAC000100AB8EE400ADFEDA40A20EE200ADFEDA50A80EE201AB0EE418AB0EE480ABDEC028B10BD10B52DED028B04469FED980AB0EE408A9C480078844212D19A48007850
:40CB00003DF026FC00EE100AB8EE400ADFED920A20EE200ADFED950A80EE201AB0EE418A5EE09348007884421AD1914800783DF00FFC00EE100AB8EE400AB0EE408ADFED9B
:40CB4000860A9FED8C0A18EE200A9FED8B1AC0EE010A9FED8A0A30EE800AB0EE408A3FE08748007884420ED1854800783DF0F0FB00EE100AB8EE400ADFED770A20EE200AD4
:40CB8000B0EE408A2CE07F480078844212D17D4800783DF0DDFB00EE100AB8EE400ADFED6E0A20EE200AF5EE000A80EE201AB0EE418A15E06A480078844211D16848007876
:40CBC0003DF0C6FB00EE100AB8EE400ADFED620A20EE200AF5EE000A80EE201AB0EE418AB0EE480ABDEC028B10BD10B52DED028B04469FED570AF0EE408A634800788442BA
:40CC00001ED1614800783DF0A3FB00EE100AB8EE400ADFED510A20EE200AB0EE408A9FED5B0A38EE400AF0EE040A80EE201AB0EE418AB3EE090A38EE000AF0EE408A19E077
:40CC400047480078844215D1454800783DF080FB00EE100AB8EE400ADFED3F0A20EE208A9FED4B0A30EE480AF1EE060A80EE201AF0EE418AB0EE680ABDEC028B10BD45495D
:40CC8000087070472DED028B4FF6FF76DFF808C100DF81466422494601203CF0F8FEDFF8F8C000DF8146494601203CF01FFF3CF00FFE804639480021016041603848016093
:40CCC00041603848016041603748016041603748016041603CF0FCFD87B21B4840692F4908601948C0682E490860174800692D4908601548D0F82C032B4908601248D0F865
:40CD0000FC002A4908603CF0E3FD294908600120284908700220284908703CF0D9FD274908600121264800783DF005F90021254800783DF000F90121234800783DF0FBF8C3
:40CD4000002043E0FC000068982400202C030068000000000406002000404E3F030600201F060020FC7C5740010600209893823D0206002000E0AB44A470A5C000005CC286
:40CD80003E0600203F0600203D06002000003E4400F809455D0100102D7A090898000010B0000010A8000010A0000010B8000010580100105C010010540100105001001025
:40CDC000320600203306002034060020F249087000BF002231460120DFF8C0C300DF0446012CF6D0022CF4D1DFF8B4C300DF054605F00100002838D0EA480079401CE949BC
:40CE00000871E9480079401CE7490871FFF7BFFB40B9FFF7E3FB28B9FFF7D3FB10B9FFF7C3FB48B1E1480079401CE0490871E0480079401CDE490871FFF7A9FB40B9FFF76C
:40CE4000CDFB28B9FFF7BDFB10B9FFF7ADFB38B1F5F7B9FC20B1D7480079401CD549087162F014FF08B162F0DDFED34800780128AFD1EFF7C0FC4FF4FA7138463CF042FD4E
:40CE800088B13A20EBF720FB3920EBF71DFB3820EBF71AFB8720EBF717FB4620EBF714FB3CF016FD87B226F0B9FE18B13CF010FD804608E04EF6602140463CF023FD10B101
:40CEC0000120FFF7DCFE01203DF079FC012037F0F4F9BA480078FFF705FEB0EE408A0A21B7480DF08EF8B74880ED000A002037F0E4F9B5480078FFF7F5FDB0EE408A0A2137
:40CF0000B2480DF07EF8B24880ED000AB1480078FFF7E8FDB0EE408A0A21AF480DF071F8AE4880ED000AAE480078FFF75EFEB0EE408A0A21AB480DF064F8AB4880ED000A61
:40CF40003CF09BFF00287BD0A8480078FFF779FDB0EE408A3221A6480DF053F8A54880ED000AA5480078FFF76CFDB0EE408A3221A2480DF046F8A24880ED000A4320EBF705
:40CF8000A3FAA048007802282BD19F480078FFF72CFEB0EE408A06219C480DF032F89C4880ED000A4FF496719A4800683CF0AAFC002872D00420934908703CF089FC954903
:40CFC00008600121944800783CF0B5FF0121934800783CF0B0FF0121914800783CF0ABFF5BE08848007804282BD187480078FFF779FDB0EE408A06218A480DF002F88A4852
:40D0000080ED000A4FF49671824800683CF07AFCF0B301207B4908703CF05AFC7D49086001217D4800783CF086FF00217B4800783CF081FF00217A4800783CF07CFF2CE085
:40D0400044E071480078FFF7FCFCB0EE408A062176480CF0D6FF764880ED000A4FF496716C4800683CF04EFC90B10220654908703CF02EFC674908600121674800783CF0D2
:40D080005AFF0021654800783CF055FF012100E003E0634800783CF04EFF3DF082FB20B13CF016FC6349086010E043F69821614800683CF027FC48B101215F4800783CF05B
:40D0C0003AFF01215D4800783CF035FF01213548FFF765FC01280DD132490968491C314A08461160FFF79FFC1920EBF7EDF916202AF072FE00212C48FFF751FC012807D1A5
:40D1000029490968491C284A08461160FFF77DFC00212648FFF743FC012807D123490968491C224A08461160FFF761FC00212048FFF735FC012807D11D490968491C1C4A2F
:40D1400008461160FFF745FC00211A48FFF727FC01287FF43EAE17490968491C154A08461160FFF7EDFB34E603468B4201DB934201DD012070470020FCE70748007870474B
:40D1800000B5FFF7FAFF022801D0012000E000200146084600BD00005D010010916D0908D96C0908B0000010A0000010A800001098000010B8000010CC0200203F0600209F
:40D1C000DC0000101C0100103E060020D40000102001001002060020C4000010180100103D060020F40000102C01001004060020CC0000102401001003060020E40000107C
:40D2000028010010540100101F0600200C0100103401001050010010320600203306002034060020FC000010380100100401001030010010C00000102D0600202E0600201B
:40D2400058B1FC4991F87B17012904D100EB4001F94A517201E0F84A5072704701B500BF04226946F5480068001DFAF785FF20B99DF80010EF48C0F83C1300BF08BD10B5F2
:40D28000EF48D0F854110220DFF8B8C300DFEC48016D0220DFF8ACC300DFF7F71AFC6320EBF712F910BD10B5FFF7E9FFE14890F88E030A2801D110F076FC10BDDD4890F8B8
:40D2C0003803704701B5FFF7F9FF9DF8001088420DD000BF04226946D8480068FAF74CFF20B99DF80000D349C1F8380300BF08BDD54A1278D44B5A701A46107091707047C8
:40D3000038B5CD484078402802D0CB2850D111E000210620FFF7ECFFC7480079032808D1CB20C54948706A20EBF7CEF82620EBF7CBF83EE0BF4890F87B07012803D1FB202B
:40D34000FFF7C0FF02E0FA20FFF7BCFFBC48D0F868111020DFF8ECC200DF0020B6494870FFF7A1FFFEF7B9FC0446FEF77AFB054622461521FEF779FB00212020EFF776FF99
:40D38000F5F791FA40B9F5F777FA28B9F5F784FA10B9F5F779FA50B1AC4800680090AC4802220321036840F276202FF00BFC00E000BF00BF38BD10B59F4840783F282DD18F
:40D3C0009D480079012806D09B484079012810D1A048007868B90120974948719E4800680E2102689448904700210846FFF780FF13E091480079022802D09648007860B9C1
:40D4000002208D49487194480068112102688A48904700210620FFF76BFF00E000BF00BF10BD00208D4908707047014600208B4A1278012A04D0012902D1884A117007E0BF
:40D44000864A1278012A03D111B9844A11700120704770B50024F6F7D6FC30B16CF0CAF90546FFF7E2FF044613E0F6F7E8F850B16CF0C7F908B1012000E000200546FFF7F6
:40D48000D4FF044605E06CF07DF90546FFF7CDFF0446204670BD38B5674840783C2876D008DC38280FD0392851D03A2870D03B286FD1D9E03D286DD03E286CD0D3286BD093
:40D4C000E328F5D143E25C48007901280DD0594890F88E030A2812D0564890F87C0317280DD155484079012809D10120524948713520487000210846FFF7FAFE26E04E48AF
:40D500000079022809D04B4890F88E030A280ED0484890F87C03172809D10220464948713B20487000210220FFF7E2FE0EE04248007904280AD102203F4948713920487001
:40D5400000210220FFF7D4FE69F0D1F80EE23A480079012808D1384948713820487000210846FFF7C5FE2BE033480079022814D1314948713A2048700021BFEE000A0C20C8
:40D5800069F0F1F800210520FFF7B2FE18E077E017E0EAE1C7E053E1BEE1F5F77DF920B1244890F88E030A280AD102202249487101202B490870F8F7EBFE3E201E49487045
:40D5C000D4E11D48007904280FD101201A4948713920487000210846FFF78AFE00219FED210A084669F0BFF822E069F0B6FC03280BD1022010494871012019490870F8F7E9
:40D60000C7FE3E200C49487012E069F0A6FC01280ED1022008494871E320487000210520FFF766FE00219FED0F0A084669F09BF89CE1000098240020B01F00108400001072
:40D6400030320020316D090870010010880400208404002091010010800100108E010010930100100000000067F0E6FB67F039FCFFF7D7FE0220F84948713C20487075E119
:40D68000F5480079022802D0FFF7E3FEF8B167F0CEFB032803D067F0CAFB022802D167F020FC05E067F0C3FB012801D167F0C4FBFFF7B7FE0220E849487167F0F9FB3D2024
:40D6C000E549487000210720FFF712FE2AE0E2480079012808D1E04948713820487000210846FFF705FE1DE0DB480079042802D0F4F7F2FB70B1D848C07901280AD10220DE
:40D70000D549C871D548D0F868114020DFF850C300DF07E067F08BFB042803D165F0DAFEFFF77FFE22E16CF02DF80446FFF77DFE90B165F0CFFE3C20C74948700846C0795A
:40D74000012804D100210520FFF7D2FD77E000210220FFF7CDFD72E0F4F7BEFB30B9C14890F8D80010B9F5F7F9FEA8B1F5F79BF840B9F5F781F828B9F5F78EF810B9F5F714
:40D7800083F848B10120B4494871D320487000210520FFF7ADFD52E067F049FB022803D067F045FB01280BD10120AB494871D320487000210520FFF79BFD65F08BFE3EE0DE
:40D7C00067F035FB032815D10220A34948713E2048700020A44908709F48C079012804D100210320FFF784FD29E000210846FFF77FFD24E067F01BFB08BB9C4800780428B0
:40D800001DD168F03BFD80B93C20934948700846C079012804D100210520FFF769FD0BE000210220FFF764FD06E0D3208A49487000210520FFF75CFD01208749487195E07D
:40D840008548407901280CD18748007848B10120814948713820487000210846FFF748FD2AE07D480079022802D07F48007818B3F5F719F840B9F4F7FFFF28B9F5F70CF880
:40D8800010B9F5F701F850B1794800680090794803221146036840F276202FF093F902206D494871744800680F2102686A48904700210846FFF71CFD6748C07901280ED19F
:40D8C0006548007903280AD102206349C8716348D0F868114020DFF888C100DF1BE05E480079012817D167F0A7FA67F0FAFAFFF798FD0120584948713C2048700846C0799B
:40D90000012804D100210520FFF7F2FC03E000210220FFF7EDFC29E04F480079042815D1FFF77FFD01204C4948713C2048700846C079012804D100210520FFF7D9FC03E021
:40D9400000210220FFF7D4FC67F076FA0EE042480079042808D101203F4948713920487000210220FFF7C4FC00E000BF00BF67F05EFA3E49087038BD10B53748407834281C
:40D9800069D00CDC2B2879D004DC1F2810D02A2875D126E0322873D03328F9D1EEE035286FD0D4286ED0D5286DD0D628F0D192E129484079012808D1274948712E48006800
:40D9C0000C210268244890470AE0FFF72AFD70F066FD2A202049487000210220FFF788FC8CE11D480079022805D1002140F6D83060F0B1FE28B96BF0C5FE0446FFF715FD61
:40DA0000E0B1022014494871F5F719FE40B9F6F7E2F928B9F5F790FE10B9F5F785FE18B132200D49487002E02B200B494870FFF7F8FC00210220FFF75BFC2CE00648007917
:40DA4000012821D1044948711F20487000210846FFF74EFC1FE0CBE0B01F001030320020316D0908C81C002093010010840100108804002084040020800100100CE03AE1FC
:40DA80002EE0E8E007E116E1FB48007818B100210846FFF72DFC31E16AF0CFFC08B1012000E000200446FFF7C0FC48B10220F34948713220487000210220FFF719FC0EE03C
:40DAC000EE48007901280AD1EC494871FFF7A9FC2A20EA49487000210846FFF709FC0DE1E6480079022811D13DF011F80446002160F031FE50B100BF0220E0494871332073
:40DB0000487000210220FFF7F3FB36E0DB480079012818D1D9494871F5F791FD28B9F6F75AF910B9F5F708FE18B12A20D349487002E02B20D1494870FFF773FC0021084657
:40DB4000FFF7D6FB19E06EF0AFFC48B100210520FFF7CEFBD420C9494870012048710CE0C74890F8500500F0020030B1C548D0F868110420DFF810C300DFBFE0BF48007981
:40DB8000022809D100BFBD4948713420487000210220FFF7ADFB2AE0B848007901280CD1B64948713220487070F082FC70F08CFC00210220FFF79CFB19E06EF075FC48B154
:40DBC00000210520FFF794FBD520AC494870012048710CE0AA4890F8500500F0080030B1A848D0F868110420DFF89CC200DF85E0A2480079022809D100BFA049487135205F
:40DC0000487000210846FFF773FB23E09B48007901280CD1994948713320487070F054FC70F05EFC00210220FFF762FB12E06EF03BFC28B1D620914948700120487109E0A3
:40DC40006EF0C4FE30B18F48D0F868110420DFF838C200DF52E08948007902280CD100BF8649487138204870002066F0C7FA00210846FFF73DFB0DE080480079012809D1D8
:40DC80007E4948713420487070F02AFC00210220FFF72EFB32E07948007904280AD170F017F90120754948713220487000210220FFF71EFB22E07148007904280AD170F09E
:40DCC00007F901206D4948713320487000210220FFF70EFB12E06948007904280AD170F0F7F80120654948713420487000210220FFF7FEFA02E0FFF7CEFB00BF00BF10BD24
:40DD000010B55E484078352878D006DC32280BD0332848D0342872D182E0D42870D0D5286FD0D628F7D1FCE054480079022810D13CF0EDFE0446002160F00DFD48B102205F
:40DD40004E4948713320487000210220FFF7D0FA28E04A48007901280AD14849487126204870FFF75EFB00210846FFF7C1FA19E06EF09AFB48B100210520FFF7B9FAD420AF
:40DD80003E494870012048710CE03D4890F8500500F0020030B13B48D0F868110420DFF8E8C000DFCEE035480079022808D1334948713420487000210220FFF799FA2EE021
:40DDC0002E48007901280CD12C4948713220487070F06EFB70F078FB00210220FFF788FA1DE06EF061FB68B100210520FFF780FAD520224948700120487110E051E0A0E086
:40DE00006FE07EE01E4890F8500500F0080030B11C48D0F868110420DFF86CC000DF91E016480079022808D1144948713520487000210846FFF75CFA32E010480079012839
:40DE40000CD10E4948713320487070F03DFB70F047FB00210846FFF74BFA21E06EF024FBA0B1D620054948700120487100210520FFF73EFA14E000007D010010B01F00104C
:40DE80009824002030320020316D09086EF09EFD30B1FE48D0F868110420DFF8F4C300DF50E0FC48007902280CD1FA494871FA4800680F210268F748904700210846FFF7B4
:40DEC00017FA0DE0F3480079012809D1F14948713420487070F004FB00210220FFF708FA30E0EC48007904280AD16FF0F1FF0120E84948713220487000210220FFF7F8F982
:40DF000020E0E448007904280AD16FF0E1FF0120E04948713320487000210220FFF7E8F910E0DC48007904280AD16FF0D1FF0120D84948713420487000210220FFF7D8F9FA
:40DF400000E000BF00BF10BD10B5D2484078D92838D006DC28280BD0D42877D0D62830D1CEE0DA2874D0DB2842D0DC28F7D185E0C8480079012808D0C84890F87C0317286D
:40DF80000DD0C4484079012809D10120C14948712220487000210846FFF7AAF911E0BD480079022804D0BD4890F87C03172808D00220B8494871D920487000210846FFF754
:40DFC00097F9ADE0B3480079022808D1B1494871DB20487000210220FFF78AF907E0AD480079012803D1AB4948712820487097E0A8480079022808D1A6494871DA2048702F
:40E0000000210846FFF774F91FE0A2480079012808D1A0494871D920487000210846FFF767F912E06EF040FA28B1D420994948700120487109E0994890F8500500F002002E
:40E0400018B100210846FFF753F969E048E0FFE790480079022808D18E494871DC20487000210220FFF744F907E08A480079012803D188494871DB20487051E085480079DE
:40E0800002280CD183494871834800680F2102688048904700210846FFF72AF91FE07D480079012808D17B494871DA20487000210846FFF71DF912E06EF0F6F928B1D620E9
:40E0C000744948700120487109E0744890F8500500F0200018B100210846FFF709F91FE06C48007904280AD16FF0F2FE012069494871DB20487000210220FFF7F9F80FE035
:40E100006448007904280AD16FF0E2FE012061494871DC20487000210220FFF7E9F800BF00BF10BD38B55B484078262874D006DC1F280BD0212839D022286ED170E028287E
:40E140006CD02A286BD0D728F7D1B2E051484079012803D04F480079012809D101204D4948714D4800680C2102684A4890471CE06AF089FED52809D1022046494871212050
:40E18000487000210846FFF7B3F80EE06AF07BFED6280AD0424800680090424801220321036840F276202EF00DFD24E13948007901280DD0394890F87C03172804D1374830
:40E1C00090F8840301280DD132484079012809D10120304948711F20487000210846FFF787F818E02B480079022809D02B4890F87C03172804D1294890F8840301280AD1AC
:40E200000220244948712220487000210846FFF76FF868F06CFAEEE087E0E3E059E0ABE01C480079022809D128201A4948700220487100210846FFF75BF839E068F08DFE83
:40E24000022803D068F089FE01280FD1012011494871D720487001210020FFF749F800219FED110A084668F07EFA21E009480079012803D007480079042819D10120054963
:40E28000487121204870002108460FE030320020316D0908B01F00108001001098240020880400208404002000000000FFF720F8A1E0FD48007904280AD12220FA494870EC
:40E2C0000220487100210846FFF712F868F00FFA00BFF5480079012808D0F44890F87C0317280FD0F048407901280BD10120EE4948712220487000210846FEF7F9FF68F0E7
:40E30000F6F911E0E8480079022804D0E74890F87C03172808D00220E34948712620487000210846FEF7E4FF65E0DF480079012808D1DD4948712820487000210846FEF793
:40E34000D7FF18E0D8480079022814D1FF200090D64890F88313FF2303222620EDF713F8FFF75FF80220D04948712A20487000210220FEF7BDFF3EE0CB480079022805D1DF
:40E38000002140F6D83060F0E6F950B96BF0FAF90446FFF74AF820B9C44890F8860301280BD170F07CF80220BF4948713220487000210220FEF79CFF13E0BB4800790128CF
:40E3C00008D1B94948712620487000210846FEF78FFF06E0B648007818B100210846FEF787FF08E0F7F7E5F810B1FFF7ADFD01E0FFF786FC00BF00BF38BD38B5AA48407813
:40E40000332879D012DC2D2877D008DC1F281ED0212833D029285BD02C286FD1ADE02E286DD030286CD03228F7D127E13E2868D006DC34287BD036287AD03728EDD1F4E19A
